:1080000000000120DD6B0200213702002137020051
:108010002137020021370200213702000000000052
:1080200000000000000000000000000021370200F6
:10803000213702000000000021370200C1C1010009
:1080400021370200213702002137020021370200C8
:1080500021370200213702002137020021370200B8
:1080600021370200213702002137020021370200A8
:108070002137020021370200213702002137020098
:108080002137020021370200213702002137020088
:108090002137020021370200213702002137020078
:1080A0002137020021370200213702002137020068
:1080B0002137020021370200213702002137020058
:1080C0002137020021370200213702002137020048
:1080D0002137020021370200213702002137020038
:1080E0002137020021370200213702002137020028
:1080F00021370200FDD301002137020021370200A1
:108100002137020091D801002137020021370200F7
:1081100021370200D9D101002137020021370200A6
:1081200021370200213702002137020021370200E7
:1081300021370200213702002137020065EF0100DC
:1081400055E40100213702002137020021370200E7
:1081500021370200213702002137020021370200B7
:1081600021370200A949020021370200213702000D
:108170002137020021370200213702002137020097
:108180002137020021370200213702002137020087
:108190002137020021370200213702002137020077
:1081A000E1E30100213702002137020021370200FC
:0C81B000213702002137020021370200B5
:10840000FFFFFFFFFFFFFFFFFFFFFFFF7EF9FFFF03
:1084200010B5054C237833B9044B13B10448AFF3AE
:1084300000800123237010BD0010FF1F000000000A
:108440005099020008B5034B1BB103490348AFF331
:10845000008008BD000000000410FF1F50990200BA
:1084600038B5064C2368C31AB3F5FA7F054604D322
:10847000034B9B699B699847256038BD1C10FF1F03
:10848000847E020010B516F015F8064B00221A7013
:10849000054B1B689847054B9B69BDE810405B691D
:1084A000184700BFC409FF1FA800FF1F847E0200F9
:1084B000431E2DE9F0471546072B00F24B82DFE8FB
:1084C00013F008000E000E0050006A00BA00F80019
:1084D000B101FFF7D7FF47F6A8532B603FE0A24B4F
:1084E000A24C022816BFA14699461C46A04BDF6845
:1084F000A9F10409043C4FF0FF364FF000084FF09B
:10850000010A3B68D9F804001B6998473B6860681A
:10851000DB6898473B6854F8040F5B6998473B68F1
:1085200059F8040F1B6A984718B90AFA08F326EAA3
:1085300003063B6820689B6998473B68D9F80000B0
:108540001B6A984718B10AFA08F326EA030608F1ED
:108550000108B8F1110FD4D1C6F310062E60002027
:1085600020E0296003291CD8DFE801F0020A0E127E
:108570007F4BDB691B681A88322353431B14ACE71B
:108580007B4BDB695B68F6E7794BDB699B68F2E75D
:10859000784B1B69A1E7012929601CD004D302296B
:1085A0002FD00220BDE8F087714BDC68D4E90030A1
:1085B000DB6864309847D4E90030DB688430984742
:1085C000D4E900305B6964309847D4E900305B69D6
:1085D00084309847C3E7664BDC68D4E90030DB6839
:1085E000C4309847D4E90030DB68A4309847D4E918
:1085F00000305B69C4309847D4E900305B69A4302F
:10860000E7E75B4BDC68D4E90030DB6800F5A2707B
:108610009847D4E90030DB6800F5B2709847D4E998
:1086200000305B6900F5A2709847D4E900305B69BF
:1086300000F5B270CDE70129296025D019D30229B0
:10864000AFD14B4BDC68D4E90030DB6800F5A27099
:108650009847D4E90030DB6800F5B2709847D4E958
:1086600000305B6900F5A2709847D4E900309B693F
:10867000DEE73F4BDC68D4E90030DB6884309847A4
:10868000D4E900301B699EE7394BDC68D4E900303F
:10869000DB68C4309847D4E90030DB68A4309847E1
:1086A000D4E900305B69C4309847D4E900309B6955
:1086B000A5E7296000295FD001297FF472AF2C4B18
:1086C000DC68D4E90030DB6800F2C4609847D4E984
:1086D00000309B6900F2C4609847D4E90030DB6841
:1086E00000F2E4609847D4E900309B6900F2E4604E
:1086F0009847D4E90030DB6800F204709847D4E969
:1087000000309B6900F204709847D4E90030DB68C0
:1087100000F224709847D4E900309B6900F224707D
:108720009847D4E90030DB6800F244709847D4E9F8
:1087300000309B6900F244709847D4E90030DB6850
:1087400000F264709847D4E900309B6900F26470CD
:108750009847D4E90030DB6800F284709847D4E988
:1087600000309B695BE000BF4035FF1F2034FF1FD6
:10877000847E0200C409FF1F774BDD68D5E9003015
:10878000DB6800F2C4609847D5E900305B6900F20D
:10879000C4609847D5E90030DB6800F2E460984790
:1087A000D5E900305B6900F2E4609847D5E9003014
:1087B000DB6800F204709847D5E900305B6900F28D
:1087C00004709847D5E90030DB6800F224709847C0
:1087D000D5E900305B6900F224709847D5E9003094
:1087E000DB6800F244709847D5E900305B6900F21D
:1087F00044709847D5E90030DB6800F26470984710
:10880000D5E900305B6900F264709847D5E9003023
:10881000DB6800F284709847D5E900305B6900F2AC
:108820008470D6E6296000294AD001297FF4B9AEC8
:10883000494BDC68D4E90030DB6800F2845098478B
:10884000D4E900309B6900F284509847D4E90030A5
:10885000DB6800F2A4509847D4E900309B6900F22D
:10886000A4509847D4E90030DB6800F2C450984720
:10887000D4E900309B6900F2C4509847D4E9003035
:10888000DB6800F2E4509847D4E900309B6900F2BD
:10889000E4509847D4E90030DB6800F20460984760
:1088A000D4E900309B6900F204609847D4E90030B5
:1088B000DB6800F224609847D4E900309B6946E009
:1088C000254BDD68D5E90030DB6800F2845098471D
:1088D000D5E900305B6900F284509847D5E9003053
:1088E000DB6800F2A4509847D5E900305B6900F2DC
:1088F000A4509847D5E90030DB6800F2C45098478F
:10890000D5E900305B6900F2C4509847D5E90030E2
:10891000DB6800F2E4509847D5E900305B6900F26B
:10892000E4509847D5E90030DB6800F204609847CE
:10893000D5E900305B6900F204609847D5E9003062
:10894000DB6800F224609847D5E900305B6900F2EB
:1089500024603EE6042025E6847E02003A4B3B4A32
:10896000DB685B6803F59271116003F144015160AB
:1089700003F18401916003F1C401D16003F58271B8
:10898000116103F5B271516103F5D271916103F583
:10899000F271D16103F50971116203F51971516228
:1089A00003F52971916203F53971D16203F54971BB
:1089B000116303F55971516303F56971916303F50F
:1089C0007971D16303F224411164214A191D1160A8
:1089D00003F12401516003F16401916003F1A401EA
:1089E000D16003F1E401116103F5A271516103F556
:1089F000C271916103F5E271D16103F501711162F8
:108A000003F51171516203F52171916203F5317122
:108A1000D16203F54171116303F55171516303F59F
:108A20006171916303F5717103F204431364094B9F
:108A3000D16301221A70084B084A1A65084A9A65E0
:108A4000084A5A65704700BF847E02002034FF1F29
:108A50004035FF1FC409FF1F6434FF1FB1840000AD
:108A60008584000061840000704702207047022066
:108A700070477047704702207047022070470220FD
:108A8000704701207047704770474369124A134985
:108A900010B5C3F80422C3F80822114B8365114BAB
:108AA0008361C0E909131049C361C0E90B130F4B7F
:108AB00043640F4B83640F4B0F4C4363C0E90F3388
:108AC0000E4B0F4A0366002342658463C0E913140A
:108AD000C265836610BD00BF838A00006B8A0000F8
:108AE000698A00006F8A0000778A0000738A00009C
:108AF000758A00007B8A00007F8A0000878A000058
:108B0000898A0000704700BF0A480B4B00220121F0
:108B100010B44FF0FF3480F87C205A7083F81012A4
:108B2000C0E91D41C0F8803002671A706C3010BC7B
:108B3000FFF7ABBF6434FF1F2C10FF1F084A094822
:108B400000234FF0FF314FF0010C1370537082F887
:108B500010324261C0E9021C03744360FFF795BF05
:108B60004C12FF1F6434FF1F10B50023064C18463B
:108B70001A5D590002F0030201338A40072B40EAD4
:108B80000200F5D110BD00BF6C14FF1F0449002383
:108B90005A5C02F00302C2540133072BF8D170472C
:108BA0006C14FF1F074B1A7802705A7842709A783B
:108BB0008270DA78C2701A7902715A7942719B799F
:108BC000837170476C14FF1FF8B5094B094F0A4EAB
:108BD000DD680024E15D726C2B6852F82400DB69CB
:108BE00001F0030101349847072CF3D1F8BD00BF11
:108BF000847E02006C14FF1F0800FF1F054A00233B
:108C000000F0030199540133072B4FEA9000F7D18C
:108C1000DAE700BF6C14FF1F014B586AEEE700BF94
:108C20000800FF1F04490023C25C02F003025A54EB
:108C30000133072BF8D1C7E76C14FF1F074B0278ED
:108C40001A7042785A7082789A70C278DA70027913
:108C50001A7142795A7182799A71B5E76C14FF1FC3
:108C6000014B00221A6770476434FF1F70B50B4E2A
:108C70000B4D33682A4601460446002016F08BFE51
:108C8000002016F05BFA33682A462146012016F0D0
:108C900082FE0120BDE8704016F050BA0438FF1F74
:108CA0008435FF1F012808B503D816F03BFA0020D1
:108CB00008BD0820FCE7012808B503D816F026FAFD
:108CC000002008BD0820FCE70021F4E74942F2E754
:108CD000F1E7024B186816F06EBE00BF0438FF1FA4
:108CE00038B5002016F00AFB08B1002038BD01207D
:108CF00016F004FB05460028F7D10A4B0A4C186809
:108D000016F050FE16F040FB2B46A268216828465C
:108D100016F08AFA01202B46E268616816F084FAA0
:108D20000120E3E70438FF1FA014FF1F022804BF3F
:108D30000B4B93F8D80030B90A4BDB681B685B69B2
:108D4000094A10691847012809D1054B93F8D83012
:108D5000012B04D1034BDB681B689B69F0E770476C
:108D60006434FF1F847E0200A014FF1F70B5002032
:108D7000FFF7DCFF0A4B0B4CDD6820692B689B6812
:108D800098472B68206A9B6898472B68606A9B68A5
:108D9000984716F047FB044BBDE870405B681847E6
:108DA000847E0200A014FF1F7409FF1F012838B53C
:108DB00004460D4605D820B916F0A0FA28602046D2
:108DC00038BD0820FCE7022810B5144610D003284F
:108DD00015D0012817D10D4B0D4ADB68106A1B68AE
:108DE0001B6A9847003018BF01202060002010BD8A
:108DF000064B074ADB68506A1B681B6AF1E70846A6
:108E000016F0F0F9F1E70420F1E700BF847E0200DC
:108E1000A014FF1F012838B504460D4608D816F0E7
:108E200053FA2B68C11829602046BDE8384039E75D
:108E3000082038BD2DE9F843184C9DF820609DF8B6
:108E40002450984623680F469B68002147F0800015
:108E500091469847236800219B68484698472368B5
:108E600000219B6840469847236800219B68304654
:108E70009847236828469B6801219847084B1B6840
:108E800048EA092807F07F0746EA082603EB870728
:108E900045EA06257D60BDE8F88300BF0838FF1F5E
:108EA0000438FF1F07B5D3B20193C2F30723009321
:108EB000C2F30743120EFFF7BDFF03B05DF804FBDA
:108EC0000020FFF7EFBF38B5234B01F07F042344A8
:108ED00093F80032DB0705D4204B1B6803EB8404B6
:108EE000606838BD1E4D2B6800219B68204698475E
:108EF0002B6800219B68084698472B6800219B68D7
:108F0000084698472B6800219B68084698472B68BD
:108F100001219B68002098472B6800219B68204610
:108F200098472B6800219B68084698472B680021CA
:108F300004029B68084698472B68002104439B68FD
:108F4000084698472B68240204439B6801210020AF
:108F5000984724022043C4E78435FF1F0438FF1FCD
:108F60000838FF1F10B500201446FFF7ACFF206043
:108F700010BDA42A2DE9F04104460D461E4600F01E
:108F80008E8149D8062A00F0D98017D8022A00F02D
:108F9000B28007D8002A00F09680012A00F0A18054
:108FA00004249BE0042A00F0B78040F2AE80002841
:108FB00040F0BF80084616F0BDF988E01D2A00F099
:108FC000FC8014D8082A00F0E680C0F0CF801C2A6C
:108FD000E6D10F0147F06C07FFB239462846002C56
:108FE00040F0E280FFF76FFFC0F380406FE0A22AFD
:108FF00000F02B8100F23E818C2AD1D1002840F074
:10900000E080090141F06C0101F0FC012846FFF706
:109010005AFFC0F303605AE0AC2A00F0FE8129D861
:10902000A82A4FEA011700F0B48111D8A62A00F04F
:109030008B8140F2498147F06C07FFB239462846E0
:10904000002C40F0EE81FFF73EFF00F00F003EE005
:10905000AA2A00F0C58140F2AF8147F06D07FFB248
:1090600039462846002C40F0CF81FFF72CFFC0F393
:1090700041102CE0B42A00F0168214D8AE2A00F079
:10908000ED81C0F0D681B32A8AD10F0147F06C0779
:10909000FFB239462846002C40F0FC81FFF713FF51
:1090A000C0F3404013E0B82A00F00F82CE2A00F04F
:1090B0002182B52A7FF474AF002840F0018208466F
:1090C00016F054F903E020B9084616F009F93060AB
:1090D00004E01968284616F025F800242046BDE86B
:1090E000F08118B9084616F0EFF8F0E7196828463D
:1090F00016F0C4F8F1E718B9084616F00DF9E6E7DE
:109100001968284616F002F8E7E700287FF448AF10
:10911000084616F0F3F8DAE718B9084616F018F919
:10912000D5E719680029B8BF4942284616F0B4F8B7
:10913000D3E71968284616F0A6F9CEE720278F4016
:1091400047F01007FFB23946284624B9FFF7BBFEA7
:10915000C0F30420BBE7FFF7B6FE33681B0203F43D
:10916000F85320F4F8521A43394660E020278F4024
:1091700047F01007FFB23946284624B9FFF7A3FE8F
:1091800000F01F00A3E7FFF79EFE336820F01F02E8
:1091900003F01F03E7E700287FF402AF084616F04C
:1091A00021F8C0F3001092E7FFF78DFE33689B04AF
:1091B00003F4802320F48022D5E700287FF4F0AE6A
:1091C000A7E71B68102B3AD00DDC022B33D004DC50
:1091D000012B16D04FF0FF3314E0042B2DD0082BB9
:1091E000F8D105230EE0402B2BD003DC202BF1D14E
:1091F000032307E0802B26D0B3F5807FEAD100233C
:1092000000E008233360336801333FF466AF2C017C
:1092100044F06C04E4B221462846FFF754FE33685C
:109220001B0603F0706320F070621A432146284643
:10923000FFF738FE51E70723E4E70623E2E70423BC
:10924000E0E70223DEE70123DCE70F0147F06C07CC
:10925000FFB23946284624B9FFF735FEC0F3C130C6
:1092600035E7FFF730FE3368DB0303F4C03320F447
:10927000C03278E70F0147F06C07FFB23946284645
:1092800024B9FFF720FEC0F3803020E7FFF71BFE74
:1092900033689B0303F4804320F4804263E70F01AB
:1092A00047F06C07FFB23946284624B9FFF70BFE9A
:1092B000C0F300300BE7FFF706FE33681B0303F42F
:1092C000805320F480524EE747F06C07FFB23946D6
:1092D0002846FFF7F8FD3946804600F480432846CB
:1092E00084B923B1FFF7EFFDC0F3C310EFE6FFF73A
:1092F000EAFD18F4006FC0F3021018BF40F0080038
:109300003060EAE643B1FFF7DEFD3368DB0103F4CA
:10931000F06320F4F06226E7FFF7D5FD3268120112
:1093200020F0700002F07002024339462846FFF731
:10933000B9FD39462846FFF7C6FD33681B0203F422
:10934000006320F400620EE747F06C07FFB2394675
:109350002846FFF7B8FD394600F48048284664B92E
:10936000B8F1000F04D0FFF7AEFDC0F30210AEE677
:10937000FFF7A9FDC0F3C310C2E7B8F1000FC2D0D8
:10938000FFF7A1FD33681B0103F0700320F07002AA
:10939000E9E647F06D07FFB23946284624B9FFF7E2
:1093A00092FDC0F3C03092E6FFF78DFD3368DB031A
:1093B0009BB220F40042D6E647F06D07FFB2394673
:1093C000284624B9FFF77FFDC0F341307FE6FFF761
:1093D0007AFD33685B0303F4C04320F4C042C2E665
:1093E00047F06D07FFB23946284624B9FFF76BFDF9
:1093F000C0F303206BE6FFF766FD33681B0203F43E
:10940000706320F47062AEE6FFF75DFD33685B01C8
:1094100003F0600320F06002A5E60F0147F06D073E
:109420000BE6FFF750FD336820F00F0203F00F0347
:1094300099E60F0147F06D07FFB23946284624B977
:10944000FFF741FDC0F3006041E6FFF73CFD3368E4
:109450001B0603F0807320F0807284E60F0147F052
:109460006D07FFB2394628465CB9FFF72CFD0014A2
:1094700000F07F0310F0400018BF6FF07F0018432A
:1094800025E6FFF720FD33681B0403F4FE0320F4F8
:10949000FE0268E6FFF717FD33685B0403F4003350
:1094A00020F400325FE600287FF47AAD090141F034
:1094B0006F01C9B22846FFF706FDC0F3044006E677
:1094C0001968284615F0F2FE07E60F0147F06C0711
:1094D000FFB23946284624B9FFF7F5FCC0F3403007
:1094E000F5E5FFF7F0FC33685B0303F4005320F469
:1094F000005238E600287FF453AD090141F06F01B6
:10950000C9B22846FFF7DFFCC0F30900DFE507B565
:109510000129019207D8024601AB0120FFF729FD7E
:1095200003B05DF804FB0820FAE70129134602D8CE
:10953000024600201DE50820704770B54E4E4F488A
:109540004F4C16F0F5F9F5686B6803F1640222617F
:1095500003F1E402626203F58272226203F5A272F1
:10956000A26003F5B27203F59270626003F5C272F5
:1095700003F50173A3622B68E260DB682060984703
:109580002B68A068DB6898472B686068DB689847A1
:109590002B68E068DB6898472B682069DB68984790
:1095A0002B68A06ADB68374D98473369364A03F168
:1095B00014011160A26A9A61344B354A1A6015F0A1
:1095C000E3FE0023A2682168184615F02DFEE2682C
:1095D00061680023012015F027FE2E4B2E49D3F899
:1095E0008020C2F804122D49C2F80812002401217B
:1095F000117054702A4AC3F88C202A4AC3F8882074
:10960000294AC3F88420294AC3F89020284AC3F87D
:10961000A420284AC3F8A020274AC3F89420274A48
:10962000C3F89820264AC3F8B420264AC3F8B020CD
:10963000254AC3F8C020254AC3F8BC20244AC3F8F1
:10964000B820244AC3F8CC20234AC3F8C8203221CA
:109650004FF48F720220C3E91D21204A83F87C0059
:10966000C3F8C420FFF762FB2B689847AB6820461D
:10967000BDE87040184700BF847E02008435FF1F9C
:10968000A014FF1F7409FF1F0838FF1F0438FF1FB5
:109690002C10FF1F6434FF1FE18C0000D38C0000EE
:1096A000B78C0000D18C0000CD8C0000C98C00006C
:1096B0002B9500000F950000A58C0000158E000072
:1096C000C18E0000658F00006D8C0000C78D00000A
:1096D000AD8D00002D8D0000618C00006D8D0000AF
:1096E000014B1046DB6B18470800FF1F034B10B5FA
:1096F0001B6C14469847206010BD00BF0800FF1F78
:10970000062873B504460E467BD8404D68462B6B41
:10971000013C98472B46042C04D8DFE804F0086687
:10972000696C6F009DF80030336000200BE09DF8FD
:109730000120E978914208D19DF80200297B8842F6
:1097400003D10020306002B070BD1979914206D17A
:109750009DF80200597B884201D10123E4E7597941
:10976000914206D19DF80200997B884201D10223E3
:10977000DAE79979914206D19DF80200D97B8842B7
:1097800001D10323D0E7D979914206D19DF8020097
:10979000197C884201D10423C6E7597A914206D147
:1097A0009DF80200997C884201D10523BCE7997A93
:1097B000914206D19DF80200D97C884201D106234E
:1097C000B2E7197A914206D19DF80200597C88428D
:1097D00001D10723A8E7D97A914214D19DF802203C
:1097E0001B7D9A420FD108239EE79DF803309BE72B
:1097F0009DF8043098E79DF8053095E79DF8063010
:1098000092E704209FE710209DE700BF0800FF1F9C
:1098100007B5034B68461B6B984703B05DF804FB24
:109820000800FF1F70B50020FFF7F2FF1E4B1F4C12
:10983000DD68206B2B689B6898472B68E06A9B6803
:1098400098472B68E0689B6898472B68A0689B68DE
:1098500098472B6860689B6898472B6820689B68CE
:1098600098472B68A0699B6898472B68E0699B68BC
:1098700098472B68A06A9B6898472B6860699B682B
:1098800098472B68206A9B6898472B68606A9B689A
:1098900098472B6820699B68984715F0C3FD044BD7
:1098A000BDE870405B681847847E0200D814FF1F33
:1098B0007409FF1F002015F041BC10B5044618B90B
:1098C00015F030FC204610BD0820FCE710B504461A
:1098D00018B915F01BFC204610BD0820FCE700213C
:1098E000F4E74942F2E7F1E7062873B505460C466E
:1098F0005DD8022903D901285BD10F2959DC2E4EEE
:109900006846336B98473346052D06D8DFE805F0E7
:10991000030B4346494C8DF800406846DB6A984784
:10992000002002B070BD082CF7D8DFE804F0050C69
:1099300011161B20252A2F00F2788DF80120327B8A
:109940008DF80220E9E732798DF80120727BF7E784
:1099500072798DF80120B27BF2E7B2798DF801209F
:10996000F27BEDE7F2798DF80120327CE8E7727A3C
:109970008DF80120B27CE3E7B27A8DF80120F27C09
:10998000DEE7327A8DF80120727CD9E7F27A8DF821
:109990000120327DD4E78DF80340BEE78DF8044006
:1099A000BBE78DF80540B8E78DF80640B5E7042021
:1099B000B7E71020B5E700BF0800FF1F38B5154610
:1099C00018B1012807D0042004E0084615F00AFC6D
:1099D0002860002038BD094B094DDC68094B6068E0
:1099E00000F59270D8616B6C58612368DB6898470A
:1099F0006A6C236850699B699847EAE7847E020095
:109A00000800FF1FD814FF1F38B50D46044648B99B
:109A100015F05AFC2B68C1182960204615F082FB0E
:109A2000204638BD0820FCE710B51446002947D170
:109A3000132847D8DFE800F00A1014181C2024244B
:109A4000242424242C373E3E3E3E3E3E002015F08A
:109A500047FC2060002010BD002015F035FCF8E721
:109A6000002015F059FCF4E7002015F047FCF0E762
:109A7000002015F06DFCECE7002015F05BFCE8E73A
:109A800008281FD1002015F0ADFBC0F30010E0E75F
:109A90000D4B0E4ADB68D06A1B681B6A9847003082
:109AA00018BF0120D5E7084B084ADB68106B1B681C
:109AB0001B6AF3E70E381146C0B2FFF721FEC9E773
:109AC0000820C8E70420C6E7847E0200D814FF1FE0
:109AD00030B585B0054601920C4600295FD10B28B0
:109AE00012D8062845D2022836D004D840B301281F
:109AF0002BD004242DE0042833D00528F9D11146B9
:109B0000204615F0C0FC24E013280ED80E2844D2BD
:109B10000C2835D00D28ECD142F210739A42E8D8C7
:109B2000204B90B29B68984713E08C28E1D101A9A3
:109B30000120FFF7E5FD1C4B04469B6B02A827E0C4
:109B4000114615F0EFFA2C4603E01146204615F0B9
:109B500095FB204605B030BD1146204615F0D6FADB
:109B6000F7E782EAE271A1EBE271204615F094FB7F
:109B7000EFE706381146C0B2FFF7B6FE0446E8E745
:109B80000A4B0B49DB68C86A1B68154612B15B6952
:109B90009847DEE79B699847D5E70E38EAE708243F
:109BA000D7E700BF7409FF1F0800FF1F847E020073
:109BB000D814FF1F6B4B2DE9F041DE686A4C7068CA
:109BC0006A4F00F5E273236300F5D273E36200F598
:109BD0002173E36000F52973A36000F519736360D6
:109BE00000F50173236000F55973A36100F551730B
:109BF000E36100F16403A36200F5A273636100F501
:109C00006973236200F571736362336800F59270C3
:109C1000DB682061984733686069DB689847336880
:109C2000206BDB6898473368E06ADB6898473368E5
:109C3000206A1B6998473368606A1B6998477B6C88
:109C4000E2681A60A2685A6062689A602268DA6004
:109C5000A2691A61E2695A61A26A9A6100257A6C66
:109C600033685059DB6898477A6C336850599B6960
:109C7000043598471C2DF2D13D4DD5F880304FF07A
:109C8000000883F8008015F07FFBD4E904124346F6
:109C9000404615F0C9FA44F62061404615F0FCFA3A
:109CA00046F2A811404615F0EEFB324BC5F88C3059
:109CB000314BC5F88830314BC5F88430304BC5F88E
:109CC0009030304BC5F8A4302F4BC5F8A0302F4B47
:109CD000C5F894302E4BC5F898302E4BC5F8B430EB
:109CE0002D4BC5F8B0302D4BC5F8BC302C4BC5F80A
:109CF000C0302C4BC5F8CC30012385F87C300220D5
:109D0000294BC5F8C430FFF783FD404615F0F6FA3D
:109D100010B1264B9B789BB1BB6A984715F034FB7A
:109D20000023D4E90412184615F07EFA44F62061A7
:109D3000002015F0B1FA46F2A811002015F0A3FB9F
:109D40003368206BDB689847206B194C04234375FC
:109D500033681B68984723689847A3680020BDE8CC
:109D6000F0411847847E0200D814FF1F0800FF1F2F
:109D70006434FF1FCD980000E7980000E3980000CE
:109D8000DF980000299A0000D19A0000BB980000DB
:109D9000099A0000E1960000ED960000BD990000D0
:109DA000B59800001198000025980000C409FF1F15
:109DB0007409FF1F1B4B70B5DD681B4C2B68A06836
:109DC0005B6998472B6820689B6898472B68606898
:109DD0009B6898472B68206A9B6898472B68606A45
:109DE0009B6898472B68E0689B6898472B682069B8
:109DF0009B6898472B6860699B6898472B68A069A7
:109E00009B6898472B68E0699B6898472B68A06817
:109E10009B68984715F006FB044BBDE870405B68F3
:109E2000184700BF847E02001815FF1F7409FF1F2A
:109E300010B5144605284BD8DFE800F003211F3089
:109E40003B40146844F620639C4243D8224B234A8B
:109E5000DB68106A1B6842F210718C42DB6994BFA8
:109E600000210121984742F21173B4FBF3F003FB88
:109E700010401B4B80B29B689847002010BD164BCA
:109E80002468DA68D2E9003000F5F2701CB1DB69B1
:109E900000219847F1E79B689847EEE70E4B116861
:109EA000DB680E4A1B681069DB69003118BF0121AD
:109EB000EFE7084615F096F92060DEE7064B074A03
:109EC000DB6858681B6800F592701061DB68E3E797
:109ED0000420D3E71020D1E7847E02001815FF1F6D
:109EE0007409FF1F10B50348144615F0AEFD20603D
:109EF00010BD00BF0C38FF1F014815F098BD00BF12
:109F00000C38FF1F10B5044618B915F00BF92046A0
:109F100010BD0820FCE710B5044618B915F0F6F896
:109F2000204610BD0820FCE70021F4E74942F2E793
:109F3000F1E7014815F0DFBD0C38FF1F022804BF10
:109F40000B4B93F8D80030B90A4BDB681B685B6990
:109F5000094A90681847012809D1054B93F8D83071
:109F6000012B04D1034BDB681B689B69F0E770474A
:109F70006434FF1F847E02001815FF1F38B50D469C
:109F8000044620B915F0BAF92860204638BD0820EB
:109F9000FCE710B501460D4815F0C6FD002015F090
:109FA000CDF8002015F01EF910F008040DD182063E
:109FB0000BD56F21054815F048FDC30105D5204696
:109FC0000221BDE8104015F0E5B810BD0C38FF1FA8
:109FD000012903D1024A702115F029BD704700BF45
:109FE000C8040500A62970B50446154600F07D8218
:109FF0007DD8172900F06B812DD8042900F02A8123
:10A000000CD8012900F00C81C0F0FF80022900F07B
:10A010001081032900F017810424E2E1072900F0F0
:10A020003D810ED8052900F021810629F4D11021A7
:10A03000BC48002C40F0248115F007FDC0F304203B
:10A04000E6E0082900F03A811529E5D10028E3D09F
:10A05000126811211EE11D2900F0F5801CD81A2973
:10A0600000F0578109D81829D6D1002840F04E8138
:10A070003321AC4815F0E9FCCAE01B2900F06181EE
:10A080001C29C9D1002840F06D810146A54815F072
:10A09000DCFCC0F34000BBE0A32900F0C2810ED875
:10A0A0008C2900F06C81A229B6D16C219D48002C2E
:10A0B00040F0AE8115F0C9FCC0F3C130A8E0A4297E
:10A0C00000F0C081A529A7D16C219648002C40F052
:10A0D000DA8115F0BAFC10F4804F4FF06C01914812
:10A0E00000F0C18115F0B1FCC0F3C31090E0B529B8
:10A0F00000F0C1823BD8AB2900F06B8213D8A829AD
:10A1000000F03B82C0F02982A92900F04882AA29E8
:10A1100082D16D218348002C40F0528215F095FCCD
:10A12000C0F3032074E0AE2900F07C820FD8AC2984
:10A1300000F06082AD297FF46FAF6D217948002C6B
:10A1400040F0648215F081FCC0F3006060E0B32948
:10A1500000F08082B4297FF45FAF00287FF45CAF09
:10A160006F21704815F071FCC0F3044050E0BB292A
:10A1700000F0CD8225D8B82900F0978215D8B629ED
:10A180007FF44AAF002840F081821421654815F021
:10A190005CFC002800F078824FF0807393FBF0F0B5
:10A1A000614B9842A8BF184668E1B92900F08E8239
:10A1B000BA297FF431AF5C4E002840F09A82132117
:10A1C00088E0C02900F0E2820FD8BC2900F0BF82ED
:10A1D000BF297FF421AF002840F0C8827021514888
:10A1E00015F033FCC0F3014012E0CC2900F0DE8210
:10A1F000CE297FF411AF00287FF40EAF6F214948BC
:10A2000015F023FCC0F3090002E018B915F068F856
:10A210002860E6E01168002014F084FF0024E0E0EC
:10A2200010B915F051F8F3E71168002015F026F881
:10A23000F4E718B9002015F06FF8E9E7116800207D
:10A2400014F064FFEAE7002C7FF4E6AE204615F038
:10A2500055F8DDE710B915F07BF8D9E7116800294A
:10A26000B8BF4942002015F017F8D7E718B9002009
:10A2700015F060F8CCE71168002015F004F9CDE77F
:10A2800015F0E3FB2B681B0203F4F85320F4F8529B
:10A290001A431021234815F0CAFBBFE710212148BB
:10A2A00024B915F0D2FB00F01F00B1E715F0CDFB8B
:10A2B0002B6820F01F0203F01F03E9E700287FF45A
:10A2C000ABAE002014F08EFFC0F30010A0E7164ED6
:10A2D00070B91521134815F0B8FB002800F007826B
:10A2E0004FF0807393FBF0F0B042A8BF3046C5E05A
:10A2F00013684BB14FF0807292FBF3F2B242A8BFE9
:10A3000032462A601521C5E73246FAE71268332142
:10A31000C0E76C2103484CB915F097FBC0F38040AF
:10A3200076E700BF0C38FF1FFFFF0F0015F08DFB15
:10A330002B689B0403F4802320F480221A436C21B1
:10A34000A8E76C21B64824B915F07FFBC0F3C040E4
:10A350005EE715F07AFB2B68DB0403F4002320F49E
:10A360000022EBE70021AE4815F06FFB2B685B0085
:10A3700003F0020320F002021A4300218AE750B9D9
:10A380006C21A74815F061FB4FF48073C0F30360A4
:10A3900043FA00F03CE71368102B28D00DDC022BA9
:10A3A00021D004DC012B16D04FF0FF3314E0042B36
:10A3B0001BD0082BF8D105230EE0402B19D003DC6D
:10A3C000202BF1D1032307E0802B14D0B3F5807F3D
:10A3D000EAD1002300E008232B602B6801330CD165
:10A3E0001024204670BD0723F6E70623F4E7042374
:10A3F000F2E70223F0E70123EEE76C21884815F02D
:10A4000024FB2B681B0603F0706320F0706295E755
:10A4100015F01BFB2B68DB0303F4C03320F4C032C0
:10A420008CE76C217E4824B915F00FFBC0F3803017
:10A43000EEE615F00AFB2B689B0303F4804320F43F
:10A4400080427BE76C21764824B915F0FEFAC0F310
:10A450000030DDE615F0F9FA2B681B0303F4805396
:10A4600020F480526AE715F0F0FA6C2106466C4839
:10A4700015F0EBFA3205C0F3021001D42860CDE6E6
:10A4800040F00800C4E615F0E0FA10F480444FF004
:10A490006C01634808D015F0D8FA2B68DB0103F48F
:10A4A000F06320F4F06249E715F0CFFA6C215C48C4
:10A4B00015F0CBFA2A68120220F4006002F4006260
:10A4C00002436C21564815F0B2FA6C21544815F03D
:10A4D000BCFA2B681B0103F0700320F070021A43D2
:10A4E0006C214F4815F0A3FA7BE76C214C48D4B996
:10A4F00015F0ABFA10F480464FF06C01484804D0D8
:10A5000015F0A3FAC0F3021082E615F09EFA6C2152
:10A510000446434815F099FA2305C0F3C31048BF19
:10A5200040F00800AAE715F090FA10F480444FF0CC
:10A530006C013B4808D015F088FA2B681B0103F02A
:10A54000700320F07002F9E615F07FFA2B68DB014A
:10A5500003F4F06320F4F062C1E76C21304824B9C1
:10A5600015F073FA00F00F0052E615F06EFA2B6842
:10A5700020F00F0203F00F03E0E66D21284824B914
:10A5800015F063FAC0F3C03042E615F05EFA2B68AE
:10A59000DB039BB220F400421A436D217AE66D2161
:10A5A0001F4824B915F051FAC0F3413030E615F0D8
:10A5B0004CFA2B685B0303F4C04320F4C042EBE782
:10A5C00015F043FA2B681B0203F4706320F47062E9
:10A5D000E2E76D21124824B915F037FAC0F34110B3
:10A5E00016E615F032FA2B685B0103F0600320F0E9
:10A5F0006002D1E76D210A48002CB1D015F025FA90
:10A600002B6820F00F0203F00F03C5E715F01DFAC9
:10A610002B681B0603F0807320F08072BCE700BF3C
:10A620000C38FF1F6D216A485CB915F00EFA001452
:10A6300000F07F0310F0400018BF6FF07F00184358
:10A64000E6E515F002FA2B681B0403F4FE0320F480
:10A65000FE02A1E76C215E4824B915F0F6F9C0F3BB
:10A660004040D5E515F0F1F92B685B0403F40033A5
:10A6700020F4003262E610B914F078FEC8E51168E3
:10A68000002014F013FEC9E55248F7E6136853B1F1
:10A690004FF0807292FBF3F24E4B9A42A8BF1A46DB
:10A6A0002A601421F6E54B4AFAE76C21484824B9A0
:10A6B00015F0CBF9C0F34030AAE515F0C6F92B68C8
:10A6C0005B0303F4005320F4005237E66C2140484A
:10A6D00024B915F0BAF9C0F3035099E515F0B5F9AE
:10A6E0002B681B0503F4700320F4700226E6304645
:10A6F000C4E613684BB14FF0807292FBF3F2B242A2
:10A70000A8BF32462A601321C4E53246FAE7702119
:10A710002F4824B915F099F9C0F3072078E515F012
:10A7200094F92A68120220F47F4092B20243702109
:10A73000274815F07CF90021254815F086F92B688B
:10A74000002B20F00402CCBF0423002314E6702168
:10A750001F481CB915F079F9C0B259E515F075F923
:10A760002A7820F0FF000243702193E51368032B41
:10A770003FF636AE7021164815F067F92B681B04BA
:10A7800003F4403320F440321A43EDE770211048BF
:10A79000002C3FF4C1AD15F058F92B68002B20F4C4
:10A7A000802214BF4FF480230023EDE77021084876
:10A7B00024B915F04AF9C0F3015029E515F045F91F
:10A7C0002B681B0503F4401320F44012DCE700BFA4
:10A7D0000C38FF1FFFFF0F000B4611B9014618464A
:10A7E00000E40820704708B5002014F087FD10B180
:10A7F000084B987860B1084815F068F914F0C4FD6A
:10A80000064900231846D1E9001214F00DFD01207D
:10A8100008BD00BFC409FF1F0C38FF1F1815FF1F1C
:10A8200038B50D46044648B914F04EFD2B68C118E2
:10A830002960204614F076FC204638BD0820FCE74D
:10A8400007B5019239B9014601AA0120FFF7CAFBF9
:10A8500003B05DF804FB0820FAE7064B9B6A084644
:10A86000114613B1044B9B6E1847044B1B68DB6801
:10A87000FAE700BF1815FF1F6434FF1F903AFF1F4F
:10A880002DE9F041664D674BD5F880206648674F4B
:10A89000674C012115F0FEF86649634815F040F950
:10A8A000FE68736803F16402A26003F5927222608D
:10A8B00003F5A272626003F5D272226203F5E272BE
:10A8C000626203F55172E26003F5597203F5697033
:10A8D000226103F5617203F57173E36133686261AC
:10A8E0001B69A06198473368E0691B699847336822
:10A8F00060691B69984733682068DB68984733684C
:10A900006068DB6898473368A068DB6898473368FD
:10A910002069DB6898473368E068DB6898473368EC
:10A92000606ADB6898473368206ADB689847336859
:10A93000606A9B6998473368206A9B6998473368C7
:10A9400060699B6998473368E0689B6998473A69F2
:10A95000394B02F114011960736803F501739361B7
:10A9600014F012FD0023D4E90012184614F05CFC28
:10A97000D5F88030314AC3F80422314AC3F808229E
:10A980000021012259701A702E4BC5F88C302E4BC5
:10A99000C5F888302D4BC5F884302D4BC5F8903064
:10A9A0002C4BC5F8A4302C4BC5F8A0302B4BC5F868
:10A9B00094302B4BC5F898302A4BC5F8B4302A4B4D
:10A9C000C5F8B030294BC5F8C030294BC5F8BC30AC
:10A9D000284BC5F8B830284BC5F8CC3032214FF49D
:10A9E000F073C5E91D31254BC5F8C430AB6E85F851
:10A9F0007C2003B1A2620220FFF7A0FA3368606AEC
:10AA0000DB689847606A1E4C0423437533681B68F3
:10AA1000984723689847A3680020BDE8F04118478D
:10AA20006434FF1F7C6E02000C38FF1F847E02001E
:10AA30001815FF1FD19F0000903AFF1FE7A70000E5
:10AA4000339F0000179F0000319F00002D9F0000E2
:10AA5000299F0000D9A7000041A80000059F000021
:10AA600021A80000F99E0000E59E0000939F0000D1
:10AA7000319E00007D9F00003D9F0000B59D0000BD
:10AA80007409FF1F194B70B5DD68194C2B682068DD
:10AA90005B6998472B6860689B6898472B68A0683B
:10AAA0009B6898472B68E0689B6898472B682069EB
:10AAB0009B6898472B6860699B6898472B68A069DA
:10AAC0009B6898472B68E0699B6898472B68206AC9
:10AAD0009B6898472B6820689B68984714F0A2FCF5
:10AAE000044BBDE870405B68184700BF847E0200DD
:10AAF0005015FF1F7409FF1F10B5144605283ED8D6
:10AB0000DFE800F0031412232E33136844F62062AA
:10AB1000934236D842F21172B3FBF2F002FB1030CE
:10AB2000194B80B29B689847002010BD174B2468D2
:10AB3000DA68D2E9003000F5F2701CB1DB6900215F
:10AB40009847F1E79B689847EEE7104B1168DB6880
:10AB50000F4A1B685069DB69003118BF0121EFE71C
:10AB6000084614F03FFB2060DEE7084B084ADB682C
:10AB700058681B6800F592705061DB68E3E70420B9
:10AB8000D3E71020D1E700BF7409FF1F847E0200C5
:10AB90005015FF1F10B50348144615F042F8206009
:10ABA00010BD00BF983AFF1F014815F02CB800BF38
:10ABB000983AFF1F10B5044618B914F0B3FA2046AE
:10ABC00010BD0820FCE710B5044618B914F09EFA31
:10ABD000204610BD0820FCE70021F4E74942F2E7D7
:10ABE000F1E7014815F073B8983AFF1F022804BF37
:10ABF0000B4B93F8D80030B90A4BDB681B685B69D4
:10AC0000094A10681847012809D1054B93F8D83034
:10AC1000012B04D1034BDB681B689B69F0E770478D
:10AC20006434FF1F847E02005015FF1F38B50D46A7
:10AC3000044620B914F062FB2860204638BD082085
:10AC4000FCE710B501460D4815F05AF8002014F045
:10AC500075FA002014F0C6FA10F008040DD182062F
:10AC60000BD56F21054814F0DCFFC30105D5204644
:10AC70000221BDE8104014F08DBA10BD983AFF1FB4
:10AC8000012903D1024A702114F0BDBF704700BFF3
:10AC90001E000CC4A62970B50446154600F07D823E
:10ACA0007DD8172900F06B812DD8042900F02A8166
:10ACB0000CD8012900F00C81C0F0FF80022900F0BF
:10ACC0001081032900F017810424E2E1072900F034
:10ACD0003D810ED8052900F021810629F4D11021EB
:10ACE000BC48002C40F0248114F09BFFC0F30420EA
:10ACF000E6E0082900F03A811529E5D10028E3D0E3
:10AD0000126811211EE11D2900F0F5801CD81A29B6
:10AD100000F0578109D81829D6D1002840F04E817B
:10AD20003321AC4814F07DFFCAE01B2900F061819B
:10AD30001C29C9D1002840F06D810146A54814F0B6
:10AD400070FFC0F34000BBE0A32900F0C2810ED821
:10AD50008C2900F06C81A229B6D16C219D48002C71
:10AD600040F0AE8114F05DFFC0F3C130A8E0A4292B
:10AD700000F0C081A529A7D16C219648002C40F095
:10AD8000DA8114F04EFF10F4804F4FF06C019148BF
:10AD900000F0C18114F045FFC0F3C31090E0B52965
:10ADA00000F0C1823BD8AB2900F06B8213D8A829F0
:10ADB00000F03B82C0F02982A92900F04882AA292C
:10ADC00082D16D218348002C40F0528214F029FF7B
:10ADD000C0F3032074E0AE2900F07C820FD8AC29C8
:10ADE00000F06082AD297FF46FAF6D217948002CAF
:10ADF00040F0648214F015FFC0F3006060E0B329F6
:10AE000000F08082B4297FF45FAF00287FF45CAF4C
:10AE10006F21704814F005FFC0F3044050E0BB29D7
:10AE200000F0CD8225D8B82900F0978215D8B62930
:10AE30007FF44AAF002840F081821421654814F065
:10AE4000F0FE002800F078824FF0807393FBF0F062
:10AE5000614B9842A8BF184668E1B92900F08E827C
:10AE6000BA297FF431AF5C4E002840F09A8213215A
:10AE700088E0C02900F0E2820FD8BC2900F0BF8230
:10AE8000BF297FF421AF002840F0C88270215148CB
:10AE900014F0C7FEC0F3014012E0CC2900F0DE82BE
:10AEA000CE297FF411AF00287FF40EAF6F214948FF
:10AEB00014F0B7FEC0F3090002E018B914F010FA5C
:10AEC0002860E6E01168002014F02CF90024E0E08E
:10AED00010B914F0F9F9F3E71168002014F0CEF975
:10AEE000F4E718B9002014F017FAE9E71168002018
:10AEF00014F00CF9EAE7002C7FF4E6AE204614F0DB
:10AF0000FDF9DDE710B914F023FAD9E7116800293B
:10AF1000B8BF4942002014F0BFF9D7E718B90020A4
:10AF200014F008FACCE71168002014F0ACFACDE771
:10AF300014F077FE2B681B0203F4F85320F4F85248
:10AF40001A431021234814F05EFEBFE71021214868
:10AF500024B914F066FE00F01F00B1E714F061FEA2
:10AF60002B6820F01F0203F01F03E9E700287FF49D
:10AF7000ABAE002014F036F9C0F30010A0E7164E77
:10AF800070B91521134814F04CFE002800F0078218
:10AF90004FF0807393FBF0F0B042A8BF3046C5E09D
:10AFA00013684BB14FF0807292FBF3F2B242A8BF2C
:10AFB00032462A601521C5E73246FAE71268332186
:10AFC000C0E76C2103484CB914F02BFEC0F380405D
:10AFD00076E700BF983AFF1FFFFF0F0014F021FE35
:10AFE0002B689B0403F4802320F480221A436C21F5
:10AFF000A8E76C21B64824B914F013FEC0F3C04092
:10B000005EE714F00EFE2B68DB0403F4002320F44B
:10B010000022EBE70021AE4814F003FE2B685B0032
:10B0200003F0020320F002021A4300218AE750B91C
:10B030006C21A74814F0F5FD4FF48073C0F3036052
:10B0400043FA00F03CE71368102B28D00DDC022BEC
:10B0500021D004DC012B16D04FF0FF3314E0042B79
:10B060001BD0082BF8D105230EE0402B19D003DCB0
:10B07000202BF1D1032307E0802B14D0B3F5807F80
:10B08000EAD1002300E008232B602B6801330CD1A8
:10B090001024204670BD0723F6E70623F4E70423B7
:10B0A000F2E70223F0E70123EEE76C21884814F071
:10B0B000B8FD2B681B0603F0706320F0706295E703
:10B0C00014F0AFFD2B68DB0303F4C03320F4C0326F
:10B0D0008CE76C217E4824B914F0A3FDC0F38030C6
:10B0E000EEE614F09EFD2B689B0303F4804320F4EE
:10B0F00080427BE76C21764824B914F092FDC0F3BE
:10B100000030DDE614F08DFD2B681B0303F4805343
:10B1100020F480526AE714F084FD6C2106466C48E6
:10B1200014F07FFD3205C0F3021001D42860CDE693
:10B1300040F00800C4E614F074FD10F480444FF0B1
:10B140006C01634808D014F06CFD2B68DB0103F43C
:10B15000F06320F4F06249E714F063FD6C215C4871
:10B1600014F05FFD2A68120220F4006002F400620D
:10B1700002436C21564814F046FD6C21544814F0EB
:10B1800050FD2B681B0103F0700320F070021A437E
:10B190006C214F4814F037FD7BE76C214C48D4B943
:10B1A00014F03FFD10F480464FF06C01484804D085
:10B1B00014F037FDC0F3021082E614F032FD6C216A
:10B1C0000446434814F02DFD2305C0F3C31048BFC7
:10B1D00040F00800AAE714F024FD10F480444FF07A
:10B1E0006C013B4808D014F01CFD2B681B0103F0D8
:10B1F000700320F07002F9E614F013FD2B68DB01F8
:10B2000003F4F06320F4F062C1E76C21304824B904
:10B2100014F007FD00F00F0052E614F002FD2B6859
:10B2200020F00F0203F00F03E0E66D21284824B957
:10B2300014F0F7FCC0F3C03042E614F0F2FC2B68C7
:10B24000DB039BB220F400421A436D217AE66D21A4
:10B250001F4824B914F0E5FCC0F3413030E614F087
:10B26000E0FC2B685B0303F4C04320F4C042EBE72F
:10B2700014F0D7FC2B681B0203F4706320F4706297
:10B28000E2E76D21124824B914F0CBFCC0F3411061
:10B2900016E614F0C6FC2B685B0103F0600320F097
:10B2A0006002D1E76D210A48002CB1D014F0B9FC3E
:10B2B0002B6820F00F0203F00F03C5E714F0B1FC78
:10B2C0002B681B0603F0807320F08072BCE700BF80
:10B2D000983AFF1F6D216A485CB914F0A2FC001473
:10B2E00000F07F0310F0400018BF6FF07F0018439C
:10B2F000E6E514F096FC2B681B0403F4FE0320F42F
:10B30000FE02A1E76C215E4824B914F08AFCC0F368
:10B310004040D5E514F085FC2B685B0403F4003352
:10B3200020F4003262E610B914F020F8C8E5116884
:10B33000002013F0BBFFC9E55248F7E6136853B18C
:10B340004FF0807292FBF3F24E4B9A42A8BF1A461E
:10B350002A601421F6E54B4AFAE76C21484824B9E3
:10B3600014F05FFCC0F34030AAE514F05AFC2B68DF
:10B370005B0303F4005320F4005237E66C2140488D
:10B3800024B914F04EFCC0F3035099E514F049FCC5
:10B390002B681B0503F4700320F4700226E6304688
:10B3A000C4E613684BB14FF0807292FBF3F2B242E5
:10B3B000A8BF32462A601321C4E53246FAE770215D
:10B3C0002F4824B914F02DFCC0F3072078E514F0C1
:10B3D00028FC2A68120220F47F4092B202437021B6
:10B3E000274814F010FC0021254814F01AFC2B68A3
:10B3F000002B20F00402CCBF0423002314E67021AC
:10B400001F481CB914F00DFCC0B259E514F009FC3A
:10B410002A7820F0FF000243702193E51368032B84
:10B420003FF636AE7021164814F0FBFB2B681B0468
:10B4300003F4403320F440321A43EDE77021104802
:10B44000002C3FF4C1AD14F0ECFB2B68002B20F472
:10B45000802214BF4FF480230023EDE770210848B9
:10B4600024B914F0DEFBC0F3015029E514F0D9FB38
:10B470002B681B0503F4401320F44012DCE700BFE7
:10B48000983AFF1FFFFF0F000B4611B901461846FF
:10B4900000E40820704708B5002013F02FFF10B11A
:10B4A000084B987860B1084814F0FCFB13F06CFF6F
:10B4B000064900231846D1E9011213F0B5FE012018
:10B4C00008BD00BFC409FF1F983AFF1F5015FF1F9A
:10B4D00038B50D46044648B913F0F6FE2B68C1187E
:10B4E0002960204613F01EFE204638BD0820FCE7E8
:10B4F00007B5019239B9014601AA0120FFF7CAFB3D
:10B5000003B05DF804FB0820FAE7064B5B6A0846C7
:10B51000114613B1044B9B6E1847044B1B68DB6844
:10B52000FAE700BF5015FF1F6434FF1F943AFF1F56
:10B530002DE9F041624D634BD5F880206248634F9E
:10B54000634C012114F092FB62495F4814F0D4FB74
:10B55000FE68736803F16402226003F59272626010
:10B5600003F5A272A26003F5E272E26003F5517284
:10B57000226103F5597203F56970626103F5617226
:10B5800003F5717323623368A2611B69E061984718
:10B590003368206A1B6998473368A0691B6998471C
:10B5A00033682068DB68984733686068DB689847D1
:10B5B0003368A068DB6898473368E068DB689847C1
:10B5C00033686069DB68984733682069DB689847AF
:10B5D0003368E0685B6998473368A0699B6998475E
:10B5E000336820699B699847D6E90030DB6800F52D
:10B5F000F2709847D6E9003000F5F2709B699847E1
:10B600003A69354B02F114011960736803F5097347
:10B61000936113F0B9FE0023D4E90112184613F028
:10B6200003FED5F880302D4AC3F804222C4AC3F813
:10B6300008220021012259701A702A4BC5F88C305B
:10B64000294BC5F88830294BC5F88430284BC5F8FC
:10B650009030284BC5F8A430274BC5F8A030274BB5
:10B66000C5F89430264BC5F89830264BC5F8B43051
:10B67000254BC5F8B030254BC5F8C030244BC5F874
:10B68000BC30244BC5F8B830234BC5F8CC30322140
:10B690004FF4F073C5E91D31204BC5F8C430AB6ED3
:10B6A00085F87C2003B162621D4C0220FFF79EFAF0
:10B6B00023689847A3680020BDE8F041184700BF01
:10B6C0006434FF1F7C700200983AFF1F847E0200E2
:10B6D0005015FF1F81AC0000943AFF1F97B4000083
:10B6E000E3AB0000C7AB0000E1AB0000DDAB000046
:10B6F000D9AB000089B40000F1B40000B5AB000084
:10B70000D1B40000A9AB000095AB000043AC000031
:10B71000F9AA00002DAC0000EDAB000085AA0000E6
:10B720007409FF1F014B00221A6770476434FF1F22
:10B73000F7B50523ADF8003061F07F038DF80230D6
:10B7400013168DF8033013148DF804308DF806208D
:10B7500013120D4614460721012268460F4F8DF83B
:10B76000053013F0CDFF3B688DF807009B699847C3
:10B7700000263B681DF806009B6801369847082E96
:10B78000F7D1022010F03CFD054B1B6825F0800529
:10B7900003EB85056C6003B0F0BD00BF203DFF1FCB
:10B7A0001C3DFF1FF0B52A4B01F07F052B4485B0EF
:10B7B00093F80C32DB07164606D4264B1B6803EBC6
:10B7C00085056B68336041E0012205230321224C8B
:10B7D000ADF8043001A88DF8065013F091FF2368EE
:10B7E0008DF807009B699847236804211B690DEBBE
:10B7F0000100984710F0FEFC07462368DB69984774
:10B8000007281ED9236808215B690DEB01009847C2
:10B810000122072102A89DF80F4013F071FF844216
:10B8200014D19DF80830052B10D19DF80930FF2B5D
:10B830000CD19DF80A30AB4208D1DDF80B301BBAB1
:10B84000C0E7384610F0E6FC0A28D6D905B0F0BDAE
:10B85000243DFF1F1C3DFF1F203DFF1F08B5064B69
:10B86000064A1B680146002014F0BEFA0020BDE81D
:10B87000084013F063BC00BF1C3DFF1F243DFF1FA9
:10B8800038B51546044628B9084613F0ABFC2860C5
:10B89000204638BD0420FCE710B5044618B913F063
:10B8A00041FC204610BD0820FCE710B5044618B93D
:10B8B00013F02CFC204610BD0820FCE70021F4E723
:10B8C0004942F2E7F1E7024B186814F0A5BA00BF4D
:10B8D0001C3DFF1F08B513F057FD0649002318460D
:10B8E000D1E9011213F0A0FC034B1868BDE8084031
:10B8F00014F089BA8415FF1F1C3DFF1F022804BFE6
:10B900000B4B93F8D80030B90A4BDB681B685B69B6
:10B91000094A10681847012809D1054B93F8D83017
:10B92000012B04D1034BDB681B689B69F0E7704770
:10B930006434FF1F847E02008415FF1F38B5002089
:10B94000FFF7DCFF114B124CDD6820682B689B6809
:10B9500098472B6860689B6898472B68A0689B682D
:10B9600098472B68E0689B6898472B6820699B681C
:10B9700098472B6860699B6898472B68A0699B680B
:10B980009847BDE8384013F04DBD00BF847E0200EB
:10B990008415FF1F38B50D46044648B913F094FCD2
:10B9A0002B68C1182960204613F0BCFB204638BD27
:10B9B0000820FCE710B5144601BB052820D8DFE8B5
:10B9C00000F003090D111519002013F089FC206007
:10B9D000002010BD002013F077FCF8E7002013F0E2
:10B9E0009BFCF4E7002013F089FCF0E7002013F043
:10B9F000AFFCECE7002013F09DFCE8E70820E8E747
:10BA00000420E6E708B519BB052823D8DFE800F0D5
:10BA100003090E22131B1146002013F083FB0020A4
:10BA200008BD1146002013F029FCF8E7114600205C
:10BA300013F06CFBF3E782EAE271A1EBE271002004
:10BA400013F02AFCEBE71146002013F01CFDE6E79B
:10BA50000820E5E70420E3E76AE6A3E6012270B5E3
:10BA600011464B4E4B4C072013F0EEFD4A4814F0A4
:10BA700083F9F5686B6803F59272626003F5A27250
:10BA8000A26003F1C402E26003F1E40203F1640086
:10BA9000226103F18402A433A3612B686261DB6835
:10BAA000206098472B686068DB6898472B68A0681F
:10BAB000DB6898472B68E068DB6898472B6820694B
:10BAC000DB6898472B6860691B6998472B68A069F9
:10BAD0001B699847F56A2B689847304B30491D60C1
:10BAE000304BD3F880200A602F49C2F80412002599
:10BAF00001262E4916705570C2F808122C4AC3F858
:10BB00008C202C4AC3F888202B4AC3F884202B4A67
:10BB1000C3F890202A4AC3F8A4202A4AC3F8A020D8
:10BB2000294AC3F89420294AC3F89820284AC3F820
:10BB3000B420284AC3F8B020274AC3F8BC20274ABB
:10BB4000C3F8CC20264AC3F8C82032214FF4C37270
:10BB5000C3E91D21234AC3F8C420234A83F87C602B
:10BB6000C3F8C02013F010FCD4E901122B4628467C
:10BB700013F05AFB28464FF4484113F08DFB28463A
:10BB80004FF4484113F07FFC3046BDE87040B5E605
:10BB9000847E02008415FF1F243DFF1F203DFF1FF0
:10BBA0001C3DFF1F6434FF1FD5B80000C7B800005C
:10BBB000ABB80000C5B80000C1B80000BDB80000B7
:10BBC000B5B9000005BA000099B8000095B90000A9
:10BBD00031B70000A5B7000081B80000FDB8000033
:10BBE00025B700003DB900005DB80000014B002200
:10BBF0001A6770476434FF1FF7B50523ADF80030AE
:10BC000061F07F038DF8023013168DF803301314A2
:10BC10008DF804308DF8062013120D4614460721C6
:10BC2000012268460F4F8DF8053013F069FD3B681F
:10BC30008DF807009B69984700263B681DF80600B1
:10BC40009B6801369847082EF7D1022010F0D8FAE9
:10BC5000054B1B6825F0800503EB85056C6003B080
:10BC6000F0BD00BF4042FF1F4442FF1FF0B52A4B0A
:10BC700001F07F052B4485B093F80C32DB071646A4
:10BC800006D4264B1B6803EB85056B68336041E0E7
:10BC9000012205230321224CADF8043001A88DF8C0
:10BCA000065013F02DFD23688DF807009B69984717
:10BCB000236804211B690DEB0100984710F09AFAE4
:10BCC00007462368DB69984707281ED9236808219F
:10BCD0005B690DEB010098470122072102A89DF83E
:10BCE0000F4013F00DFD844214D19DF80830052B50
:10BCF00010D19DF80930FF2B0CD19DF80A30AB42D2
:10BD000008D1DDF80B301BBAC0E7384610F082FAD4
:10BD10001428D6D905B0F0BDB03FFF1F4442FF1F25
:10BD20004042FF1F08B5064B064A1B68014600202B
:10BD300014F0B6F80020BDE8084013F0FFB900BFCA
:10BD40004442FF1FB03FFF1F38B51546044628B9CF
:10BD5000084613F047FA2860204638BD0420FCE767
:10BD600010B5044618B913F0DDF9204610BD0820BF
:10BD7000FCE710B5044618B913F0C8F9204610BD09
:10BD80000820FCE70021F4E74942F2E7F1E7024B23
:10BD9000186814F09DB800BF4442FF1F08B513F0A7
:10BDA000F3FA064900231846D1E9011213F03CFAD0
:10BDB000034B1868BDE8084014F081B8AC15FF1FAC
:10BDC0004442FF1F022804BF0B4B93F8D80030B940
:10BDD0000A4BDB681B685B69094A10681847012831
:10BDE00009D1054B93F8D830012B04D1034BDB6804
:10BDF0001B689B69F0E770476434FF1F847E020074
:10BE0000AC15FF1F70B5144E144C0020FFF7DAFF7D
:10BE1000F56820682B689B6898472B6860689B686A
:10BE200098472B68A0689B6898472B68E0689B68D8
:10BE300098472B6820699B6898472B6860699B68C6
:10BE400098472B68A0699B689847F36A5B68984796
:10BE5000BDE8704013F0E6BA847E0200AC15FF1F07
:10BE600038B50D46044648B913F02EFA2B68C118B0
:10BE70002960204613F056F9204638BD0820FCE71B
:10BE800010B5144601BB052820D8DFE800F00309EF
:10BE90000D111519002013F023FA2060002010BDA9
:10BEA000002013F011FAF8E7002013F035FAF4E758
:10BEB000002013F023FAF0E7002013F049FAECE732
:10BEC000002013F037FAE8E70820E8E70420E6E767
:10BED00008B519BB052823D8DFE800F003090E22B6
:10BEE000131B1146002013F01DF9002008BD114658
:10BEF000002013F0C3F9F8E71146002013F006F90B
:10BF0000F3E782EAE271A1EBE271002013F0C4F9D9
:10BF1000EBE71146002013F0B6FAE6E70820E5E764
:10BF20000420E3E768E6A1E6012270B511464B4E16
:10BF30004B4C072013F088FB4A4813F077FFF56855
:10BF40006B6803F59272626003F5A272A26003F15E
:10BF5000C402E26003F1E40203F16400226103F130
:10BF60008402A433A3612B686261DB682060984778
:10BF70002B686068DB6898472B68A068DB68984787
:10BF80002B68E068DB6898472B682069DB68984776
:10BF90002B6860691B6998472B68A0691B699847E3
:10BFA000F56A2B689847304B30491D60304BD3F809
:10BFB00080200A602F49C2F80412002501262E496C
:10BFC00016705570C2F808122C4AC3F88C202C4AFF
:10BFD000C3F888202B4AC3F884202B4AC3F890204A
:10BFE0002A4AC3F8A4202A4AC3F8A020294AC3F841
:10BFF0009420294AC3F89820284AC3F8B420284A34
:10C00000C3F8B020274AC3F8BC20274AC3F8CC2085
:10C01000264AC3F8C82032214FF4C372C3E91D2158
:10C02000234AC3F8C420234A83F87C60C3F8C020A5
:10C0300013F0AAF9D4E901122B46284613F0F4F8BC
:10C0400028464FF4484113F027F928464FF4484159
:10C0500013F019FA3046BDE87040B3E6847E020062
:10C06000AC15FF1FB03FFF1F4042FF1F4442FF1FA0
:10C070006434FF1F9DBD00008FBD000073BD000034
:10C080008DBD000089BD000085BD000081BE00009F
:10C09000D1BE000061BD000061BE0000F9BB000020
:10C0A0006DBC000049BD0000C5BD0000EDBB000037
:10C0B00005BE000025BD0000012810B514460CD0B7
:10C0C00003D3022810D0042006E01368094AB3FA0B
:10C0D00083F35B099372002010BD1368064AB3FA1C
:10C0E00083F35B091360F6E7084613F07BF82060E2
:10C0F000F1E700BF4842FF1F6C00FF1F10B5044668
:10C1000018B913F00FF8204610BD0820FCE7024BC9
:10C11000186813F078BF00BF9442FF1F022804BFC5
:10C120000B4B93F8D80030B90A4BDB681B685B698E
:10C13000094AD0681847012809D1054B93F8D8302F
:10C14000012B04D1034BDB681B689B69F0E7704748
:10C150006434FF1F847E0200D415FF1F38B5002011
:10C16000FFF7DCFF0F4B104CDD68E0682B685B6964
:10C1700098472B6820689B6898472B68A0689B6845
:10C1800098472B68E0689B6898472B6820699B68F4
:10C1900098472B6860689B689847BDE8384013F063
:10C1A00041B900BF847E0200D415FF1F38B50D468B
:10C1B000044620B913F0A2F82860204638BD0820B4
:10C1C000FCE710B5044628B9034B188112F09EFF16
:10C1D000204610BD0820FCE74842FF1F0021F0E781
:10C1E0004942EEE7EDE738B5002013F087F8054641
:10C1F000A8B90C4B0C48196813F0E8FE0B4B022051
:10C2000001241C60FFF78AFF13F0BEF80849284696
:10C210000B69D1E9011213F007F8204638BD002060
:10C22000FCE700BF9442FF1F4842FF1F6C00FF1F46
:10C23000D415FF1F38B50D46044648B913F044F82D
:10C240002B68C1182960204612F06CFF204638BDCB
:10C250000820FCE7F8B5830C04460DD0C0F3424338
:10C26000062B09D1234B5A7A20F01F04002A3AD01A
:10C270001B7803F01F031C431F4F204E3B68204DCB
:10C280009B680021C4F3074098472A7E336803EB7C
:10C290008203000258603B6800219B68C4F30720BA
:10C2A00098472B7E326802EB8302012153681843C2
:10C2B0003B68000250609B68E0B298473268297E74
:10C2C00002EB81014B6818430011A30C4860106118
:10C2D0000BD0C4F34243072B02D1C4F301112976DA
:10C2E00043F0080302E0DB7AC3E7082302EB830391
:10C2F0005C60F8BD4842FF1F9042FF1F9442FF1F41
:10C30000D415FF1F0D4B00F077021B6842F00802A6
:10C3100030B406280A4D03EB8203C1F3130404BFB3
:10C3200001F01F01E9725C60AB7A23B944EA404036
:10C3300030BCFFF78FBF30BC704700BF9442FF1F77
:10C340004842FF1F08461146DCE738B504460F2077
:10C3500000F013F80323B4FBF3F303EB4303E41AF5
:10C360000546E4B220F0300040EA0410FFF772FF07
:10C370002846BDE83840FFF76DBF10B5074B9B7AE4
:10C3800004461BB9030701D4FFF7DFFF044B1B680A
:10C3900004F07F0403EB8404606810BD4842FF1F73
:10C3A0009442FF1FA829F8B504460E46154600F032
:10C3B000C6815BD81D2900F0D28021D8042900F065
:10C3C000D5800CD8012900F0B780C0F0A9800229DF
:10C3D00000F0BB80032900F0C2800424A4E00629F9
:10C3E00000F0D980C0F0CE80072900F0E88008294D
:10C3F000F3D10028F1D112F0F5FEC0F3001092E065
:10C40000A32900F054811ED8A02900F025810CD862
:10C410008C29E2D1002840F0E4800820FFF7ADFF2E
:10C4200000F00F00C0F108007DE0A12900F0248198
:10C43000A229D2D10C20002C40F02E81FFF79DFFC5
:10C44000C0F3C1306FE0A52900F05181C0F03F81F9
:10C45000A62900F05C81A729BFD10C20002C40F058
:10C460006681FFF78AFF00F00F005CE0B22900F060
:10C470000F8225D8AD2900F0B3810ED8AA2900F08B
:10C480008181C0F06E81AB2900F09081AC29A4D1EC
:10C49000002840F09C810520E3E7AF2900F0CB8124
:10C4A000C0F0B181B02900F0D881B12995D1002820
:10C4B00040F0E4810720FFF760FFC0F3802032E006
:10C4C000B72900F01D8210D8B42900F00382C0F013
:10C4D000F081B52900F00782B6297FF47EAFB24B18
:10C4E000002840F00A821B6958E0CE2900F0338210
:10C4F0000AD8B82900F01482B9297FF46EAF002859
:10C5000040F01F8207206DE1D02900F03882D62943
:10C510007FF463AFA44B002840F039825B683DE0B4
:10C5200020B912F0DDFE28602046F8BD1168002019
:10C5300012F0F8FD0024F7E710B912F0C5FEF2E79B
:10C540001168002012F09AFEF4E718B9002012F0EA
:10C55000E3FEE8E71168002012F0D8FDEAE7002CBE
:10C560007FF43BAF204612F0C9FEDCE710B912F0B1
:10C57000EFFED8E711680029B8BF4942002012F049
:10C580008BFED7E710B912F0D5FECCE7116800207A
:10C5900012F079FFCEE7844F10B9FB7A2B60C3E726
:10C5A0001368FB720020FFF7E8FE10F08004C1D191
:10C5B000F97A304601F01F01FFF7A4FEB4E77A4E86
:10C5C00008B93378EAE7136833700020FFF7D5FE27
:10C5D0000306AFD53178062001F01F01FFF792FE68
:10C5E000A8E71368102B31D00DDC022B2AD004DC15
:10C5F000012B16D04FF0FF3314E0042B24D0082B6E
:10C60000F8D105230EE0402B22D003DC202BF1D102
:10C61000032307E0802B1DD0B3F5807FEAD10023F0
:10C6200000E008232B602B68013300F0B381082061
:10C63000FFF7A3FE2B6820F00F0103F00F0319434F
:10C640000820CBE70723EDE70623EBE70423E9E720
:10C650000223E7E70123E5E7082024B9FFF78DFE71
:10C66000C0F340205FE7FFF788FE2B685B0203F40E
:10C67000007320F40071E2E7082024B9FFF77DFE83
:10C68000C0F300204FE7FFF778FE2B681B0203F48E
:10C69000807320F48071D2E7FFF76FFE2B68DB0315
:10C6A00003F4C03320F4C03119430C2096E70C206A
:10C6B00024B9FFF762FEC0F3803034E7FFF75DFE78
:10C6C0002B689B0303F4804320F48041ECE70C20AB
:10C6D00024B9FFF752FEC0F3C12024E7FFF74DFE57
:10C6E0002B68DB0203F4C05320F4C051DCE70C20BC
:10C6F00024B9FFF742FEC0F3C31014E7FFF73DFE75
:10C700002B68DB0103F4F06320F4F061CCE70C202C
:10C7100024B9FFF732FEC0F3021004E7FFF72DFE45
:10C720002B681B0103F0700320F07001BCE7FFF7DA
:10C7300024FE2B6820F00F0103F00F03B4E728B9A3
:10C740000520FFF71AFEC0F3C030ECE60D20FFF71E
:10C7500014FE2B68DB039BB220F4004119430D202B
:10C760003CE728B90520FFF708FEC0F34130DAE6C0
:10C770000D20FFF702FE2B685B0303F4C04320F497
:10C78000C041EBE728B90520FFF7F7FDC0F3032010
:10C79000C9E60D20FFF7F1FD2B681B0203F470635F
:10C7A00020F47061DAE700BF4842FF1F28B9052076
:10C7B000FFF7E3FDC0F34110B5E60D20FFF7DDFD07
:10C7C0002B685B0103F0600320F06001C6E70D20D9
:10C7D000FFF7D3FD2B6820F00F0103F00F03BDE737
:10C7E00028B90620FFF7C9FDC0F300409BE60E20E4
:10C7F000FFF7C3FD2B681B0403F4803320F4803162
:10C8000019430E20EAE660B90620FFF7B6FD000ADC
:10C8100000F07F0310F0400018BF6FF07F00184356
:10C8200081E60E20FFF7A9FD2B681B0203F4FE43EF
:10C8300020F4FE41E4E728B90720FFF79EFDC0F38E
:10C84000813070E60F20FFF798FD2B689B039BB2A9
:10C8500020F4404119430F20C0E628B90720FFF714
:10C860008CFDC0F301305EE60F20FFF786FD2B68DC
:10C870001B0303F4405320F44051EBE70F20FFF774
:10C880007CFD2B689B0203F4806320F48061E1E768
:10C8900028B90720FFF771FDC0F3012043E60F2000
:10C8A000FFF76BFD2B681B0203F4407320F440710B
:10C8B000D0E728B90720FFF760FDC0F3801032E60B
:10C8C0000F20FFF75AFD2B689B0103F0400320F077
:10C8D0004001BFE700287FF480AD0220FFF74DFD47
:10C8E000C0F384201FE618B9002012F03FFD1AE6BD
:10C8F0001168002012F0DAFC1CE612681A6119E6D1
:10C9000028B90720FFF739FDC0F3C0100BE60F2050
:10C91000FFF733FD2B68DB01DBB220F0800199E7E4
:10C9200028B90420FFF729FDC0F34030FBE50C20B7
:10C93000FFF723FD2B685B0303F4005320F4005141
:10C94000B2E60F20FFF719FD2B681B0403F48033B8
:10C9500020F480317EE700287FF43FAD0E4B1B684A
:10C960003BB10220FFF709FD800A00F478702860CF
:10C97000E0E50120FFF701FDC0F38920F7E700287B
:10C980007FF42BAD0320FFF7F8FCC0B2CBE51268B3
:10C990005A60CFE51024C7E56C00FF1F0B4611B9A4
:10C9A00001461846FEE40820704707B5019239B9E0
:10C9B000014601AA0120FFF7F5FC03B05DF804FB76
:10C9C0000820FAE710B508461446FFF7D6FC2060A9
:10C9D00010BDF8B506460020FFF7CFFC274D284CC8
:10C9E0006B7EC0F3C017BB4208D0002F3ED0217829
:10C9F00001F01F010620FFF785FC6F76214A217A9E
:10CA0000136F002934D043F00103617A002932D03A
:10CA100043F002030020136712F070FC2369AA7E22
:10CA20000028B8BF4042984234BF00270127BA42CD
:10CA300010D098424FF00D002CBF647B247BFFF791
:10CA40009CFC04F00F0420F00F0121430D20FFF7A0
:10CA500059FCAF760C4B0A4A1B683146002013F094
:10CA600060FA0020BDE8F84012F068BBE17ABFE749
:10CA700023F00103C9E723F00203CBE7D415FF1F1E
:10CA80004842FF1F6434FF1F9442FF1F10B4062961
:10CA90000C4C0D4BC2F3130004BF02F01F02E272F4
:10CAA0001B6801F0770242F0080203EB8203586032
:10CAB000A37A23B940EA414010BCFFF7CBBB10BCBE
:10CAC000704700BF4842FF1F9442FF1F10B5084B3C
:10CAD0009B7A0C4623B90B0702D40846FFF735FCB6
:10CAE000044B196804F07F0401EB8404606810BDF6
:10CAF0004842FF1F9442FF1FF8B58B0C0C460DD027
:10CB0000C1F34243062B09D1234B5A7A21F01F046B
:10CB1000002A3AD01B7803F01F031C431F4F204EFE
:10CB20003B68204D9B680021C4F307409847EA7E8C
:10CB3000336803EB8203000258603B6800219B6866
:10CB4000C4F307209847EB7E326802EB8302012191
:10CB5000536818433B68000250609B68E0B29847F6
:10CB60003268E97E02EB81014B6818430011A30C87
:10CB7000486010610BD0C4F34243072B02D1C4F3C9
:10CB80000111E97643F0080302E0DB7AC3E70823EA
:10CB900002EB83035C60F8BD4842FF1F9042FF1F19
:10CBA0009442FF1FD415FF1F2DE9F041454E464B1F
:10CBB000DFF86C81454C012730461F6013F092F975
:10CBC000D8F80C506B6803F16402E26003F1840250
:10CBD00003F59270226103F5A27203F501732360DD
:10CBE0002B68A260DB68606098472B68A068DB68F0
:10CBF00098472B68E068DB6898472B6820691B69B9
:10CC000098472B682068DB689847D8F81030304A7E
:10CC100003F11401116022689A61052333704FF407
:10CC20007A73736012F0B0FBD4E90112236900201B
:10CC300012F0FAFA274B2849D3F880200A602749D6
:10CC4000C2F808122649C2F804120021517011706E
:10CC5000244AC3F88C20244AC3F88820234AC3F806
:10CC60008420234AC3F89020224AC3F8A420224AF1
:10CC7000C3F8A020214AC3F89420214AC3F8982081
:10CC8000204AC3F8B420204AC3F8B0201F4AC3F892
:10CC9000C0201F4AC3F8BC201E4AC3F8B8201E4A51
:10CCA000C3F8CC2083F87C704FF416723221C3E9AC
:10CCB0001D210220194AC3F8C420BDE8F041FFF746
:10CCC0002DBA00BF4842FF1F6C00FF1FD415FF1F85
:10CCD0009042FF1F6434FF1F9442FF1F0FC10000EA
:10CCE000E7C10000C3C10000E5C10000E1C10000D0
:10CCF000DDC100009DC90000ABC90000FDC00000FF
:10CD000035C2000045C30000C5C90000D3C90000FA
:10CD1000B9C00000ADC100001DC100005DC1000030
:10CD2000847E0200F8B5830C04460DD0C0F3424364
:10CD3000062B09D1234B5A7A20F01F04002A3AD03F
:10CD40001B7803F01F031C431F4F204E3B68204DF0
:10CD50009B680021C4F3074098472A78336803EBA7
:10CD60008203000258603B6800219B68C4F30720DF
:10CD700098472B78326802EB8302012153681843ED
:10CD80003B68000250609B68E0B29847326829789F
:10CD900002EB81014B6818430011A30C486010613D
:10CDA0000BD0C4F34243072B02D1C4F30111297005
:10CDB00043F0080302E0DB7AC3E7082302EB8303B6
:10CDC0005C60F8BD9C42FF1F9842FF1FE442FF1FBA
:10CDD000FC15FF1F012810B514460CD003D3022800
:10CDE00010D0042006E01368094AB3FA83F35B0904
:10CDF0009372002010BD1368064AB3FA83F35B09EF
:10CE00001360F6E7084612F0EDF92060F1E700BF85
:10CE10009C42FF1F7000FF1F10B5044618B912F0A6
:10CE200081F9204610BD0820FCE7024B186813F07A
:10CE300096B900BFE442FF1F022804BF0B4B93F8D2
:10CE4000D80030B90A4BDB681B685B69094A106976
:10CE50001847012809D1054B93F8D830012B04D18C
:10CE6000034BDB681B689B69F0E770476434FF1F66
:10CE7000847E0200FC15FF1F38B50020FFF7DCFFA1
:10CE80000F4B104CDD6820692B685B6998472B6855
:10CE900060689B6898472B68E0689B6898472B6898
:10CEA00020699B6898472B6860699B6898472B6846
:10CEB000A0689B689847BDE8384012F0B3BA00BF3D
:10CEC000847E0200FC15FF1F38B50D46044620B9CC
:10CED00012F014FA2860204638BD0820FCE710B58F
:10CEE000044628B9034B188112F010F9204610BDF2
:10CEF0000820FCE79C42FF1F0021F0E74942EEE7D3
:10CF0000EDE738B5002012F0F9F90546A8B90C4B49
:10CF10000C48196813F006F90B4B022001241C6021
:10CF2000FFF78AFF12F030FA084928464B69D1E929
:10CF3000021212F079F9204638BD0020FCE700BF4C
:10CF4000E442FF1F9C42FF1F7000FF1FFC15FF1FE4
:10CF50000346C1F31300820C10B40B4C05D04214ED
:10CF6000062A04BF01F01F01E172084A03F07703AB
:10CF7000126843F0080302EB83035860A37A0BB9ED
:10CF800010BCCFE610BC70479C42FF1FE442FF1F5D
:10CF900008461146DCE710B5074B9B7A04461BB9DF
:10CFA000030701D400F070FB044B1B6804F07F04FE
:10CFB00003EB8404606810BD9C42FF1FE442FF1F26
:10CFC000A829F8B504460E46154600F0C7815BD87F
:10CFD0001D2900F0D38021D8042900F0D6800CD878
:10CFE000012900F0B880C0F0AA80022900F0BC80BE
:10CFF000032900F0C3800424A5E0062900F0DA80AC
:10D00000C0F0CF80072900F0E9800829F3D100287B
:10D01000F1D112F0E7F8C0F3001093E0A32900F07B
:10D0200055811ED8A02900F026810CD88C29E2D188
:10D03000002840F0E5800820FFF7ADFF00F00F006A
:10D04000C0F108007EE0A12900F02581A229D2D1FB
:10D050000C20002C40F02F81FFF79DFFC0F3C13062
:10D0600070E0A52900F05281C0F04081A62900F0AF
:10D070005D81A729BFD10C20002C40F06781FFF70C
:10D080008AFF00F00F005DE0B22900F00A8226D886
:10D09000AD2900F0AE810FD8AA2900F08581C0F03B
:10D0A0007281AB2900F09181AC29A4D1AF4B00284B
:10D0B00040F09C815B7B80E0AF2900F0C581C0F02F
:10D0C000AB81B02900F0D281B12994D1002840F081
:10D0D000DE810720FFF75FFFC0F3802032E0B72931
:10D0E00000F0178210D8B42900F0FD81C0F0EA8169
:10D0F000B52900F00182B6297FF47DAF9B4B002853
:10D1000040F004821B6958E0CE2900F02D820AD835
:10D11000B82900F00E82B9297FF46DAF002840F0E5
:10D120001982072067E1D02900F03282D6297FF4E6
:10D1300062AF8E4B002840F033825B683DE020B93F
:10D1400012F0CEF828602046F8BD1168002011F0DA
:10D15000E9FF0024F7E710B912F0B6F8F2E711681A
:10D16000002012F08BF8F4E718B9002012F0D4F880
:10D17000E8E71168002011F0C9FFEAE7002C7FF40E
:10D180003AAF204612F0BAF8DCE710B912F0E0F836
:10D19000D8E711680029B8BF4942002012F07CF896
:10D1A000D7E710B912F0C6F8CCE71168002012F0EA
:10D1B0006AF9CEE76D4F10B9FB7A2B60C3E71368AD
:10D1C000FB720020FFF7E7FE10F08004C1D1F97A6E
:10D1D000304601F01F01FFF7BBFEB4E7634E08B90C
:10D1E0003378EAE7136833700020FFF7D4FE0306B4
:10D1F000AFD53178062001F01F01FFF7A9FEA8E79F
:10D200001368102B31D00DDC022B2AD004DC012B4B
:10D2100016D04FF0FF3314E0042B24D0082BF8D1A4
:10D2200005230EE0402B22D003DC202BF1D1032379
:10D2300007E0802B1DD0B3F5807FEAD1002300E00A
:10D2400008232B602B68013300F0AD810820FFF725
:10D25000A2FE2B6820F00F0103F00F0319430820F2
:10D26000CBE70723EDE70623EBE70423E9E70223F7
:10D27000E7E70123E5E7082024B9FFF78CFEC0F3B8
:10D2800040205FE7FFF787FE2B685B0203F4007323
:10D2900020F40071E2E7082024B9FFF77CFEC0F318
:10D2A00000204FE7FFF777FE2B681B0203F4807323
:10D2B00020F48071D2E7FFF76EFE2B68DB0303F4E6
:10D2C000C03320F4C03119430C2096E70C2024B958
:10D2D000FFF761FEC0F3803034E7FFF75CFE2B6898
:10D2E0009B0303F4804320F48041ECE70C2024B935
:10D2F000FFF751FEC0F3C12024E7FFF74CFE2B6877
:10D30000DB0203F4C05320F4C051DCE70C2024B945
:10D31000FFF741FEC0F3C31014E7FFF73CFE2B6894
:10D32000DB0103F4F06320F4F061CCE70C2024B9B6
:10D33000FFF731FEC0F3021004E7FFF72CFE2B6865
:10D340001B0103F0700320F07001BCE7FFF723FE20
:10D350002B6820F00F0103F00F03B4E740B905205C
:10D36000FFF719FEC0F3C030ECE600BF9C42FF1F80
:10D370000D20FFF710FE2B68DB039BB220F4004169
:10D3800019430D2039E728B90520FFF704FEC0F343
:10D390004130D7E60D20FFF7FEFD2B685B0303F459
:10D3A000C04320F4C041EBE728B90520FFF7F3FDA7
:10D3B000C0F30320C6E60D20FFF7EDFD2B681B022E
:10D3C00003F4706320F47061DAE728B90520FFF7F1
:10D3D000E2FDC0F34110B5E60D20FFF7DCFD2B6840
:10D3E0005B0103F0600320F06001C9E712685A7323
:10D3F000AFE628B90620FFF7CEFDC0F30040A1E656
:10D400000E20FFF7C8FD2B681B0403F4803320F4C3
:10D41000803119430E20F0E660B90620FFF7BBFD0E
:10D42000000A00F07F0310F0400018BF6FF07F008B
:10D43000184387E60E20FFF7AEFD2B681B0203F4AE
:10D44000FE4320F4FE41E4E728B90720FFF7A3FDDF
:10D45000C0F3813076E60F20FFF79DFD2B689B031C
:10D460009BB220F4404119430F20C6E628B907209B
:10D47000FFF791FDC0F3013064E60F20FFF78BFD4D
:10D480002B681B0303F4405320F44051EBE70F20BB
:10D49000FFF781FD2B689B0203F4806320F4806119
:10D4A000E1E728B90720FFF776FDC0F3012049E640
:10D4B0000F20FFF770FD2B681B0203F4407320F46C
:10D4C0004071D0E728B90720FFF765FDC0F3801051
:10D4D00038E60F20FFF75FFD2B689B0103F0400348
:10D4E00020F04001BFE700287FF485AD0220FFF760
:10D4F00052FDC0F3842025E618B9002011F036FF54
:10D5000020E61168002011F0D1FE22E612681A61AF
:10D510001FE628B90720FFF73EFDC0F3C01011E653
:10D520000F20FFF738FD2B68DB01DBB220F0800114
:10D5300099E728B90420FFF72EFDC0F3403001E63B
:10D540000C20FFF728FD2B685B0303F4005320F445
:10D550000051B8E60F20FFF71EFD2B681B0403F4F3
:10D56000803320F480317EE700287FF444AD0F4BF8
:10D570001B683BB10220FFF70EFD800A00F47870B3
:10D580002860E6E50120FFF706FDC0F38920F7E7F4
:10D5900000287FF430AD0320FFF7FDFCC0B2D1E5D9
:10D5A00012685A60D5E51024CDE500BF7000FF1F5A
:10D5B0000B4611B90146184602E50820704710B520
:10D5C00008461446FFF7E7FC206010BDF8B5064694
:10D5D0000020FFF7E0FC284D284C2B7FC0F3C0173C
:10D5E000BB4208D0002F3ED0217801F01F01062059
:10D5F000FFF7AEFC2F77224A217A136F002934D02F
:10D6000043F00103617A002932D043F00203002085
:10D61000136711F073FE23696A7F0028B8BF404288
:10D62000984234BF00270127BA4210D098424FF0E9
:10D630000D002CBF647B247BFFF7ADFC04F00F04CE
:10D6400020F00F0121430D20FFF782FC6F770D4B77
:10D650000A4A1B683146002012F011FD0020BDE887
:10D66000F84011F06BBDE17ABFE723F00103C9E791
:10D6700023F00203CBE700BFFC15FF1F9C42FF1FF6
:10D680006434FF1FE442FF1F38B504460F20FFF744
:10D6900082FC0323B4FBF3F303EB4303E41A0546D4
:10D6A000E4B220F0300040EA0410FFF73BFB2846CC
:10D6B000BDE83840FFF736BB38B50D46044648B9DB
:10D6C00011F002FE2B68C1182960204611F02AFDD6
:10D6D000204638BD0820FCE707B5019239B901465C
:10D6E00001AA0120FFF76CFC03B05DF804FB0820E1
:10D6F000FAE7C2F31300830C10B40C4C05D04314AA
:10D70000062B04BF02F01F02E272094B01F0770101
:10D710001B6841F0080103EB81014860A37A13B94B
:10D7200010BCFFF7FFBA10BC704700BF9C42FF1F40
:10D73000E442FF1F10B5084B9B7A0C4623B90B0738
:10D7400002D40846FFF7A0FF044B196804F07F04D9
:10D7500001EB8404606810BD9C42FF1FE442FF1F80
:10D76000F8B58B0C0C460DD0C1F34243062B09D102
:10D77000234B5A7A21F01F04002A3AD01B7803F079
:10D780001F031C431F4F204E3B68204D9B68002108
:10D79000C4F307409847AA7F336803EB8203000273
:10D7A00058603B6800219B68C4F307209847AB7F13
:10D7B000326802EB83020121536818433B68000280
:10D7C00050609B68E0B298473268A97F02EB810104
:10D7D0004B6818430011A30C486010610BD0C4F3D0
:10D7E0004243072B02D1C4F30111A97743F0080388
:10D7F00002E0DB7AC3E7082302EB83035C60F8BD39
:10D800009C42FF1F9842FF1FE442FF1FFC15FF1FB1
:10D810002DE9F041454E464BDFF86C81454C012720
:10D8200030461F6012F00CFCD8F80C506B6803F106
:10D830006402226103F1840203F59270626103F5D0
:10D84000A27203F5017363602B68E260DB68A0607D
:10D8500098472B68E068DB6898472B682069DB688D
:10D8600098472B6860691B6998472B686068DB687C
:10D870009847D8F81030304A03F1140111606268FB
:10D880009A61052333704FF47A73736011F07CFD55
:10D89000D4E902126369002011F0C6FC274B284925
:10D8A000D3F880200A602749C2F808122649C2F836
:10D8B0000412002151701170244AC3F88C20244AAC
:10D8C000C3F88820234AC3F88420234AC3F8902051
:10D8D000224AC3F8A420224AC3F8A020214AC3F850
:10D8E0009420214AC3F89820204AC3F8B420204A43
:10D8F000C3F8B0201F4AC3F8C0201F4AC3F8BC2099
:10D900001E4AC3F8B8201E4AC3F8CC2083F87C70A6
:10D9100040F225123221C3E91D210220194AC3F821
:10D92000C420BDE8F041FFF787BA00BF9C42FF1F4B
:10D930007000FF1FFC15FF1F9842FF1F6434FF1F7C
:10D94000E442FF1F2BCE000003CF0000DFCE00001B
:10D9500001CF0000FDCE0000F9CE0000B1D50000DF
:10D96000D9D6000019CE0000B9D6000091CF000032
:10D97000BFD50000CDD50000D5CD0000C9CE000038
:10D9800039CE000079CE0000847E0200014B0022D7
:10D990005A6070476434FF1F70B5184E184CF56814
:10D9A00060682B689B6998472B68A0699B689847BB
:10D9B0002B6860699B6898472B6820699B6898472B
:10D9C0002B68E0689B6898472B68A0689B6898471D
:10D9D0002B68206A9B6898472B68E0699B6898478A
:10D9E0002B6820689B6898472B6860689B689847FD
:10D9F0003369BDE870405B6A184700BF847E02004F
:10DA00002816FF1F022870B5144649D004D890B1DB
:10DA1000012836D0042432E003284FD0FF28F9D162
:10DA20002B4CD4F88030D3F8043298476369D3F88C
:10DA30000432984703E0126832F0030301D0002457
:10DA40001DE0244B244DDE6868693368D2070AD58F
:10DA50001B69984724683268A86914F0020408D04A
:10DA600013699847EBE7DB689847336868699B69F7
:10DA7000EFE7D36898473368A8699B6998472046C1
:10DA800070BD144B144DDE681468286933680CB1FE
:10DA90001B69E6E7DB689847336828699B69EDE70F
:10DAA0000C4B0D4DDE6814683368A868002CEFD16C
:10DAB000DB6898473368A8689B69DFE7012107485E
:10DAC00012F080FC20600028B9D12024D7E700BFE5
:10DAD0006434FF1F847E02002816FF1FEC42FF1FE4
:10DAE0000146014812F024BDEC42FF1F10B5034867
:10DAF000144612F096FB206010BD00BFEC42FF1FE1
:10DB0000014812F080BB00BFEC42FF1F08B5034B79
:10DB100003485A6A12F046FC002008BD2816FF1F71
:10DB2000EC42FF1F08B5034B03485A6A12F01EFC73
:10DB3000002008BD2816FF1FEC42FF1F08B500217A
:10DB4000024812F0F5FB002008BD00BFEC42FF1FA9
:10DB500008B54942024812F0EBFB002008BD00BFA7
:10DB6000EC42FF1F08B5024812F0E2FB002008BD9E
:10DB7000EC42FF1F38B5094B094CDD6860682B6823
:10DB80009B69984701200EF03BFB2B6860685B693E
:10DB90009847044812F0A1FB012038BD847E0200A2
:10DBA0002816FF1FEC42FF1F38B5094B094CDD68F2
:10DBB00060682B689B69984701200EF021FB2B6859
:10DBC00060685B699847044812F072FB012038BD19
:10DBD000847E02002816FF1FEC42FF1F6E2970B5DD
:10DBE0000446154600F0B3816FD8122900F0638116
:10DBF00037D8052900F0208117D8022900F00081CC
:10DC000007D8002900F0E780012900F0F380042400
:10DC1000E7E0032900F001810429F8D1B24E002881
:10DC200040F00081736A2B60DBE00F2900F028814F
:10DC30000DD8082900F013810E29E8D1002840F002
:10DC400018812021A94812F0ECFA4000C8E0102900
:10DC500000F01C811129DAD1002840F0238129210C
:10DC6000ECE0182900F0558117D8152900F038810B
:10DC700009D8132900F025811429C8D1002840F0C3
:10DC80002C812621A9E0162900F03A811729BED15E
:10DC9000002840F03B812E219FE01B2900F04881A5
:10DCA00009D8192900F03B811A29B0D1002840F089
:10DCB0003C81332191E06C2900F040816D29A6D18F
:10DCC000002840F04181612187E07E2900F0A88191
:10DCD0003CD8742900F0728119D8712963D009D811
:10DCE0006F2900F04481702991D1002840F04F81C4
:10DCF000592172E0722900F04D81732987D10028E3
:10DD000040F05981794B1B68D3F86C318BE7772948
:10DD100000F077810FD8752900F0598176297FF4BA
:10DD200076AF72480368D3F87021002C40F0608110
:10DD3000C2F307422BE07C2900F069817D297FF442
:10DD400066AF002840F069815F2146E0892900F034
:10DD5000AA811ED8852900F08B810AD8812900F07C
:10DD6000708184297FF453AF00287FF450AF652180
:10DD700033E0862900F0898188297FF448AF5B4829
:10DD80000368D3F89021002C40F08581D2B22A603C
:10DD900027E0D12900F0A68112D88A2900F09281CB
:10DDA000C8297FF434AF05215048002C00F0E280F0
:10DDB00012F037FA2A7820F0FF000243052114E020
:10DDC000D42900F09581D6297FF421AF002840F0B6
:10DDD0009781152101E030B93721444812F021FA2A
:10DDE0002860204670BD12683721404812F00BFAB7
:10DDF0000024F6E708B92121EFE712682121F4E7B2
:10DE000028B92421394812F00CFA0012E8E710680A
:10DE100012F07CFA24210246E7E700287FF4F7AEEF
:10DE20002221DAE7136831487362202112F0F9F9F0
:10DE30004207DDD5706AEBE728B928212B4812F09C
:10DE4000F0F98010CCE71268940DA405002C40F086
:10DE50005C8192002821254812F0D5F9C1E70028FD
:10DE60007FF4D5AE0F21214812F0DBF900F001005C
:10DE7000B6E71368002B0CBF012202222021B4E771
:10DE800008B92521A9E712682521AEE708B92A219A
:10DE9000D4E71268940DA405002C40F0368192005E
:10DEA0002A21D8E71268940DA405002C40F02D819A
:10DEB00092002921CFE708B927218EE71268272190
:10DEC00093E708B92B21B9E71268940DA405002C3B
:10DED00040F01B8192002B21BDE71268262184E7C8
:10DEE00030B92C2179E700BF2816FF1FEC42FF1F35
:10DEF0001268940DA405002C40F007812C21AAE79C
:10DF000008B92D2169E712682D216EE712682E21CC
:10DF10006BE708B92F2160E712682F2165E708B980
:10DF200030215AE7126830215FE7126833215CE73D
:10DF300008B9342151E71268342156E708B9602145
:10DF40004BE71268602150E7126861214DE71C2100
:10DF50006F481CB912F065F9001441E712F061F93D
:10DF60002A68C0F3080040EA02421C213DE71C2158
:10DF700067481CB912F055F9C0B231E712F051F9F7
:10DF80002B6800F47F02C3F308031A43EDE712681D
:10DF900059212AE705215E4824B912F042F9C0F35D
:10DFA00007201DE712F03DF92B681B0220F47F4289
:10DFB0009BB21A4302E712685A2116E720B9544B64
:10DFC0001B68D3F870312EE612685B210DE7504BC9
:10DFD0001B68D3F8703110B9C3F30E0323E612683F
:10DFE00023F4FF4323F07F03C2F30E021A43ECE74E
:10DFF0002B681B0422F47F0203F47F031A435B2186
:10E00000F4E608B95E21E8E612685E21EDE608B99B
:10E010005C21E2E612685C21E7E612685F21E4E633
:10E0200005213B4824B912F0FCF8C0F30740D7E6BD
:10E0300012F0F7F82B681B0420F47F0203F47F032F
:10E04000B7E700283FF4D4AE14684CB10121304842
:10E0500012F0B8F9286000287FF4CAAE2024C0E688
:10E0600007212B4812F0DDF8072120F48002F2E6A8
:10E0700000287FF4BDAE0721254812F0D2F8C0F386
:10E080008150431E58425841AAE608B95221A4E6DD
:10E0900012685221A9E62B6822F0FF0203F00F0359
:10E0A0001A436321A2E61A480368D3F8902114B9F1
:10E0B000C2F303226BE62B681B0222F4706203F4A6
:10E0C0007063EDE7124B1B68D3F8902100283FF4F2
:10E0D0002FAE2B681B0422F47F0203F47F031A4344
:10E0E000632182E608B9502177E6126850217CE668
:10E0F00018B9074B1B689B6995E51268532174E6B4
:10E100001368044A15215A436FE6102469E600BFDC
:10E11000EC42FF1F007102000B4611B90146184680
:10E120005CE50820704708B5024812F001F90020AC
:10E1300008BD00BFEC42FF1F07B5019239B9014687
:10E1400001AA0120FFF74AFD03B05DF804FB082097
:10E15000FAE7034B1B680846DB681146184700BF07
:10E16000E842FF1FF8B5484D484F494B6A69494896
:10E17000494C002112F07EF8FE68736803F1E40256
:10E18000226203F58272E26103F55172A26103F526
:10E190005972626103F56172226103F5697203F5D8
:10E1A0007970E26003F5717203F20443236033680F
:10E1B000A260DB68606098473368A069DB689847B5
:10E1C00033686069DB68984733682069DB68984783
:10E1D0003368E068DB6898473368A068DB68984775
:10E1E000336860685B6998473368A0695B699847E2
:10E1F000336860695B699847336820695B69984751
:10E200003368E0685B6998473368A0685B69984742
:10E210003368206A1B6998473368E0691B6998472F
:10E22000336820681B6998471C4B3A691A60736809
:10E2300003F5317353606B69002159701849C3F8B5
:10E240000412012217491A70C3F80812164B2B62E8
:10E25000164BEB61164BAB61164B6B62164BAB6307
:10E26000164B6B63164BAB62164BEB62164BAB64F3
:10E27000164B6B64164B6B65164B2B65164BEB659B
:10E28000164B2A74AB65F8BD6434FF1F847E020010
:10E290007C720200EC42FF1F2816FF1FE842FF1F9E
:10E2A000A9DB000075DB000027E1000065DB000052
:10E2B00051DB00003DDB000019E1000039E1000006
:10E2C00025DB00000DDB000001DB0000EDDA0000C3
:10E2D000E1DA000005DA00008DD9000099D90000CC
:10E2E000014B00225A6070476434FF1F022870B54A
:10E2F000144648D004D8A0B1012835D004200FE03E
:10E3000003280CD0FF28F9D1264CD4F88030D3F85C
:10E31000043298476369D3F80432984716E0202006
:10E3200070BD126832F00303FAD11F4B1F4DDE6837
:10E3300068693368D2070BD51B699847246832682F
:10E34000A86914F0020409D0136998470020E7E790
:10E35000DB689847336868699B69EEE7D36898473C
:10E360003368A8699B69F0E70F4B104DDE681468AD
:10E37000286933680CB11B69E7E7DB6898473368A5
:10E3800028699B69E1E7084B084DDE68146833682B
:10E39000A868002CEFD1DB6898473368A8689B69B0
:10E3A000D3E700BF6434FF1F847E02006016FF1FA6
:10E3B00070B5184E184CF56860682B689B699847D3
:10E3C0002B68A0699B6898472B6860699B68984791
:10E3D0002B6820699B6898472B68E0689B68984782
:10E3E0002B68A0689B6898472B68206A9B689847B1
:10E3F0002B68E0699B6898472B6820689B68984762
:10E400002B6860689B6898473369BDE870405B6A19
:10E41000184700BF847E02006016FF1F0A460146AF
:10E42000014812F039B900BF8445FF1F0146014879
:10E4300012F0DCB98445FF1F10B50348144612F0F2
:10E4400002F9206010BD00BF8445FF1F014812F093
:10E45000ECB800BF8445FF1F08B5034B03485A6A58
:10E4600012F052FA002008BD6016FF1F8445FF1FFE
:10E4700008B5034B03485A6A12F02AFA002008BD77
:10E480006016FF1F8445FF1F08B50021024812F0E7
:10E4900001FA002008BD00BF8445FF1F08B54942AE
:10E4A000024812F0F7F9002008BD00BF8445FF1FA5
:10E4B00008B5024812F0EEF9002008BD8445FF1FA0
:10E4C00038B5094B094CDD6860682B689B69984733
:10E4D00001200DF095FE2B6860685B699847044841
:10E4E00012F06BF9012038BD847E02006016FF1F18
:10E4F0008445FF1F38B5094B094CDD6860682B68FF
:10E500009B69984701200DF07BFE2B6860685B6972
:10E510009847044812F03CF9012038BD847E02007F
:10E520006016FF1F8445FF1F70B5114C94F86C30C6
:10E53000012B0D4619D0032B0BBF002228220C23E0
:10E540000F2343F0884343F0401343EA423204214F
:10E5500012F06BF8D4F88030012D0CBFD3F80432E0
:10E56000D3F80832BDE87040184700220B23E8E7D3
:10E570006434FF1F2DE9F8433A4CD4E90A564FEAB8
:10E58000062949EA1569C6B24FEA0528002748EA74
:10E59000060249EA0703D4E90E7694F83000350EF6
:10E5A0000130360246EA1766C0B23F02C4E90A23C8
:10E5B00084F83000C4E90E7600294FD0042804D92D
:10E5C0001A466D21284812F030F8A26A26486C21BC
:10E5D00012F02BF801200DF013FEA26A22486C21E4
:10E5E00012F023F894F830304FF00009042BC4E9FE
:10E5F0000E990CD96F211C4812F025F8D4E90E238E
:10E60000074643EA070142EA0900C4E90E016E2108
:10E61000154812F018F8D4E90E2343EAE07794F88D
:10E620003030C3F10803DB0042EA000630463946C9
:10E63000A3F12007C3F1200601FA03F200FA07F75D
:10E6400020FA06F63A4332439840C4E90E0200230A
:10E650000022C4E90A23002384F830302846BDE8AC
:10E66000F88300BF6016FF1F8445FF1F08B50248EE
:10E6700012F010F9002008BD8445FF1F38B515467B
:10E680000C4600297AD1112868D01FD804284ED012
:10E6900008D8012840D03AD302283FD0032844D0DC
:10E6A000042447E00E284DD00AD8052844D0082875
:10E6B000F6D10F21324811F0C6FF00F0010032E020
:10E6C0000F2849D01028EBD12A2136E017284DD049
:10E6D0000ED8142846D005D8122841D01328DFD1EF
:10E6E0002B212AE015283FD01628D9D12D210FE063
:10E6F0001A283FD005D818283AD01928D0D130216F
:10E7000006E01B2838D0D628CAD1152100E03721D1
:10E710001B4811F098FF06E02121F9E72421184851
:10E7200011F091FF0012286004E02221F0E7154B60
:10E730005B6A1360204638BD2821114811F083FF21
:10E740008010F0E720210E4811F07DFF00F003005B
:10E75000831E58425841E6E72521D9E72921ECE7F5
:10E760002721D5E72621D3E72C21D1E72E21CFE79A
:10E770002F21CDE73321CBE73421C9E70824D9E79E
:10E780008445FF1F6016FF1F38B514460D4600294B
:10E7900040F0878012286DD021D805285CD008D899
:10E7A00001283FD038D302283ED0042842D0042587
:10E7B00036E00F2856D007D80E28F8D1002A14BF0B
:10E7C00002220122202128E010284DD01128EED16C
:10E7D000930D9B05002B66D19200292137E0172865
:10E7E00057D008D814284DD046D315284CD0162819
:10E7F000DDD12D2111E01A284FD005D818284AD094
:10E800001928D4D1302108E01B2848D0D628CED1F1
:10E81000264A1521624300E03721254811F005FF03
:10E82000284638BD2121F8E782EAE272A2EBE472C1
:10E830002421F2E71F4D1E486A62202111F003FFD8
:10E84000430707D5686A12F013F8242102461848D6
:10E8500011F0EBFE0025E3E7950DAD051DBB920021
:10E860002821DAE72521D8E7950DAD05DDB992001D
:10E870002A21D2E72721D0E7950DAD059DB9920059
:10E880002B21CAE72621C8E7950DAD055DB92C21DE
:10E89000C3E72E21C1E72F21BFE73321BDE7342194
:10E8A000BBE70825BCE71025BAE700BF00710200EE
:10E8B0008445FF1F6016FF1F024B1B680846DB687C
:10E8C000114618478045FF1FF8B54D4D4D4C4E4B36
:10E8D0006A694E4F2046002111F03CFF4C4920460A
:10E8E00011F080FFFE684B4C736803F1E402226272
:10E8F00003F58272E26103F55172A26103F5597268
:10E90000626103F56172226103F5697203F5797042
:10E91000E26003F5717203F2044323603368A2607E
:10E92000DB68606098473368A069DB6898473368A4
:10E930006069DB68984733682069DB68984733680B
:10E94000E068DB6898473368A068DB6898473368FD
:10E9500060685B6998473368A0695B69984733686A
:10E9600060695B699847336820695B6998473368D9
:10E97000E0685B6998473368A0685B6998473368CB
:10E98000206A1B6998473368E0691B6998473368B8
:10E9900020681B699847204B3A691A60736803F531
:10E9A000317353606B69002159701C49C3F804121C
:10E9B00001221B491A70C3F808121A4B6B661A4BD6
:10E9C0002B621A4BEB611A4BAB611A4B6B621A4B01
:10E9D000AB631A4B6B631A4BAB621A4BEB621A4B6D
:10E9E000AB641A4B6B641A4B6B651A4B2B651A4B55
:10E9F000EB651A4BAB651A4B2A74AB66F8BD00BFCA
:10EA00006434FF1F8445FF1F7C740200847E020073
:10EA100029E500006016FF1F8045FF1FF5E4000098
:10EA2000C1E4000075E500006DE60000B1E40000FF
:10EA30009DE4000089E400007DE6000089E7000015
:10EA400071E4000059E400004DE4000039E40000E6
:10EA50002DE40000EDE20000E1E20000B1E300007F
:10EA60001DE40000014B00225A6070476434FF1F10
:10EA700070B5184E184CF56860682B689B6998470C
:10EA80002B68A0699B6898472B6860699B689847CA
:10EA90002B6820699B6898472B68E0689B689847BB
:10EAA0002B68A0689B6898472B68206A9B689847EA
:10EAB0002B68E0699B6898472B6820689B6898479B
:10EAC0002B6860689B6898473369BDE870405B6A53
:10EAD000184700BF847E0200B016FF1F0A46014699
:10EAE000014811F08FBF00BF1C48FF1F022870B5FE
:10EAF000144649D004D890B1012836D0042432E01D
:10EB000003284FD0FF28F9D12B4CD4F88030D3F80C
:10EB1000043298476369D3F80432984703E01268D7
:10EB200032F0030301D000241DE0244B244DDE68A5
:10EB300068693368D2070AD51B6998472468326828
:10EB4000A86914F0020408D013699847EBE7DB6862
:10EB50009847336868699B69EFE7D36898473368DB
:10EB6000A8699B699847204670BD144B144DDE6818
:10EB70001468286933680CB11B69E6E7DB689847BD
:10EB8000336828699B69EDE70C4B0D4DDE6814680E
:10EB90003368A868002CEFD1DB6898473368A86811
:10EBA0009B69DFE70121074812F032F82060002856
:10EBB000B9D12024D7E700BF6434FF1F847E020050
:10EBC000B016FF1F1C48FF1F0146014812F0D6B8BF
:10EBD0001C48FF1F10B50348144611F0EAFE2060E0
:10EBE00010BD00BF1C48FF1F014811F0D4BE00BF7C
:10EBF0001C48FF1F08B5034B03485A6A11F0F8FF81
:10EC0000002008BDB016FF1F1C48FF1F08B5034BAE
:10EC100003485A6A11F0D0FF002008BDB016FF1F4C
:10EC20001C48FF1F08B50021024811F0A7FF002073
:10EC300008BD00BF1C48FF1F08B54942024811F03B
:10EC40009DFF002008BD00BF1C48FF1F08B50248FB
:10EC500011F094FF002008BD1C48FF1F38B5094B78
:10EC6000094CDD6860682B689B69984701200DF0AE
:10EC7000C7FA2B6860685B699847044811F053FF36
:10EC8000012038BD847E0200B016FF1F1C48FF1F04
:10EC900038B5094B094CDD6860682B689B6998475B
:10ECA00001200DF0ADFA2B6860685B699847044855
:10ECB00011F024FF012038BD847E0200B016FF1F32
:10ECC0001C48FF1F70B5114C94F86C30012B0D4699
:10ECD00019D0032B0BBF002228220C230F2343F053
:10ECE000884343F0401343EA4232042111F053FEBB
:10ECF000D4F88030012D0CBFD3F80432D3F8083299
:10ED0000BDE87040184700220B23E8E76434FF1F7A
:10ED10006F2970B50446154600F07D8200F28880A8
:10ED2000122900F0CD813DD8052900F06D8117D85A
:10ED3000022900F03A8107D8002900F01981012941
:10ED400000F02581042419E1032900F04081042901
:10ED5000F8D1B74E002840F04381736A13600DE18B
:10ED60000F2900F07F810ED8082900F065810E2957
:10ED7000E8D1002840F06B812021AE4811F019FE47
:10ED800040002860FAE0102900F07A811129D9D1D9
:10ED9000002840F089812921A64811F00AFE801040
:10EDA0002860EBE0182900F0DB811FD8152900F05E
:10EDB000B0810DD8132900F091811429C2D1002807
:10EDC00040F0A08126219B4811F0F3FD2860D5E09A
:10EDD000162900F0B0811729B4D1002840F0B9817C
:10EDE0002E21944811F0E5FD2860C7E01B2900F0B2
:10EDF000DA810DD8192900F0C1811A29A2D1002881
:10EE000040F0CA8133218B4811F0D3FD2860B5E072
:10EE10006D2900F0DD8100F2E9816C2992D1002892
:10EE200040F0CF816021834811F0C3FD2860A5E048
:10EE30007D2900F0A58248D8752900F04B8222D8A0
:10EE4000722900F018820FD8702900F0FA81712918
:10EE50007FF478AF06217748002C40F0008211F053
:10EE6000A8FDC0B2286089E0732900F01B827429D4
:10EE70007FF468AF002840F023826E4B1B68D3F804
:10EE8000703113607AE0782900F057820ED8762925
:10EE900000F0368277297FF455AF002840F0468293
:10EEA0005E21644811F085FD286067E0792900F053
:10EEB00052827C297FF446AF002840F05A825C21C0
:10EEC0005C4811F076FD286058E0882900F0A782A0
:10EED00028D8842900F0858215D87E2900F05E822A
:10EEE00081297FF42FAF002800F082801468002C65
:10EEF00000F06C8201214F4811F08AFE2860002842
:10EF000076D120243AE0852900F0748286297FF4A6
:10EF100019AF002840F07C825221464811F049FD8B
:10EF200028602BE0C82995D010D8892900F08A8262
:10EF30008A297FF407AF3F480368D3F89021002C5B
:10EF400040F09682C2F307422A6017E0D42900F00D
:10EF5000A282D62900F0AC82D1297FF4F3AE00283A
:10EF600040F092825021334811F023FD286005E0E3
:10EF700030B937212F4811F01CFD2860204670BDA4
:10EF800012682C48372111F006FD0024F6E728B955
:10EF90002121284811F00DFD2860EFE7126825486F
:10EFA000212111F0F8FC0024E8E730B924212148A0
:10EFB00011F0FFFC00122860E0E7106811F0CCFDB2
:10EFC000242102461B4811F0E6FC0024D6E7002865
:10EFD00040F07E822221174811F0EBFC2860CDE73B
:10EFE000136814487362202111F0E3FC420701D436
:10EFF0000024C3E7706A11F0AFFD242102460D48DA
:10F0000011F0C9FC0024B9E730B92821094811F0F2
:10F01000D0FC80102860B1E71268940DA405002C84
:10F0200040F0588292002821024811F0B4FCA5E774
:10F03000B016FF1F1C48FF1F002840F04D820F2113
:10F04000A34811F0B6FC00F00100286096E71368B1
:10F050009F48002B0CBF01220222202111F09BFCB3
:10F0600000248BE728B92521994811F0A2FC2860DB
:10F0700084E712689648252111F08DFC00247DE775
:10F0800030B92A21924811F094FC8010286075E76D
:10F090001268940DA405002C40F0208292002A21D1
:10F0A0008B4811F078FC69E71268940DA405002CD8
:10F0B00040F0168292002921854811F06CFC5DE732
:10F0C00028B92721824811F074FC286056E712689D
:10F0D0007F48272111F05FFC00244FE730B92B2136
:10F0E0007B4811F066FC8010286047E71268940D99
:10F0F000A405002C40F0F68192002B21744811F0F9
:10F100004AFC3BE712687248262111F044FC0024B7
:10F1100034E728B92C216E4811F04BFC28602DE70C
:10F120001268940DA405002C40F0DE812C21684863
:10F1300011F031FC22E728B92D21654811F039FC86
:10F1400028601BE7126862482D2111F024FC00247E
:10F1500014E712685E482E2111F01DFC00240DE713
:10F1600028B92F215A4811F024FC286006E71268BC
:10F1700057482F2111F00FFC0024FFE628B9302159
:10F18000534811F016FC2860F8E612685048302108
:10F1900011F001FC0024F1E612684D48332111F012
:10F1A000FAFB0024EAE628B93421494811F001FCB1
:10F1B0002860E3E612684648342111F0ECFB002495
:10F1C000DCE612684248602111F0E5FB0024D5E638
:10F1D00028B961213E4811F0ECFB2860CEE61268A8
:10F1E0003B48612111F0D7FB0024C7E61C213848B9
:10F1F00024B911F0DEFB00142860BFE611F0D9FB42
:10F200002A68C0F3080040EA02421C21304811F08D
:10F21000C2FB0024B2E61C212D4824B911F0C9FB21
:10F22000C0B22860AAE611F0C4FB2B6800F47F028C
:10F23000C3F308031A431C21254811F0ACFB00243A
:10F240009CE628B95921224811F0B3FB286095E6C5
:10F2500012681F48592111F09EFB00248EE611F020
:10F26000A8FB2A7820F0FF0002430621184811F07D
:10F2700092FB002482E6062115482CB911F099FB77
:10F28000C0F30720286079E611F093FB2B681B027E
:10F2900020F47F429BB21A4306210D4811F07BFBFC
:10F2A00000246BE628B90A4B1B68D3F86C31136055
:10F2B00064E6126806485A2111F06DFB00245DE6F1
:10F2C000126803485B2111F066FB002456E600BF7C
:10F2D0001C48FF1F86480368D3F870311CB9C3F37C
:10F2E0000E0313604AE6126823F4FF4323F07F0302
:10F2F000C2F30E021A435B2111F04DFB00243DE6E0
:10F300007B4B1B68D3F8702118B9C2F307422A60FF
:10F3100034E62B6876481B0403F47F0322F47F0253
:10F320001A435B2111F037FB002427E6126870486E
:10F330005E2111F030FB002420E628B918216C482A
:10F3400011F037FB286019E612686948182111F09E
:10F3500022FB002412E628B91921654811F029FB87
:10F3600028600BE612686248192111F014FB002492
:10F3700004E612685E485C2111F00DFB0024FDE5F7
:10F3800028B95F215A4811F014FB2860F6E512688D
:10F3900057485F2111F0FFFA0024EFE50621544899
:10F3A0002CB911F006FBC0F307402860E6E511F028
:10F3B00000FB2B681B0420F47F0203F47F031A4335
:10F3C00006214B4811F0E7FA0024D7E50721484809
:10F3D00011F0EFFA072120F48002454811F0DBFA22
:10F3E000CCE5002840F082806521414811F0E1FA27
:10F3F0002860C3E500287FF4FBAD07213C4811F0ED
:10F40000D8FAC0F38150431E584258412860B5E5F0
:10F4100012683748522111F0BEFA0024AEE5344894
:10F420000368D3F8902114B9D2B22A60A6E52B68FC
:10F4300022F0FF0203F00F031A43632111F0ABFA2D
:10F4400000249BE52A4B1B68D3F8902118B9C2F31E
:10F4500003222A6092E52B6825481B0203F470639F
:10F4600022F470621A43632111F095FA002485E5B5
:10F470002B681B0403F47F0322F47F021A436321E9
:10F4800011F089FA002479E512681948502111F029
:10F4900082FA002472E520B9154B1B68DB69136002
:10F4A0006CE512681248532111F075FA002465E5E5
:10F4B00028B915210E4811F07CFA28605EE5136822
:10F4C0000C4A0B485A43152111F065FA002455E502
:10F4D000042453E5102451E504244FE510244DE5A0
:10F4E00010244BE5102449E5102447E5042445E5A4
:10F4F0001C48FF1F007102000B4611B90146184657
:10F5000006E4082070472DE9F8433A4CD4E90A563E
:10F510004FEA062949EA1569C6B24FEA05280027CD
:10F5200048EA060249EA0703D4E90E7694F8300067
:10F53000350E0130360246EA1766C0B23F02C4E912
:10F540000A2384F83000C4E90E7600294FD004283D
:10F5500004D91A466D21284811F01DFAA26A2648DE
:10F560006C2111F018FA01200CF04AFEA26A224820
:10F570006C2111F010FA94F830304FF00009042B90
:10F58000C4E90E990CD96F211B4811F012FAD4E985
:10F590000E23074643EA070142EA0900C4E90E01C7
:10F5A0006E21154811F005FAD4E90E2343EAE077FD
:10F5B00094F83030C3F10803DB0042EA000630461D
:10F5C0003946A3F12007C3F1200601FA03F200FA3D
:10F5D00007F720FA06F63A4332439840C4E90E0290
:10F5E00000230022C4E90A23002384F8303028468F
:10F5F000BDE8F883B016FF1F1C48FF1F08B502487E
:10F6000011F0BCFA002008BD1C48FF1F07B501928D
:10F6100039B9014601AA0120FFF77AFB03B05DF872
:10F6200004FB0820FAE7034B1B680846DB68114619
:10F63000184700BF1848FF1FF8B54D4D4D4C4E4BB5
:10F640006A694E4F2046002111F03AFA4C49204693
:10F6500011F07EFAFE684B4C736803F1E4022262FB
:10F6600003F58272E26103F55172A26103F55972EA
:10F67000626103F56172226103F5697203F57970C5
:10F68000E26003F5717203F2044323603368A26001
:10F69000DB68606098473368A069DB689847336827
:10F6A0006069DB68984733682069DB68984733688E
:10F6B000E068DB6898473368A068DB689847336880
:10F6C00060685B6998473368A0695B6998473368ED
:10F6D00060695B699847336820695B69984733685C
:10F6E000E0685B6998473368A0685B69984733684E
:10F6F000206A1B6998473368E0691B69984733683B
:10F7000020681B699847204B3A691A60736803F5B3
:10F71000317353606B69002159701C49C3F804129E
:10F7200001221B491A70C3F808121A4B6B661A4B58
:10F730002B621A4BEB611A4BAB611A4B6B621A4B83
:10F74000AB631A4B6B631A4BAB621A4BEB621A4BEF
:10F75000AB641A4B6B641A4B6B651A4B2B651A4BD7
:10F76000EB651A4BAB651A4B2A74AB66F8BD00BF4C
:10F770006434FF1F1C48FF1F7C760200847E020059
:10F78000C5EC0000B016FF1F1848FF1F91EC0000E9
:10F790005DEC000007F50000FDF500004DEC0000F9
:10F7A00039EC000025EC0000F9F400000DF6000033
:10F7B0000DEC0000F5EB0000E9EB0000D5EB0000DC
:10F7C000C9EB0000EDEA000065EA000071EA000004
:10F7D000DDEA0000014B00225A6070476434FF1FCD
:10F7E00070B5184E184CF56860682B689B6998478F
:10F7F0002B68A0699B6898472B6860699B6898474D
:10F800002B6820699B6898472B68E0689B6898473D
:10F810002B68A0689B6898472B68206A9B6898476C
:10F820002B68E0699B6898472B6820689B6898471D
:10F830002B6860689B6898473369BDE870405B6AD5
:10F84000184700BF847E02000017FF1F0A460146CA
:10F85000014811F047BB00BFB04AFF1F022870B536
:10F86000144649D004D890B1012836D0042432E09F
:10F8700003284FD0FF28F9D12B4CD4F88030D3F88F
:10F88000043298476369D3F80432984703E012685A
:10F8900032F0030301D000241DE0244B244DDE6828
:10F8A00068693368D2070AD51B69984724683268AB
:10F8B000A86914F0020408D013699847EBE7DB68E5
:10F8C0009847336868699B69EFE7D368984733685E
:10F8D000A8699B699847204670BD144B144DDE689B
:10F8E0001468286933680CB11B69E6E7DB68984740
:10F8F000336828699B69EDE70C4B0D4DDE68146891
:10F900003368A868002CEFD1DB6898473368A86893
:10F910009B69DFE70121074811F0EAFB206000281E
:10F92000B9D12024D7E700BF6434FF1F847E0200D2
:10F930000017FF1FB04AFF1F0146014811F08EBC9F
:10F94000B04AFF1F10B50348144611F0A2FA206018
:10F9500010BD00BFB04AFF1F014811F08CBA00BFB4
:10F96000B04AFF1F08B5034B03485A6A11F0B0FBB9
:10F97000002008BD0017FF1FB04AFF1F08B5034B4A
:10F9800003485A6A11F088FB002008BD0017FF1FCA
:10F99000B04AFF1F08B50021024811F05FFB0020AC
:10F9A00008BD00BFB04AFF1F08B54942024811F028
:10F9B00055FB002008BD00BFB04AFF1F08B5024834
:10F9C00011F04CFB002008BDB04AFF1F38B5094BB1
:10F9D000094CDD6860682B689B69984701200CF032
:10F9E0000FFC2B6860685B699847044811F00BFBBB
:10F9F000012038BD847E02000017FF1FB04AFF1FA0
:10FA000038B5094B094CDD6860682B689B699847DD
:10FA100001200CF0F5FB2B6860685B69984704488F
:10FA200011F0DCFA012038BD847E02000017FF1FB0
:10FA3000B04AFF1F70B5114C94F86C30012B0D4685
:10FA400019D0032B0BBF002228220C230F2343F0D5
:10FA5000884343F0401343EA4232042111F00BFA89
:10FA6000D4F88030012D0CBFD3F80432D3F808321B
:10FA7000BDE87040184700220B23E8E76434FF1FFD
:10FA80006F2970B50446154600F07D8200F288802B
:10FA9000122900F0CD813DD8052900F06D8117D8DD
:10FAA000022900F03A8107D8002900F019810129C4
:10FAB00000F02581042419E1032900F04081042984
:10FAC000F8D1B74E002840F04381736A13600DE10E
:10FAD0000F2900F07F810ED8082900F065810E29DA
:10FAE000E8D1002840F06B812021AE4811F0D1F917
:10FAF00040002860FAE0102900F07A811129D9D15C
:10FB0000002840F089812921A64811F0C2F980100F
:10FB10002860EBE0182900F0DB811FD8152900F0E0
:10FB2000B0810DD8132900F091811429C2D1002889
:10FB300040F0A08126219B4811F0ABF92860D5E068
:10FB4000162900F0B0811729B4D1002840F0B981FE
:10FB50002E21944811F09DF92860C7E01B2900F080
:10FB6000DA810DD8192900F0C1811A29A2D1002803
:10FB700040F0CA8133218B4811F08BF92860B5E041
:10FB80006D2900F0DD8100F2E9816C2992D1002815
:10FB900040F0CF816021834811F07BF92860A5E017
:10FBA0007D2900F0A58248D8752900F04B8222D823
:10FBB000722900F018820FD8702900F0FA8171299B
:10FBC0007FF478AF06217748002C40F0008211F0D6
:10FBD00060F9C0B2286089E0732900F01B827429A3
:10FBE0007FF468AF002840F023826E4B1B68D3F887
:10FBF000703113607AE0782900F057820ED87629A8
:10FC000000F0368277297FF455AF002840F0468215
:10FC10005E21644811F03DF9286067E0792900F021
:10FC200052827C297FF446AF002840F05A825C2142
:10FC30005C4811F02EF9286058E0882900F0A7826E
:10FC400028D8842900F0858215D87E2900F05E82AC
:10FC500081297FF42FAF002800F082801468002CE7
:10FC600000F06C8201214F4811F042FA2860002810
:10FC700076D120243AE0852900F0748286297FF429
:10FC800019AF002840F07C825221464811F001F95A
:10FC900028602BE0C82995D010D8892900F08A82E5
:10FCA0008A297FF407AF3F480368D3F89021002CDE
:10FCB00040F09682C2F307422A6017E0D42900F090
:10FCC000A282D62900F0AC82D1297FF4F3AE0028BD
:10FCD00040F092825021334811F0DBF8286005E0B3
:10FCE00030B937212F4811F0D4F82860204670BD74
:10FCF00012682C48372111F0BEF80024F6E728B925
:10FD00002121284811F0C5F82860EFE7126825483E
:10FD1000212111F0B0F80024E8E730B9242121486E
:10FD200011F0B7F800122860E0E7106811F084F9CC
:10FD3000242102461B4811F09EF80024D6E7002833
:10FD400040F07E822221174811F0A3F82860CDE709
:10FD5000136814487362202111F09BF8420701D404
:10FD60000024C3E7706A11F067F9242102460D48A8
:10FD700011F081F80024B9E730B92821094811F0C1
:10FD800088F880102860B1E71268940DA405002C53
:10FD900040F0588292002821024811F06CF8A5E743
:10FDA0000017FF1FB04AFF1F002840F04D820F21AF
:10FDB000A34811F06EF800F00100286096E7136880
:10FDC0009F48002B0CBF01220222202111F053F882
:10FDD00000248BE728B92521994811F05AF82860AA
:10FDE00084E712689648252111F045F800247DE744
:10FDF00030B92A21924811F04CF88010286075E73C
:10FE00001268940DA405002C40F0208292002A2153
:10FE10008B4811F030F869E71268940DA405002CA6
:10FE200040F0168292002921854811F024F85DE700
:10FE300028B92721824811F02CF8286056E712686B
:10FE40007F48272111F017F800244FE730B92B2104
:10FE50007B4811F01EF88010286047E71268940D67
:10FE6000A405002C40F0F68192002B21744811F07B
:10FE700002F83BE712687248262110F0FCFF0024CC
:10FE800034E728B92C216E4811F003F828602DE7DB
:10FE90001268940DA405002C40F0DE812C216848E6
:10FEA00010F0E9FF22E728B92D21654810F0F1FF95
:10FEB00028601BE7126862482D2110F0DCFF002447
:10FEC00014E712685E482E2110F0D5FF00240DE7DC
:10FED00028B92F215A4810F0DCFF286006E7126885
:10FEE00057482F2110F0C7FF0024FFE628B9302122
:10FEF000534810F0CEFF2860F8E6126850483021D1
:10FF000010F0B9FF0024F1E612684D48332110F0DB
:10FF1000B2FF0024EAE628B93421494810F0B9FFBD
:10FF20002860E3E612684648342110F0A4FF00245C
:10FF3000DCE612684248602110F09DFF0024D5E6FF
:10FF400028B961213E4810F0A4FF2860CEE612686F
:10FF50003B48612110F08FFF0024C7E61C21384880
:10FF600024B910F096FF00142860BFE610F091FF4E
:10FF70002A68C0F3080040EA02421C21304810F011
:10FF80007AFF0024B2E61C212D4824B910F081FF2D
:10FF9000C0B22860AAE610F07CFF2B6800F47F0254
:10FFA000C3F308031A431C21254810F064FF002402
:10FFB0009CE628B95921224810F06BFF286095E68D
:10FFC00012681F48592110F056FF00248EE610F0E9
:10FFD00060FF2A7820F0FF0002430621184810F045
:10FFE0004AFF002482E6062115482CB910F051FF83
:10FFF000C0F30720286079E610F04BFF2B681B0246
:020000021000EC
:1000000020F47F429BB21A4306210D4810F033FFC3
:1000100000246BE628B90A4B1B68D3F86C311360D7
:1000200064E6126806485A2110F025FF00245DE6B8
:10003000126803485B2110F01EFF002456E600BF43
:10004000B04AFF1F86480368D3F870311CB9C3F368
:100050000E0313604AE6126823F4FF4323F07F0384
:10006000C2F30E021A435B2110F005FF00243DE6A7
:100070007B4B1B68D3F8702118B9C2F307422A6082
:1000800034E62B6876481B0403F47F0322F47F02D6
:100090001A435B2110F0EFFE002427E61268704837
:1000A0005E2110F0E8FE002420E628B918216C48F3
:1000B00010F0EFFE286019E612686948182110F068
:1000C000DAFE002412E628B91921654810F0E1FE95
:1000D00028600BE612686248192110F0CCFE00245B
:1000E00004E612685E485C2110F0C5FE0024FDE5C0
:1000F00028B95F215A4810F0CCFE2860F6E5126856
:1001000057485F2110F0B7FE0024EFE50621544860
:100110002CB910F0BEFEC0F307402860E6E510F0F1
:10012000B8FE2B681B0420F47F0203F47F031A43FC
:1001300006214B4810F09FFE0024D7E507214848D0
:1001400010F0A7FE072120F48002454810F093FE2E
:10015000CCE5002840F082806521414810F099FEEE
:100160002860C3E500287FF4FBAD07213C4810F070
:1001700090FEC0F38150431E584258412860B5E5B7
:1001800012683748522110F076FE0024AEE534485C
:100190000368D3F8902114B9D2B22A60A6E52B687F
:1001A00022F0FF0203F00F031A43632110F063FEF5
:1001B00000249BE52A4B1B68D3F8902118B9C2F3A1
:1001C00003222A6092E52B6825481B0203F4706322
:1001D00022F470621A43632110F04DFE002485E57D
:1001E0002B681B0403F47F0322F47F021A4363216C
:1001F00010F041FE002479E512681948502110F0F2
:100200003AFE002472E520B9154B1B68DB691360C8
:100210006CE512681248532110F02DFE002465E5AC
:1002200028B915210E4810F034FE28605EE51368E9
:100230000C4A0B485A43152110F01DFE002455E5C9
:10024000042453E5102451E504244FE510244DE522
:1002500010244BE5102449E5102447E5042445E526
:10026000B04AFF1F007102000B4611B90146184643
:1002700006E4082070472DE9F8433A4CD4E90A56C1
:100280004FEA062949EA1569C6B24FEA0528002750
:1002900048EA060249EA0703D4E90E7694F83000EA
:1002A000350E0130360246EA1766C0B23F02C4E995
:1002B0000A2384F83000C4E90E7600294FD00428C0
:1002C00004D91A466D21284810F0D5FDA26A2648A7
:1002D0006C2110F0D0FD01200BF092FFA26A2248A1
:1002E0006C2110F0C8FD94F830304FF00009042B59
:1002F000C4E90E990CD96F211B4810F0CAFDD4E94E
:100300000E23074643EA070142EA0900C4E90E0149
:100310006E21154810F0BDFDD4E90E2343EAE077C5
:1003200094F83030C3F10803DB0042EA000630469F
:100330003946A3F12007C3F1200601FA03F200FABF
:1003400007F720FA06F63A4332439840C4E90E0212
:1003500000230022C4E90A23002384F83030284611
:10036000BDE8F8830017FF1FB04AFF1F08B5024819
:1003700010F074FE002008BDB04AFF1F07B50192BF
:1003800039B9014601AA0120FFF77AFB03B05DF8F5
:1003900004FB0820FAE7034B1B680846DB6811469C
:1003A000184700BF444DFF1FF8B54D4D4D4C4E4B07
:1003B0006A694E4F2046002110F0F2FD4C4920465C
:1003C00010F036FEFE684B4C736803F1E4022262C3
:1003D00003F58272E26103F55172A26103F559726D
:1003E000626103F56172226103F5697203F5797048
:1003F000E26003F5717203F2044323603368A26084
:10040000DB68606098473368A069DB6898473368A9
:100410006069DB68984733682069DB689847336810
:10042000E068DB6898473368A068DB689847336802
:1004300060685B6998473368A0695B69984733686F
:1004400060695B699847336820695B6998473368DE
:10045000E0685B6998473368A0685B6998473368D0
:10046000206A1B6998473368E0691B6998473368BD
:1004700020681B699847204B3A691A60736803F536
:10048000317353606B69002159701C49C3F8041221
:1004900001221B491A70C3F808121A4B6B661A4BDB
:1004A0002B621A4BEB611A4BAB611A4B6B621A4B06
:1004B000AB631A4B6B631A4BAB621A4BEB621A4B72
:1004C000AB641A4B6B641A4B6B651A4B2B651A4B5A
:1004D000EB651A4BAB651A4B2A74AB66F8BD00BFCF
:1004E0006434FF1FB04AFF1F7C780200847E020044
:1004F00035FA00000017FF1F444DFF1F01FA0000EE
:10050000CDF90000770201006D030100BDF9000084
:10051000A9F9000095F90000690201007D030100BE
:100520007DF9000065F9000059F9000045F9000067
:1005300039F900005DF80000D5F70000E1F7000090
:100540004DF800000020704701207047014B002249
:100550005A6070476434FF1F1FB5084B33F8084CCE
:100560005A7802949C1E019433F8041C00910146B1
:10057000002011F0E9F804B010BD00BF504DFF1F7E
:1005800010B50020144610F0AFFE206010BD002012
:1005900010F0CCBE10B5044618B910F0C7FF2046C5
:1005A00010BD0820FCE710B5044618B910F0A0FFF4
:1005B000204610BD0820FCE70021F4E74942F2E79D
:1005C000F1E7022804BF0C4B93F8D80030B90B4B6D
:1005D000DB681B689B690A4A10681847012809D123
:1005E000054B93F8D830012B04D1044BDB681B6812
:1005F0005B69F0E7704700BF6434FF1F847E020030
:10060000584DFF1F10B50020FFF7DBFF044B054AD4
:10061000DB6810681B68BDE810409B69184700BF85
:10062000847E0200584DFF1F10B5044620B90968AA
:1006300010F089FF204610BD0820FCE738B50D46B4
:10064000044620B910F06DFF2860204638BD082010
:10065000FCE7043938B504461546FA2900F2398713
:10066000DFE811F0FB003707370737073707370791
:10067000370737073707370737073707370737078A
:10068000370737073707370737073707370737077A
:10069000370737073707370737073707370737076A
:1006A000370737073707370737073707370737075A
:1006B000370737073707370737073707370737074A
:1006C00009011901370729013901370737073707AA
:1006D000370737073707370737073707370737072A
:1006E000370737073707370737073707370737071A
:1006F000370737073707370737073707370737070A
:1007000037073707370737073707370737073707F9
:1007100037073707370737073707370737073707E9
:1007200037073707490157016501730181018F01BF
:100730009D01AB01B901C701D501E301F101FF0141
:100740000D021B02290233023D0237074702510204
:100750005B0265026F027E028D029C02A5023707D2
:1007600037073707AE02B602BE02C802D202370709
:1007700037073707DA02E202EA0237073707370797
:100780003707370737073707F402FE02080312035B
:100790003707370737073707370737071C0326039D
:1007A00030033A034403370737073707370737075C
:1007B0004E0358036803780380038C0396039F035A
:1007C000A903B003BB03C803D503E203EF03FC0393
:1007D00009041604370723042E043B044804530479
:1007E00060046D047A0487049404A304B204C10471
:1007F000D004DF04EE04FD040D052005300540059E
:1008000050056005700580059005A005B005C00580
:10081000CF05370737073707370737073707370752
:100820003707370737073707DE05EE05FE050E06E3
:100830001E062E063E064E065E066D067C068B06DE
:100840009A06A906B806C706D606E406F206000709
:1008500037070E07190727072F0728B9602110F05F
:1008600043FD2860204638BD12686021002010F04A
:100870005DFD0024F6E730B90246082110F076FD50
:1008800000B22860EEE7138800220821104610F01D
:100890007AFD0024E6E730B90246092110F066FD32
:1008A00000B22860DEE7138800220921104610F00C
:1008B0006AFD0024D6E730B90122082110F056FD68
:1008C00000B22860CEE7138808210122002010F032
:1008D0005AFD0024C6E730B90122092110F046FD77
:1008E00000B22860BEE7138809210122002010F021
:1008F0004AFD0024B6E7002840F0EE8501220321DE
:1009000010F014FD22460221204610F02FFD286031
:10091000A8E7002840F0E3850122032110F006FD3E
:1009200001220221204610F021FD28609AE70028CC
:1009300040F0D8850222032110F0F8FC2246022163
:10094000204610F013FD28608CE7002840F0CD858C
:100950000246032110F0EAFC22460221204610F054
:1009600005FD28607EE7002840F0C285024603218D
:1009700010F0DCFC01220221204610F0F7FC286078
:1009800070E7002840F0B7850322114610F0CEFC36
:1009900022460221204610F0E9FC286062E7002888
:1009A00040F0AC850422032110F0C0FC2246022155
:1009B000204610F0DBFC286054E7002840F0A185B9
:1009C0000422032110F0B2FC01220221204610F083
:1009D000CDFC286046E7002840F0968505220321DB
:1009E00010F0A4FC22460221204610F0BFFC286033
:1009F00038E7002840F08B850522032110F096FC93
:100A000001220221204610F0B1FC28602AE70028CC
:100A100040F080850622032110F088FC2246022146
:100A2000204610F0A3FC28601CE7002840F07585E4
:100A30000722032110F07AFC22460221204610F002
:100A400095FC28600EE7002840F06A850722032104
:100A500010F06CFC01220221204610F087FC286077
:100A600000E7002840F05F850822032110F05EFCBB
:100A700022460221204610F079FC2860F2E6002888
:100A800040F054850822032110F050FC012202217D
:100A9000204610F06BFC2860E4E6002840F0498511
:100AA0000922032110F042FC22460221204610F0C8
:100AB0005DFC2860D6E6002840F03E850246122103
:100AC00010F054FC00B22860CCE6002840F03785D6
:100AD0000122122110F04AFC00B22860C2E6002870
:100AE00040F030850246132110F040FC00B228602F
:100AF000B8E6002840F029850246152110F036FCA2
:100B000000B22860AEE6002840F0228501221521BF
:100B100010F02CFC00B22860A4E6002840F01B85F1
:100B20000246162110F022FC00B228609AE6002846
:100B300040F014850122162110F018FC00B2286044
:100B400090E6002840F00D850A22032110F0EEFB0C
:100B500022460221204610F009FC00B2286081E6FE
:100B6000002840F001850A22032110F0DFFB01225A
:100B70000221204610F0FAFB00B2286072E600283D
:100B800040F0F5840B22032110F0D0FB2246022115
:100B9000204610F0EBFB00B2286063E6002840F02E
:100BA000E9840246062110F0E1FB28605AE600289D
:100BB00040F0E3840122062110F0D8FB286051E6C2
:100BC000002840F0DD84412110F08EFB286049E6CA
:100BD000002840F0D884422110F086FB286041E6CE
:100BE000002840F0D3840122462110F0BFFB00B260
:100BF000286037E6002840F0CC840246462110F0F9
:100C0000B5FB00B228602DE6002840F0C5844721DE
:100C100010F06AFB286025E6002840F0C0842121FE
:100C200010F062FB28601DE6002840F0BB84222102
:100C300010F05AFB286015E6002840F0B684024602
:100C4000232110F093FB00B228600BE6002840F04F
:100C5000AF84272110F048FB20F07F40286001E698
:100C6000002840F0A884282110F03EFB20F07F40AF
:100C70002860F7E5002840F0A18401222A2110F025
:100C800075FB00B22860EDE5002840F09A8402462A
:100C90002A2110F06BFB00B22860E3E5002840F049
:100CA00093840246392110F061FB00B22860D9E537
:100CB000002840F08C840122392110F057FB00B24B
:100CC0002860CFE5002840F0858402463D2110F0E1
:100CD0004DFB00B22860C5E5002840F07E84024646
:100CE0003F2110F043FB00B22860BBE5002840F034
:100CF000778402463A2110F039FB00B22860B1E552
:100D0000002840F070840246532110F02FFB00B2FF
:100D10002860A7E530B90122642110F027FB00B25A
:100D200028609FE5138864210122002010F02BFB2E
:100D3000002497E530B90246642110F017FB00B299
:100D400028608FE5138800226421104610F01BFBF9
:100D5000002487E5002840F04984662110F0C4FA99
:100D600028607FE520B9682110F0BEFA286079E597
:100D70001168002010F0DAFB002473E5002840F031
:100D800038840122692110F0F1FA00B2286069E587
:100D9000002840F03184C24B598910F059FB28607B
:100DA00060E5002840F02B840246692110F0DEFA4D
:100DB00000B2286056E5002840F0248410F0B1FB12
:100DC00028604FE518B910F0D6FB28604AE5116895
:100DD000002010F0CCFB002444E5002840F01584EE
:100DE00002466D2110F0A2FA6C21204610F07CFA28
:100DF000286037E5002840F00B8401226D2110F0B7
:100E000095FA6C21204610F06FFA28602AE5002838
:100E100040F0018402226D2110F088FA6C212046F6
:100E200010F062FA28601DE5002840F0F7830322E5
:100E30006D2110F07BFA6C21204610F055FA2860E5
:100E400010E5002840F0ED8304226D2110F06EFAC9
:100E50006C21204610F048FA286003E5002840F095
:100E6000E38305226D2110F061FA6C21204610F019
:100E70003BFA2860F6E4002840F0D98306226D2171
:100E800010F054FA6C21204610F02EFA2860E9E4A4
:100E9000002840F0CF8307226D2110F047FA6C2123
:100EA000204610F021FA2860DCE418B910F0A0FA0E
:100EB0002860D7E41168002010F08CFA0024D1E4F7
:100EC000774B598918B910F0B9FA2860CAE412684A
:100ED000002010F0A1FA0024C4E4002840F0AD8303
:100EE00001226F2110F022FA6E21204610F0FCF949
:100EF0002860B7E418B910F008FB2860B2E4116864
:100F0000002010F0F5FA0024ACE4002840F09883AB
:100F100003226F2110F00AFA6E21204610F0E4F946
:100F200028609FE4002840F08E8304226F2110F097
:100F3000FDF96E21204610F0D7F9286092E40028D0
:100F400040F0848305226F2110F0F0F96E212046D5
:100F500010F0CAF9286085E4002840F07A83062260
:100F60006F2110F0E3F96E21204610F0BDF92860E2
:100F700078E4002840F0708307226F2110F0D6F942
:100F80006E21204610F0B0F928606BE4002840F094
:100F9000668308226F2110F0C9F922466E2120468F
:100FA00010F0E4F900B228605CE4002840F05A83B5
:100FB00008226F2110F0BAF901226E21204610F0AC
:100FC000D5F900B228604DE4002840F04E83092294
:100FD0006F2110F0ABF922466E21204610F0C6F9C1
:100FE00000B228603EE4002840F042830A226F21CC
:100FF00010F09CF922466E21204610F0B7F900B29D
:1010000028602FE4002840F036830A226F2110F078
:101010008DF901226E21204610F0A8F900B2286057
:1010200020E4002840F02A830B226F2110F07EF983
:1010300022466E21204610F099F900B2286011E492
:10104000002840F01E830B226F2110F06FF901225F
:101050006E21204610F08AF900B2286002E40028D0
:1010600040F012830C226F2110F060F922466E21AD
:10107000204610F07BF900B22860FFF7F3BB002890
:1010800040F005830C226F2110F050F901226E21EF
:10109000204610F06BF900B22860FFF7E3BB00BFF9
:1010A000484DFF1F002840F0F5820D226F2110F0FF
:1010B0003DF922466E21204610F058F900B2286012
:1010C000FFF7D0BB002840F0E8820D226F2110F01E
:1010D0002DF901226E21204610F048F900B2286057
:1010E000FFF7C0BB002840F0DB820E226F2110F01A
:1010F0001DF922466E21204610F038F900B2286012
:10110000FFF7B0BB002840F0CE820E226F2110F016
:101110000DF901226E21204610F028F900B2286056
:10112000FFF7A0BB002840F0C1820F226F2110F012
:10113000FDF822466E21204610F018F900B2286012
:10114000FFF790BB002840F0B4820F226F2110F00F
:10115000EDF801226E21204610F008F900B2286057
:10116000FFF780BB002840F0A78210226F2110F00B
:10117000DDF822466E21204610F0F8F800B2286013
:10118000FFF770BB002840F09A8211226F2110F007
:10119000CDF822466E21204610F0E8F800B2286013
:1011A000FFF760BB002840F08D8211226F2110F004
:1011B000BDF801226E21204610F0D8F800B2286058
:1011C000FFF750BB002840F0808212226F2110F000
:1011D000ADF822466E21204610F0C8F800B2286013
:1011E000FFF740BB002840F0738213226F2110F0FC
:1011F0009DF822466E21204610F0B8F82860FFF7CF
:1012000031BB002840F0678213226F2110F08EF866
:1012100001226E21204610F0A9F82860FFF722BBBA
:10122000002840F05B82C0226F2110F07FF8224638
:101230006E21204610F09AF800B22860FFF712BB2A
:10124000002840F04E82C0226F2110F06FF801227A
:101250006E21204610F08AF800B22860FFF702BB2A
:10126000002840F04182C1226F2110F05FF8224631
:101270006E21204610F07AF800B22860FFF7F2BA2B
:10128000002840F03482C1226F2110F04FF8012273
:101290006E21204610F06AF800B22860FFF7E2BA2B
:1012A000002840F02782C2226F2110F03FF822462A
:1012B0006E21204610F05AF800B22860FFF7D2BA2B
:1012C000002840F01A82C2226F2110F02FF801226C
:1012D0006E21204610F04AF800B22860FFF7C2BA2B
:1012E000002840F00D82C3226F2110F01FF8224623
:1012F0006E21204610F03AF800B22860FFF7B2BA2B
:10130000002840F00082C3226F2110F00FF8012264
:101310006E21204610F02AF800B22860FFF7A2BA2A
:10132000002840F0F381C4226F210FF0FFFF224616
:101330006E21204610F01AF82860FFF793BA0028B3
:1013400040F0E781C4226F210FF0F0FF01226E21EF
:10135000204610F00BF82860FFF784BA002840F010
:10136000DB81C5226F210FF0E1FF22466E2120466E
:101370000FF0FCFF2860FFF775BA002840F0CF811E
:10138000C5226F210FF0D2FF01226E2120460FF0FF
:10139000EDFF2860FFF766BA002840F0C381C6223F
:1013A0006F210FF0C3FF22466E2120460FF0DEFFB3
:1013B0002860FFF757BA002840F0B781C6226F2196
:1013C0000FF0B4FF01226E2120460FF0CFFF2860FE
:1013D000FFF748BA002840F0AB81C7226F210FF019
:1013E000A5FF22466E2120460FF0C0FF2860FFF7C0
:1013F00039BA002840F09F81C7226F210FF096FF75
:1014000001226E2120460FF0B1FF2860FFF72ABAB3
:10141000002840F09381C8226F210FF087FF6E21D2
:1014200020460FF061FF2860FFF71CBA002840F04B
:101430008881C9226F210FF079FF6E2120460FF0BD
:1014400053FF2860FFF70EBA002840F07D81CA22C2
:101450006F210FF06BFF6E2120460FF045FF2860D3
:10146000FFF700BA002840F07281CB226F210FF005
:101470005DFF6E2120460FF037FF2860FFF7F2B9BD
:10148000B74B18B95B891360FFF7ECB912685A8142
:101490000024FFF7E7B920B9B14B5B7A1360FFF77F
:1014A000E1B9B04A2878511C10F058F90024FFF730
:1014B000D9B9002840F04E81A94B1B7A1360FFF781
:1014C000D1B9002840F04981A54BDB881360FFF7B4
:1014D000C9B90424FFF7C6B90424FFF7C3B904242B
:1014E000FFF7C0B90424FFF7BDB90424FFF7BAB968
:1014F0000424FFF7B7B90424FFF7B4B90424FFF7B5
:10150000B1B90424FFF7AEB90424FFF7ABB9042442
:10151000FFF7A8B90424FFF7A5B90424FFF7A2B97F
:101520000424FFF79FB90424FFF79CB90424FFF7B4
:1015300099B90424FFF796B90424FFF793B904245A
:10154000FFF790B90424FFF78DB90424FFF78AB997
:101550000424FFF787B90424FFF784B90424FFF7B4
:1015600081B90424FFF77EB90424FFF77BB9042472
:10157000FFF778B90424FFF775B90424FFF772B9AF
:101580000424FFF76FB90424FFF76CB90424FFF7B4
:1015900069B90424FFF766B90424FFF763B904248A
:1015A000FFF760B90424FFF75DB90424FFF75AB9C7
:1015B0000424FFF757B90424FFF754B90424FFF7B4
:1015C00051B90424FFF74EB90424FFF74BB90424A2
:1015D000FFF748B90424FFF745B90424FFF742B9DF
:1015E0000424FFF73FB90424FFF73CB90424FFF7B4
:1015F00039B90424FFF736B90424FFF733B90424BA
:10160000FFF730B90424FFF72DB90424FFF72AB9F6
:101610000424FFF727B90424FFF724B90424FFF7B3
:1016200021B90424FFF71EB90424FFF71BB90424D1
:10163000FFF718B90424FFF715B90424FFF712B90E
:101640000424FFF70FB90424FFF70CB90424FFF7B3
:1016500009B90424FFF706B90424FFF703B90424E9
:10166000FFF700B90424FFF7FDB80424FFF7FAB828
:101670000424FFF7F7B80424FFF7F4B80424FFF7B5
:10168000F1B80424FFF7EEB80424FFF7EBB8042404
:10169000FFF7E8B80424FFF7E5B80424FFF7E2B841
:1016A0000424FFF7DFB80424FFF7DCB80424FFF7B5
:1016B000D9B80424FFF7D6B80424FFF7D3B804241C
:1016C000FFF7D0B80424FFF7CDB80424FFF7CAB859
:1016D0000424FFF7C7B80424FFF7C4B80424FFF7B5
:1016E000C1B80424FFF7BEB80424FFF7BBB8042434
:1016F000FFF7B8B80424FFF7B5B80424FFF7B2B871
:101700000424FFF7AFB80424FFF7ACB80424FFF7B4
:10171000A9B80424FFF7A6B80424FFF7A3B804244B
:10172000FFF7A0B80424FFF79DB80424FFF79AB888
:101730000424FFF797B80424FFF794B80424FFF7B4
:1017400091B80424FFF78EB80424FFF78BB8042463
:10175000FFF788B80424FFF785B80424FFF782B8A0
:10176000484DFF1F504DFF1F0B4619B90146184643
:10177000FEF76FBF082070470120704707B5019240
:1017800039B9014601AA0120FEF763FF03B05DF8F5
:1017900004FB0820FAE710B40C4630B9044B1B6870
:1017A00020469B6810BC11461847002010BC7047AB
:1017B0005C4DFF1F70B52B4D2B4EEC6860682368A5
:1017C00064303060DB689847236830685B6998470D
:1017D000264B2A691A606368254903F53173536003
:1017E000244B5A690A602449C2F804122349C2F8FA
:1017F0000812002111705170214A1A62214ADA61DF
:10180000214A9A61214A5A62214ADA64214A9A633A
:10181000214A5A63214A9A62214ADA62214A9A6429
:10182000214A5A64214A5A65214A1A65214A1A6690
:10183000214ADA65214A9A65322440F28A2201203F
:10184000C3E9022418741E4B4FF47A729A8041F255
:1018500070721A604FF4807259725A81BDE87040FC
:10186000FEF7AFBE847E0200584DFF1F5C4DFF1F88
:10187000604DFF1F6434FF1F490501007917010007
:10188000A7050100C1050100BD050100B905010062
:101890003D060100691701007D1701009505010053
:1018A000290601008F05010081050100590501008D
:1018B00045050100C30501004D05010005060100B5
:1018C000484DFF1F0020704701207047014B002248
:1018D0005A6070476434FF1F00200FF06FBF10B5CF
:1018E000002014460FF048FF206010BD022804BFFE
:1018F0000B4B93F8D80030B90A4BDB681B689B6927
:10190000094A10681847012809D1054B93F8D830C7
:10191000012B04D1034BDB681B685B69F0E7704760
:101920006434FF1F847E0200584DFF1F10B5002055
:10193000FFF7DCFF044B054ADB6810681B68BDE855
:1019400010409B69184700BF847E0200584DFF1F5E
:101950007FB5244B244C5A78064633F8060C029087
:10196000981E019033F8041C00910020314610F0BD
:101970003FF92368B34226D104B070BD022B12D1C7
:101980001A4D28460DF014FF6B2100200FF0F4FED5
:1019900068210246A86000200FF010FF0020E861D7
:1019A0002A6966211AE0012B1AD16B2100200FF061
:1019B000E3FE0E4D0246A860682100200FF0FEFEF7
:1019C0000023EB610CE00A4B1B78032BD6D1074DAB
:1019D00028460DF01FFFAA68682100200FF0EEFED8
:1019E0002660C9E74E4DFF1F4C17FF1F644DFF1FB8
:1019F000904DFF1F38B50D46044620B90FF0E6FFA5
:101A00002860204638BD0820FCE770B50E46A8B90E
:101A10000B4C0C4D2278012A02D10FF0D7FF286120
:101A20000321002021700FF00DFF6B2100200FF02B
:101A3000A3FE336818446860002070BD0820FCE7EE
:101A4000904DFF1F644DFF1F70B50E4678B9094CCD
:101A5000094D2278012A02D10FF0B8FF2861032135
:101A6000002021700FF0EEFE6E60002070BD082097
:101A7000FCE700BF904DFF1F644DFF1F70B50E4681
:101A800078B9094C094D2278012A02D10FF09EFF46
:101A900028610221002021700FF0D4FEEE600020AA
:101AA00070BD0820FCE700BF904DFF1F644DFF1F75
:101AB0000021E3E74942E1E7E0E7043970B5044675
:101AC0001546FA2900F2FD87DFE811F0FB00FB075D
:101AD000FB07FB07FB07FB07FB070D011E012901A5
:101AE000FB07FB07FB07FB07FB07FB07FB07FB07E6
:101AF000FB07FB07FB07FB07FB07FB07FB07FB07D6
:101B0000FB07FB07FB07FB07FB07FB07FB07FB07C5
:101B1000FB07FB07FB07FB07FB07FB07FB07FB07B5
:101B2000FB07FB07FB07FB0730013F01FB074E01EB
:101B30005E01FB07FB07FB07FB07FB07FB07FB0738
:101B4000FB07FB07FB07FB07FB07FB07FB07FB0785
:101B5000FB07FB07FB07FB07FB07FB07FB07FB0775
:101B6000FB07FB07FB07FB07FB07FB07FB07FB0765
:101B7000FB07FB07FB07FB07FB07FB07FB07FB0755
:101B8000FB07FB07FB07FB07FB07FB076E017C015D
:101B90008A01FB07FB07FB07FB07FB07FB07FB07AC
:101BA000FB079801A601B401FB07FB07C201CC01AA
:101BB000D601FB07E001EA01F401FB07FE010C027C
:101BC000FB071A022302FB07FB07FB072C02340268
:101BD0003C0246025002FB07FB07FB07580260026B
:101BE0006A02FB07FB07FB07FB07FB07FB07FB077B
:101BF00074027E02880292029C02B102C602DE02D8
:101C0000F6020E0325032F03390343034D03FB079D
:101C1000FB07FB07FB07FB07570361037103810306
:101C2000890391039B03A403AE03B503D003DD0333
:101C3000EA03F703040411041E042B04FB07380411
:101C40004304530460046D047A0487049404A104DB
:101C5000AE04BD04CC04DB04EA04F9040905200544
:101C60003005400550056005700580059005A0050C
:101C7000B005C005D005E005EF05FB07FE0515061C
:101C80002C06460660067A069406FB07FB07FB0750
:101C9000A206B206C206D206E206F2060207120742
:101CA0002207310740074F075E076D077C078B0748
:101CB0009A07A807B607C407FB07D207DD07EB079B
:101CC000F307B64E30B960210FF056FD2860306042
:101CD000204670BD1268602100200FF06FFD2B6858
:101CE00033600024F4E7AD4E28B95F210FF044FDC6
:101CF00028607061ECE712685F2100200FF05EFD44
:101D00002B6873610024E3E7A44B18B993F82030E3
:101D10001360DDE7126883F820200024D8E700284C
:101D200040F0D2869D4B1B691360D1E728B902466B
:101D300008210FF063FD2860CAE7138800220821FC
:101D400010460FF068FD0024C2E728B902460921B9
:101D50000FF054FD2860BBE71388002209211046CC
:101D60000FF059FD0024B3E730B9012208210FF02C
:101D700045FD00B22860ABE713880821012200204E
:101D80000FF049FD0024A3E730B9012209210FF02B
:101D900035FD00B228609BE713880921012200204D
:101DA0000FF039FD002493E7002840F090860122CF
:101DB00003210FF003FD2246022120460FF01EFDF5
:101DC000286085E7002840F08586012203210FF076
:101DD000F5FC0122022120460FF010FD286077E774
:101DE000002840F07A86022203210FF0E7FC224609
:101DF000022120460FF002FD286069E7002840F02C
:101E00006F86022203210FF0D9FC01220221204615
:101E10000FF0F4FC28605BE7002840F064860322A2
:101E200011460FF0CBFC0122022120460FF0E6FC08
:101E300028604DE7002840F05986032211460FF034
:101E4000BDFC2246022120460FF0D8FC28603FE767
:101E5000002840F04E86024612210FF0CFFC00B25F
:101E6000286035E7002840F04786012212210FF054
:101E7000C5FC00B228602BE7002840F040860246EF
:101E800013210FF0BBFC00B2286021E7002840F0CE
:101E90003986024615210FF0B1FC00B2286017E721
:101EA000002840F03286012215210FF0A7FC00B275
:101EB00028600DE7002840F02B86024616210FF01F
:101EC0009DFC00B2286003E7002840F0248602460B
:101ED00003210FF073FC2246022120460FF08EFCF6
:101EE0002860F5E6002840F01986024603210FF02D
:101EF00065FC0122022120460FF080FC2860E7E605
:101F0000002840F00E8602460B210FF077FC286077
:101F1000DEE6002840F0088601220B210FF06EFC5F
:101F20002860D5E6002840F0028641210FF024FC0D
:101F30002860CDE6002840F0FD8542210FF01CFC12
:101F40002860C5E6002840F0F885012246210FF000
:101F500055FC00B22860BBE6002840F0F18502463F
:101F600046210FF04BFC00B22860B1E6002840F09B
:101F7000EA8547210FF000FC2860A9E6002840F020
:101F8000E58521210FF0F8FB2860A1E6002840F04C
:101F9000E08522210FF0F0FB286099E6644DFF1FD9
:101FA000002840F0D985024623210FF027FC00B21B
:101FB00028608DE6002840F0D28527210FF0DCFB59
:101FC00020F07F40286083E6002840F0CB85282160
:101FD0000FF0D2FB20F07F40286079E6002840F027
:101FE000C48501222A210FF009FC00B228606FE6A7
:101FF000002840F0BD8502462A210FF0FFFB00B209
:10200000286065E6D4226F2138B90FF0D7FB6E2126
:1020100020460FF0B1FB28605AE600200FF0CEFBFF
:102020002A686E2100200FF0C9FB002450E6D5225B
:102030006F2138B90FF0C2FB6E2120460FF09CFBD8
:10204000286045E600200FF0B9FB2A686E210020C9
:102050000FF0B4FB00243BE6D6226F2148B90FF005
:10206000ADFB22466E2120460FF0C8FB00B228606F
:102070002EE600200FF0A2FB00222B886E211046D6
:102080000FF0C9FB002423E6D6226F2148B90FF0D8
:1020900095FB01226E2120460FF0B0FB00B22860B4
:1020A00016E600200FF08AFB2B8801226E2100200B
:1020B0000FF0B1FB00240BE6D7226F2148B90FF0D7
:1020C0007DFB22466E2120460FF098FB00B228606F
:1020D000FEE500200FF072FB00222B886E211046D7
:1020E0000FF099FB0024F3E5D7226F2140B90FF0E0
:1020F00065FB01226E2120460FF080FB2860E7E59A
:1021000000200FF05BFB2B8801226E2100200FF0D6
:1021100082FB0024DCE5002840F02D8502463921B1
:102120000FF06CFB00B22860D2E5002840F0268555
:10213000012239210FF062FB00B22860C8E50028B7
:1021400040F01F8502463D210FF058FB00B2286089
:10215000BEE5002840F0188502463F210FF04EFBF7
:1021600000B22860B4E5002840F0118502463A210B
:102170000FF044FB00B22860AAE5002840F00A8571
:10218000024653210FF03AFB00B22860A0E530B9B7
:10219000012264210FF032FB00B2286098E5138819
:1021A0006421012200200FF036FB002490E530B9B5
:1021B000024664210FF022FB00B2286088E51388F4
:1021C0000022642110460FF026FB002480E5002841
:1021D00040F0E38466210FF0CFFA286078E500280C
:1021E00040F0DE8468210FF0C7FA286070E500280F
:1021F00040F0D984012269210FF000FB00B2286071
:1022000066E5002840F0D284BD4B19890FF073FBBE
:1022100028605DE5002840F0CC84024669210FF07B
:10222000EDFA00B2286053E5002840F0C5840FF0B5
:10223000CDFB28604CE518B90FF0F2FB286047E5AC
:1022400012686B2100200FF0B9FAAE4B1B78032BFC
:1022500040F0B584AC4B2A685A602A689A602A68B4
:10226000682100200FF0AAFA002431E5002840F090
:10227000A98402466D210FF0A1FA6C2120460FF0CF
:102280007BFA286024E5002840F09F8401226D211C
:102290000FF094FA6C2120460FF06EFA286017E5D3
:1022A000002840F0958402226D210FF087FA6C21FE
:1022B00020460FF061FA28600AE5002840F08B8480
:1022C00003226D210FF07AFA6C2120460FF054FAA8
:1022D0002860FDE4002840F0818404226D210FF085
:1022E0006DFA6C2120460FF047FA2860F0E40028D0
:1022F00040F0778405226D210FF060FA6C212046B2
:102300000FF03AFA2860E3E4002840F06D840622DA
:102310006D210FF053FA6C2120460FF02DFA286042
:10232000D6E4002840F0638407226D210FF046FABE
:102330006C2120460FF020FA2860C9E418B90FF08C
:102340009FFA2860C4E4116800200FF08BFA002483
:10235000BEE46B4B198918B90FF0C3FA2860B7E4D3
:10236000126800200FF0ABFA664B01221A700024AD
:10237000AEE4002840F03E8401226F210FF01EFAE7
:102380006E2120460FF0F8F92860A1E4002840F003
:10239000348402226F210FF011FA6E2120460FF0D3
:1023A000EBF9286094E4002840F02A8403226F218E
:1023B0000FF004FA6E2120460FF0DEF9286087E462
:1023C000002840F0208404226F210FF0F7F96E21DD
:1023D00020460FF0D1F928607AE4002840F01684F6
:1023E00005226F210FF0EAF96E2120460FF0C4F9A3
:1023F00028606DE4002840F00C8406226F210FF065
:10240000DDF96E2120460FF0B7F9286060E400285E
:1024100040F0028407226F210FF0D0F96E21204690
:102420000FF0AAF9286053E4002840F0F88308224E
:102430006F210FF0C3F922466E2120460FF0DEF91E
:1024400000B2286044E4002840F0EC8308226F21A9
:102450000FF0B4F901226E2120460FF0CFF900B23F
:10246000286035E4002840F0E08309226F210FF056
:10247000A5F922466E2120460FF0C0F900B228606F
:1024800026E4002840F0D4830A226F210FF096F949
:1024900022466E2120460FF0B1F900B2286017E401
:1024A000002840F0C8830A226F210FF087F901222B
:1024B0006E2120460FF0A2F900B2286008E400283F
:1024C00040F0BC830B226F210FF078F922466E2179
:1024D00020460FF093F900B22860FFF7F9BB0028FF
:1024E00040F0AF830B226F210FF068F901226E21BB
:1024F00020460FF083F900B22860FFF7E9BB00BF68
:10250000484DFF1F904DFF1F644DFF1F002840F0F6
:102510009B830C226F210FF051F922466E21204639
:102520000FF06CF900B22860FFF7D2BB002840F032
:102530008E830C226F210FF041F901226E2120467B
:102540000FF05CF900B22860FFF7C2BB002840F032
:1025500081830D226F210FF031F922466E21204632
:102560000FF04CF900B22860FFF7B2BB002840F032
:1025700074830D226F210FF021F901226E21204674
:102580000FF03CF900B22860FFF7A2BB002840F032
:1025900067830E226F210FF011F922466E2120462B
:1025A0000FF02CF900B22860FFF792BB002840F032
:1025B0005A830E226F210FF001F901226E2120466D
:1025C0000FF01CF900B22860FFF782BB002840F032
:1025D0004D830F226F210FF0F1F822466E21204625
:1025E0000FF00CF900B22860FFF772BB002840F032
:1025F00040830F226F210FF0E1F801226E21204667
:102600000FF0FCF800B22860FFF762BB002840F032
:10261000338310226F210FF0D1F822466E2120461D
:102620000FF0ECF800B22860FFF752BB002840F032
:10263000268311226F210FF0C1F822466E21204619
:102640000FF0DCF800B22860FFF742BB002840F032
:10265000198311226F210FF0B1F801226E2120465B
:102660000FF0CCF800B22860FFF732BB002840F032
:102670000C8312226F210FF0A1F822466E21204612
:102680000FF0BCF800B22860FFF722BB002840F032
:10269000FF8213226F210FF091F822466E2120460F
:1026A0000FF0ACF82860FFF713BB002840F0F3826E
:1026B00013226F210FF082F801226E2120460FF0C5
:1026C0009DF82860FFF704BBD0226F2140B90FF0BE
:1026D00075F86E2120460FF04FF82860FFF7F8BA22
:1026E00000200FF06BF82A686E2100200FF066F8CA
:1026F0000024FFF7EDBAD1226F2140B90FF05EF848
:102700006E2120460FF038F82860FFF7E1BA00206C
:102710000FF054F82A686E2100200FF04FF80024C3
:10272000FFF7D6BAD2226F2150B90FF047F82246F0
:102730006E2120460FF062F800B22860FFF7C8BA99
:1027400000200FF03BF800222B886E2110460FF07E
:1027500062F80024FFF7BCBAD2226F2150B90FF003
:102760002DF801226E2120460FF048F800B22860B3
:10277000FFF7AEBA00200FF021F82B8801226E215E
:1027800000200FF048F80024FFF7A2BAD3226F21EF
:1027900050B90FF013F822466E2120460FF02EF8A4
:1027A00000B22860FFF794BA00200FF007F800226B
:1027B0002B886E2110460FF02EF80024FFF788BA00
:1027C000D3226F2150B90EF0F9FF01226E2120466D
:1027D0000FF014F800B22860FFF77ABA00200EF06C
:1027E000EDFF2B8801226E2100200FF014F8002449
:1027F000FFF76EBA002840F051821D226F210EF0C3
:10280000DDFF6E2120460EF0B7FF2860FFF760BAAB
:10281000002840F04682C0226F210EF0CFFF2246F2
:102820006E2120460EF0EAFF00B22860FFF750BA92
:10283000002840F03982C0226F210EF0BFFF012234
:102840006E2120460EF0DAFF00B22860FFF740BA92
:10285000002840F02C82C1226F210EF0AFFF2246EB
:102860006E2120460EF0CAFF00B22860FFF730BA92
:10287000002840F01F82C1226F210EF09FFF01222D
:102880006E2120460EF0BAFF00B22860FFF720BA92
:10289000002840F01282C2226F210EF08FFF2246E4
:1028A0006E2120460EF0AAFF00B22860FFF710BA92
:1028B000002840F00582C2226F210EF07FFF012226
:1028C0006E2120460EF09AFF00B22860FFF700BA92
:1028D000002840F0F881C3226F210EF06FFF2246DE
:1028E0006E2120460EF08AFF00B22860FFF7F0B993
:1028F000002840F0EB81C3226F210EF05FFF012220
:102900006E2120460EF07AFF00B22860FFF7E0B992
:10291000002840F0DE81C4226F210EF04FFF2246D6
:102920006E2120460EF06AFF2860FFF7D1B900281B
:1029300040F0D281C4226F210EF040FF01226E21AF
:1029400020460EF05BFF2860FFF7C2B9002840F078
:10295000C681C5226F210EF031FF22466E2120462E
:102960000EF04CFF2860FFF7B3B9002840F0BA81A1
:10297000C5226F210EF022FF01226E2120460EF0AB
:102980003DFF2860FFF7A4B9002840F0AE81C622C1
:102990006F210EF013FF22466E2120460EF02EFF0F
:1029A0002860FFF795B9002840F0A281C6226F2168
:1029B0000EF004FF01226E2120460EF01FFF28605A
:1029C000FFF786B9002840F09681C7226F210EF0EC
:1029D000F5FE22466E2120460EF010FF2860FFF71C
:1029E00077B9002840F08A81C7226F210EF0E6FEF9
:1029F00001226E2120460EF001FF2860FFF768B922
:102A0000002840F07E81C8226F210EF0D7FE6E2193
:102A100020460EF0B1FE2860FFF75AB9002840F0BA
:102A20007381C9226F210EF0C9FE6E2120460EF07F
:102A3000A3FE2860FFF74CB9002840F06881CA2245
:102A40006F210EF0BBFE6E2120460EF095FE286031
:102A5000FFF73EB9002840F05D81CB226F210EF0D8
:102A6000ADFE6E2120460EF087FE2860FFF730B9DC
:102A7000AD4B18B91B891360FFF72AB912681A8188
:102A80000024FFF725B920B9A74BDB791360FFF7C6
:102A90001FB9A64A2878511C0FF0B4F80024FFF79C
:102AA00017B9002840F039819F4B9B791360FFF7DD
:102AB0000FB9002840F034819B4B9B881360FFF7CF
:102AC00007B90424FFF704B90024FFF701B904246F
:102AD000FFF7FEB80424FFF7FBB80424FFF7F8B8AB
:102AE0000424FFF7F5B80424FFF7F2B80424FFF735
:102AF000EFB80424FFF7ECB80424FFF7E9B8042486
:102B0000FFF7E6B80424FFF7E3B80424FFF7E0B8C2
:102B10000424FFF7DDB80424FFF7DAB80424FFF734
:102B2000D7B80424FFF7D4B80424FFF7D1B804249D
:102B3000FFF7CEB80424FFF7CBB80424FFF7C8B8DA
:102B40000424FFF7C5B80424FFF7C2B80424FFF734
:102B5000BFB80424FFF7BCB80424FFF7B9B80424B5
:102B6000FFF7B6B80424FFF7B3B80424FFF7B0B8F2
:102B70000424FFF7ADB80424FFF7AAB80424FFF734
:102B8000A7B80424FFF7A4B80424FFF7A1B80424CD
:102B9000FFF79EB80424FFF79BB80424FFF798B80A
:102BA0000424FFF795B80424FFF792B80424FFF734
:102BB0008FB80424FFF78CB80424FFF789B80024E9
:102BC000FFF786B80424FFF783B80424FFF780B822
:102BD0000424FFF77DB80424FFF77AB80424FFF734
:102BE00077B80424FFF774B80424FFF771B80424FD
:102BF000FFF76EB80424FFF76BB80424FFF768B83A
:102C00000424FFF765B80424FFF762B80424FFF733
:102C10005FB80424FFF75CB80424FFF759B8042414
:102C2000FFF756B80424FFF753B80424FFF750B851
:102C30000424FFF74DB80424FFF74AB80424FFF733
:102C400047B80424FFF744B80424FFF741B804242C
:102C5000FFF73EB80424FFF73BB80424FFF738B869
:102C60000424FFF735B80424FFF732B80424FFF733
:102C70002FB80424FFF72CB80424FFF729B8042444
:102C8000FFF726B80424FFF723B80424FFF720B881
:102C90000424FFF71DB80424FFF71AB80424FFF733
:102CA00017B80424FFF714B80424FFF711B804245C
:102CB000FFF70EB80424FFF70BB80424FFF708B899
:102CC0000424FFF705B80424FFF702B80424FEF734
:102CD000FFBF0424FEF7FCBF0424FEF7F9BF042461
:102CE000FEF7F6BF0424FEF7F3BF0424FEF7F0BF9F
:102CF0000424FEF7EDBF0424FEF7EABF0424FEF728
:102D0000E7BF0424FEF7E4BF0424FEF7E1BF042478
:102D1000FEF7DEBF0424FEF7DBBF0424FEF7D8BFB6
:102D20000424FEF7D5BF00BF484DFF1F4E4DFF1FC7
:102D30000B4619B901461846FEF7BFBE082070477A
:102D40000120704707B5019239B9014601AA012057
:102D5000FEF7B3FE03B05DF804FB0820FAE710B4F9
:102D60000C4630B9044B1B6820469B6810BC1146CA
:102D70001847002010BC70478C4DFF1F70B52E4DBA
:102D80002E4EEC686068236864303060DB689847DA
:102D9000236830685B699847294B2A691A60636821
:102DA0002849294803F531735360284B5A690A6052
:102DB0002749C2F8041201240025264914705570D1
:102DC000C2F80812244A1A62244ADA61244A9A6133
:102DD000244A5A62244ADA64244A9A63244A5A6387
:102DE000244A9A62244ADA62244A9A64244A5A6437
:102DF000244A5A65244A1A65244A1A66244ADA651E
:102E0000244A9A65322140F28A22C3E902211C74C5
:102E1000214B4FF47A725A8041F270721A804FF44B
:102E20008072DD711A810CF0B7FC1C4B1D702046BE
:102E3000BDE87040FEF75ABD847E0200584DFF1F6A
:102E40008C4DFF1F884DFF1F644DFF1F6434FF1F13
:102E5000C9180100412D01007D1A0100B91A0100B5
:102E6000B51A0100B11A0100F5190100312D010058
:102E7000452D0100491A01000B1A0100D918010063
:102E8000DF18010051190100C5180100ED180100FB
:102E9000CD1801002D190100484DFF1F904DFF1F57
:102EA000014B00225A6070476434FF1F70B5084E12
:102EB000084D336804462A46014600200EF000FF04
:102EC00033682A4621460120BDE870400EF0F8BE66
:102ED0003050FF1F944DFF1F014B18680EF051BF7B
:102EE0003050FF1F01280CD8074B1A68202303FA23
:102EF00000F040F0020002EB800043680B6000200D
:102F000070470820704700BF3050FF1F012810B5E0
:102F1000144611D003D302281AD0042009E0104B24
:102F2000104ADB6824681B68D0681CB15B6998474D
:102F3000002010BD9B69FAE7094B0A4ADB6850681C
:102F40001B681B6A9847003018BF01202060EFE71C
:102F5000034B044ADB6890681B681B6AF2E700BFFA
:102F6000847E02005C17FF1F022804BF0B4B93F8FE
:102F7000D80030B90A4BDB681B685B69094A1068E6
:102F80001847012809D1054B93F8D830012B04D1FB
:102F9000034BDB681B689B69F0E770476434FF1FD5
:102FA000847E02005C17FF1F70B50020FFF7DCFF76
:102FB000104B114CDD6820682B689B6898472B6884
:102FC00060689B6898472B68A0689B6898472B6847
:102FD000A0699B6898472B6820699B6898472B6875
:102FE00060699B6898472B68E0689B68BDE8704003
:102FF000184700BF847E02005C17FF1F2DE9F843CD
:10300000184C9DF820609DF82450984623680F4680
:103010009B68002147F08000914698472368002173
:103020009B6848469847236800219B68404698471C
:10303000236800219B6830469847236828469B6890
:1030400001219847084B1B6848EA092807F07F07C9
:1030500046EA082603EB870745EA06257D60BDE8BA
:10306000F88300BF2C50FF1F3050FF1F07B5D3B2AD
:103070000193C2F307230093C2F30743120EFFF735
:10308000BDFF03B05DF804FB0020FFF7EFBF012890
:103090002DE9F34105460F4627D8DFF85880202652
:1030A00018F80030864074B25BB1114B03EB80031B
:1030B00044F00701DA69C9B2FFF7D8FF002308F826
:1030C000053044F00D013A460024C9B22846FFF706
:1030D000CDFF2846CDE9004423462246F1B2FFF752
:1030E0008DFF204602B0BDE8F0810820FAE700BF5E
:1030F0005C17FF1F7400FF1F012873B505460E46BD
:103100001CD82024844044F0070186EAE672A2EB32
:10311000E672C9B2FFF7AAFF094A0123002E5355F0
:10312000E1B2B8BF02230024CDE90043284623467C
:103130002246FFF763FF204602B070BD0820FBE780
:103140007400FF1F0021D7E74942D5E7D4E738B51F
:10315000234B01F07F04234493F81432DB0705D49A
:10316000204B1B6803EB8404606838BD1E4D2B6840
:1031700000219B68204698472B6800219B680846E1
:1031800098472B6800219B68084698472B680021C8
:103190009B68084698472B6801219B680020984748
:1031A0002B6800219B68204698472B6800219B686C
:1031B000084698472B68002104029B6808469847F8
:1031C0002B68002104439B68084698472B6824021B
:1031D00004439B6801210020984724022043C4E750
:1031E000944DFF1F3050FF1F2C50FF1F10B50020C3
:1031F0001446FFF7ACFF206010BD38B50D46202106
:10320000814041F00101C9B20446FFF7A0FF2968DF
:10321000014429602046BDE8384038E71C2A2DE9E2
:10322000F84304460D461E4600F0168300F2A780C0
:103230000C2A00F046824BD8052A00F0E58119D807
:10324000022A00F09A8107D8002A00F07281012A30
:1032500000F08281042476E1032A00F0A781042A89
:10326000F8D1CB4B8A001344002840F0B281DB69CF
:10327000336068E1082A00F0038214D8062A00F0BF
:10328000D481072AE6D120278F4047F01007FFB2EC
:1032900039462846002C40F0E581FFF758FF00F042
:1032A0001F0030604FE10A2A00F0F9810B2AD1D1CA
:1032B000002840F0D9852021A94041F01501C9B26C
:1032C0002846FFF744FFC04300F0010030603AE1B8
:1032D000122A00F0608227D80F2A00F0348211D819
:1032E0000D2A00F00C820E2AB4D12021A94041F011
:1032F0001401C9B2002840F020822846FFF727FFBA
:10330000306020E1102A00F02F82112AA2D1202162
:10331000A94041F00801C9B2002840F03682284691
:10332000FFF715FF30600EE1152A00F05C8211D81E
:10333000132A00F04182142A8CD12021A94041F0A7
:103340000B01C9B2002840F048822846FFF7FFFE73
:103350003060F8E0172A00F06882C0F05582182A21
:103360007FF478AF2021A94041F01301C9B20028B1
:1033700040F06C822846FFF7EAFE3060E3E0AC2ABA
:1033800000F0278463D8A52A00F02E8331D8A22A22
:1033900000F0E38218D81D2A00F07D828C2A7FF489
:1033A00059AF002840F08582090141F06C0101F01D
:1033B000FC012846FFF7CBFE4FF48073C0F3036097
:1033C00043FA00F03060BEE0A32A00F0E282A42AB3
:1033D0007FF440AF0F0147F06C07FFB23946284633
:1033E000002C40F0F282FFF7B2FEC0F300303060F4
:1033F000A9E0A82A00F08A8314D8A62A00F03A830C
:10340000A72A7FF427AF0F0147F06C07FFB23946B8
:103410002846002C40F06C83FFF799FE00F00F0067
:10342000306090E0AA2A4FEA011700F0A58340F22D
:10343000888347F06D07FFB239462846002C40F0DC
:10344000B983FFF784FEC0F3411030607BE0B62AF9
:1034500000F04B843ED8B32A00F001841BD8AD2A7B
:1034600000F0D283AE2A7FF4F5AE0F0147F06D076E
:10347000FFB239462846002C40F0E283FFF767FE92
:10348000001400F07F0310F0400018BF6FF07F00C1
:103490001843306057E0B42A00F0FD83B52A7FF46A
:1034A000D9AE20278F407FB247F014085FFA88F822
:1034B00041462846FFF74BFE002C40F0FC834105B7
:1034C00040F1F78347F01101C9B22846FFF73FFEEC
:1034D000306038E0CE2A00F0458414D8B82A00F0D5
:1034E0001584B92A7FF4B6AE0F0147F06C07FFB21E
:1034F00039462846002C40F02584FFF728FEC0F30B
:10350000035030601FE0D22A00F04284D32A00F03A
:103510005284D12A7FF49EAE2021A94041F01901A6
:10352000C9B2002840F02D842846FFF710FE306015
:1035300009E02021A94041F00D01C9B230B9284667
:10354000FFF705FE30602046BDE8F8831A6828467C
:10355000FFF78CFD0024F6E72021A94041F001018E
:10356000C9B220B92846FFF7F2FD3060EBE71A68D0
:103570002846FFF77BFD0024E5E72021A94041F024
:103580000701C9B230B92846FFF7E1FD3060DAE73C
:103590005C17FF1FB74B01225A553268002AB8BF8B
:1035A00052422846FFF762FD0024CCE7002840F095
:1035B00052842021A94041F00201C9B22846FFF7F8
:1035C000C6FD10F4000318BF4FF07F43184330606E
:1035D000B9E732682027002A07FA01F7B8BF52423C
:1035E000F9B22846DA61FFF7B2FD044608B10024BB
:1035F000A9E7326847F00701002AB8BF5242C9B2B2
:103600002846FFF733FD9EE72021A94041F006013F
:10361000C9B220B92846FFF79AFD306093E71A68CF
:103620002846FFF723FD00248DE720278F4047F031
:103630001007FFB2394628462CB9FFF788FDC0F3C2
:10364000042030607FE7FFF782FD33681B0203F43C
:10365000F85320F4F8521A4339462846FFF706FD7E
:10366000002470E7FFF773FD336820F01F0203F0BA
:103670001F031A4339462846FFF7F8FC002462E787
:10368000002840F0EB832021A94041F01501C9B288
:103690002846FFF75CFDC0F34020306053E7002868
:1036A00040F0DF832021A94041F01501C9B228462E
:1036B000FFF74DFD10F0020F0CBF01230023336014
:1036C00041E720278F4047F01407FFB239462846CC
:1036D0002CB9FFF73CFDC0F34000306033E7FFF743
:1036E00036FD3368002B20F0020214BF00230223B2
:1036F0001A4339462846FFF7B9FC002423E7202760
:103700008F4047F01407FFB2394628462CB9FFF71F
:103710001EFD00F00100306015E7FFF718FD32686C
:1037200020F00100002A14BF024640F00102394691
:103730002846FFF79BFC002405E71A682846FFF798
:1037400095FC0024FFE62021A94041F00401C9B204
:1037500020B92846FFF7FBFC3060F4E61A682846DB
:10376000FFF784FC0024EEE62021A94041F005018A
:10377000C9B220B92846FFF7EAFC3060E3E61A68D0
:103780002846FFF773FC0024DDE61A682846FFF799
:103790006DFC0024D7E62021A94041F00A01C9B2FE
:1037A00020B92846FFF7D3FC3060CCE61A682846DB
:1037B000FFF75CFC0024C6E62021A94041F003018C
:1037C000C9B220B92846FFF7C2FC3060BBE61A68D0
:1037D0002846FFF74BFC0024B5E61A682846FFF799
:1037E00045FC0024AFE62021A94041F00C01C9B2FC
:1037F00020B92846FFF7ABFC3060A4E61A682846DB
:10380000FFF734FC00249EE62021A94041F011017D
:10381000C9B220B92846FFF79AFC306093E61A68CF
:103820002846FFF723FC00248DE62021A94041F023
:103830001201C9B220B92846FFF789FC306082E640
:103840001A682846FFF712FC00247CE61A6828460E
:10385000FFF70CFC002476E60F0147F06C07FFB27F
:103860003946284644B9FFF772FCC0F38040306007
:1038700069E600BF7400FF1FFFF769FC33689B0413
:1038800003F4802320F480221A4339462846FFF7A8
:10389000EDFB002457E6002840F0E982C44B2020CD
:1038A0001B68884040F0020003EB800043683360EF
:1038B00049E61B68102B4AD00DDC022B43D004DCF8
:1038C000012B16D04FF0FF3314E0042B3DD0082B12
:1038D000F8D105230EE0402B3BD003DC202BF1D1A7
:1038E000032307E0802B36D0B3F5807FEAD1002395
:1038F00000E008233360336801333FF478AE2C01D5
:1039000044F06C04E4B221462846FFF720FC3368FB
:103910001B0603F0706320F070621A4321462846AC
:10392000FFF7A4FB21462846FFF711FC33681B066E
:1039300003F0706320F0706221461A432846FFF7B7
:1039400095FB0024FFE50723D4E70623D2E70423F1
:10395000D0E70223CEE70123CCE70F0147F06C0745
:10396000FFB2394628462CB9FFF7F1FBC0F3C1304E
:103970003060E8E5FFF7EBFB3368DB0303F4C033AB
:1039800020F4C0321A4339462846FFF76FFB002463
:10399000D9E50F0147F06C07FFB2394628462CB92C
:1039A000FFF7D5FBC0F380303060CCE5FFF7CFFBED
:1039B00033689B0303F4804320F480421A43394662
:1039C0002846FFF753FB0024BDE5FFF7C0FB336833
:1039D0001B0303F4805320F480521A4339462846CF
:1039E000FFF744FB0024AEE50F0147F06C07FFB280
:1039F00039462846FFF7ABFB3946814600F480483C
:103A00002846B4B9B8F1000F05D0FFF7A0FBC0F30A
:103A1000C310306097E5FFF79AFB19F4006FC0F30D
:103A2000021001D13060E2E540F008003060444609
:103A300089E5B8F1000F0ED0FFF789FB3368DB0191
:103A400003F4F06320F4F0621A4339462846FFF786
:103A50000DFB002477E5FFF77AFB33681B0103F0C9
:103A6000700320F070021A4339462846FFF7FEFA29
:103A7000444668E50F0147F06C07FFB23946284617
:103A8000FFF765FB394600F4804828467CB9B8F159
:103A9000000F05D0FFF75BFBC0F30210306052E56A
:103AA000FFF755FBC0F3C310306044464BE5B8F157
:103AB000000F0ED0FFF74BFB33681B0103F07003C0
:103AC00020F070021A4339462846FFF7CFFA002447
:103AD00039E5FFF73CFB3368DB0103F4F06320F4C6
:103AE000F0621A4339462846FFF7C0FA44462AE5F1
:103AF000FFF72DFB336820F00F0203F00F031A438A
:103B000039462846FFF7B2FA00241CE50F0147F0BA
:103B10006D07FFB2394628462CB9FFF718FBC0F3F2
:103B2000C03030600FE5FFF712FB3368DB039BB258
:103B300020F400421A4339462846FFF797FA00243A
:103B400001E547F06D07FFB2394628462CB9FFF76B
:103B5000FEFAC0F341303060F5E4FFF7F8FA33685D
:103B60005B0303F4C04320F4C0421A43394628469D
:103B7000FFF77CFA0024E6E447F06D07FFB2394610
:103B800028462CB9FFF7E3FAC0F303203060DAE4EB
:103B9000FFF7DDFA33681B0203F4706320F47062F0
:103BA0001A4339462846FFF761FA0024CBE400BFE8
:103BB0003050FF1FFFF7CBFA33685B0103F060035F
:103BC00020F060021A4339462846FFF74FFA0024D6
:103BD000B9E40F0147F06D07FFB2394628462CB90A
:103BE000FFF7B5FA00F00F003060ACE4FFF7AFFA72
:103BF000336820F00F0203F00F031A4339462846BA
:103C0000FFF734FA00249EE40F0147F06D07FFB27E
:103C1000394628462CB9FFF79AFAC0F300603060A5
:103C200091E4FFF794FA33681B0603F0807320F0E9
:103C300080721A4339462846FFF718FA002482E4B6
:103C4000FFF785FA33681B0403F4FE0320F4FE0239
:103C50001A4339462846FFF709FA002473E40F0196
:103C600047F06C07FFB2394628462CB9FFF76FFAC8
:103C7000C0F34040306066E4FFF769FA33685B04E4
:103C800003F4003320F400321A4339462846FFF784
:103C9000EDF9002457E4002840F0EC80090141F0E0
:103CA0006F01C9B22846FFF752FAC0F304403060F2
:103CB00049E4346047E447F011013268C9B228464C
:103CC000FFF7D4F941462846FFF741FA3368002B45
:103CD00020F480620CBF00234FF480631A434146F6
:103CE0002846FFF7C3F900242DE42021A94041F024
:103CF0001101C9B220B92846FFF729FA306022E441
:103D00001A682846FFF7B2F900241CE40F0147F0B7
:103D10006C07FFB2394628462CB9FFF718FAC0F3F2
:103D2000403030600FE4FFF712FA33685B0303F4AE
:103D3000005320F400521A4339462846FFF796F9FB
:103D4000002400E4FFF703FA33681B0503F4700353
:103D500020F470021A4339462846FFF787F90024F9
:103D6000FFF7F1BB002840F08880090141F06F01A6
:103D7000C9B22846FFF7EBF9C0F309003060FFF73E
:103D8000E2BB1A682846FFF771F90024FFF7DBBB96
:103D90002021A94041F01A01C9B228B92846FFF7ED
:103DA000D6F93060FFF7CFBB1A682846FFF75EF9F7
:103DB0000024FFF7C8BBE8B979B101297FF4C3AB90
:103DC00001462846FFF7C3F900F06000A0F1200388
:103DD000584258413060FFF7B6BB0846FFF7B7F9C5
:103DE00000F01800A0F110025042504130602C4603
:103DF000FFF7A9BB21B1012917D00024FFF7A3BB0E
:103E00000846FFF7A4F9336853B120F0080242F0E6
:103E1000100200210846FFF729F90024FFF793BBA1
:103E200020F0100242F00802F3E700212846FFF7D5
:103E30008EF9336853B120F0400242F02002002195
:103E40000120FFF713F90024FFF77DBB20F02002CB
:103E500042F04002F3E70424FFF775BB0424FFF7A8
:103E600072BB0424FFF76FBB0424FFF76CBB042470
:103E7000FFF769BB0424FFF766BB0424FFF763BBAD
:103E80000129134603D802460020FFF7C7B90820CE
:103E9000704707B50129019207D8024601AB0120FE
:103EA000FFF7BCF903B05DF804FB0820FAE708B59A
:103EB00022210020FFF74BF950B942210120FFF7E2
:103EC00046F928B9034B1868BDE808400DF052BF09
:103ED000002008BD3050FF1F70B53D4E3D483E4CA0
:103EE0000DF0B2FEF5686B6803F58272626003F54F
:103EF0009272A26003F57172E26003F5797203F1C8
:103F00006400226103F2044203F22443A3612B689C
:103F10006261DB68206098472B68E068DB6898473F
:103F20002B68E0689B6998472B6860681B69984715
:103F30002B68A0681B6998472B68A0691B69984784
:103F40002B6820691B6998472B6860691B69984733
:103F5000224B32691A606B68214903F53173536053
:103F6000204B5A690A602049C2F804121F49C2F85E
:103F7000081201200021517010701D4A1A621D4A5A
:103F8000DA611D4A9A611D4A5A621D4A9A631D4AA6
:103F90005A631D4A9A621D4ADA621D4A9A641D4A92
:103FA0005A641D4A5A651D4A1A651D4ADA641D4A3B
:103FB0001A661D4ADA6502221A743221B622C3E952
:103FC00002211A4A9A65BDE87040FEF7CDBF00BFD6
:103FD000847E0200944DFF1F5C17FF1F2C50FF1FB3
:103FE0003050FF1F6434FF1FAF3E0100D92E010087
:103FF000F93001004D310100493101004531010026
:10400000813E0100933E01008F300100FB31010031
:1040100089300100ED310100AD2E01000D2F0100AE
:10402000E52E0100692F0100A12E0100A92F01003A
:1040300001289FBF034B53F820300B60002088BF3E
:10404000082070473C50FF1F014B00225A60704708
:104050006434FF1F70B5084E084D336804462A4685
:10406000014600200DF0D2FE33682A462146012089
:10407000BDE870400DF0CABE3450FF1F3C50FF1F1A
:10408000014B18680DF00DBF3450FF1F012810B50B
:10409000144603D002280ED004200BE0094B0A4A34
:1040A000DB6850681B681B6A9847003018BF012006
:1040B0002060002010BD034B034ADB6890681B683A
:1040C0001B6AF1E7847E02008C17FF1F022804BFE1
:1040D0000B4B93F8D80030B90A4BDB681B685B695F
:1040E000094A10681847012809D1054B93F8D830C0
:1040F000012B04D1034BDB681B689B69F0E7704719
:104100006434FF1F847E02008C17FF1F70B50020EF
:10411000FFF7DCFF084B094CDD6820682B689B68C3
:1041200098472B6860689B6898472B68A0689B68D5
:10413000BDE87040184700BF847E02008C17FF1F47
:104140002DE9F843184C9DF820609DF824509846BE
:1041500023680F469B68002147F0800091469847EE
:10416000236800219B6848469847236800219B6884
:1041700040469847236800219B683046984723684B
:1041800028469B6801219847084B1B6848EA092884
:1041900007F07F0746EA082603EB870745EA06256E
:1041A0007D60BDE8F88300BF3850FF1F3450FF1F0B
:1041B00007B5D3B20193C2F307230093C2F30743B9
:1041C000120EFFF7BDFF03B05DF804FB0020FFF700
:1041D000EFBF01282DE9F341054688462AD8164F3E
:1041E0000744202697F89432864074B273B1134B7B
:1041F0001B6846F0070203EB820344F007015A688C
:10420000C9B2FFF7D5FF002387F8943244F00D01BF
:1042100042460024C9B22846FFF7CAFF2846CDE926
:10422000004423462246F1B2FFF78AFF204602B03F
:10423000BDE8F0810820FAE73C50FF1F3450FF1F13
:10424000012873B505460C4621D82026864084EA0D
:10425000E47246F00701A2EBE472C9B2FFF7A8FFCF
:104260000C4B2B44002C4FF0010283F894224FF0AA
:104270000004ACBF13460223019328460094234652
:104280002246F1B2FFF75CFF204602B070BD082065
:10429000FBE700BF3C50FF1F0021D1E74942CFE7B9
:1042A000CEE738B5234B01F07F04234493F8143252
:1042B000DB0705D4204B1B6803EB8404606838BD22
:1042C0001E4D2B6800219B68204698472B680021D3
:1042D0009B68084698472B6800219B6808469847CA
:1042E0002B6800219B68084698472B6801219B6832
:1042F000002098472B6800219B68204698472B6830
:1043000000219B68084698472B68002104029B689F
:10431000084698472B68002104439B680846984745
:104320002B68240204439B68012100209847240243
:104330002043C4E73C50FF1F3450FF1F3850FF1F7D
:1043400010B500201446FFF7ACFF206010BD38B553
:104350000D462021814041F00101C9B20446FFF71A
:10436000A0FF2968014429602046BDE8384030E7B5
:104370001C2A2DE9F04104460D461E4600F02F830D
:1043800000F2AE800C2A00F03D8252D8052A00F0DF
:10439000DC8120D8022A00F0938109D8002A00F09D
:1043A0006D81012A00F07B8104242046BDE8F08164
:1043B000032A00F0A181042AF6D1C74B2021A9408D
:1043C0001B6841F00707BA001344002840F0A7819A
:1043D0005B683360E9E7082A00F0F38114D8062A05
:1043E00000F0C481072ADFD120278F4047F0100753
:1043F000FFB239462846002C40F0D581FFF751FF27
:1044000000F01F003060D0E70A2A00F0E9810B2A93
:10441000CAD1002840F0B9852021A94041F01501FA
:10442000C9B22846FFF73DFFC04300F001003060ED
:10443000BBE7122A00F0708227D80F2A00F04482CE
:1044400011D80D2A00F00C820E2AADD12021A940EE
:1044500041F01401C9B2002840F030822846FFF72D
:1044600020FF3060A1E7102A00F03F82112A9BD183
:104470002021A94041F00801C9B2002840F046823D
:104480002846FFF70EFF30608FE7152A00F06C8298
:1044900011D8132A00F05182142A85D12021A94075
:1044A00041F00B01C9B2002840F058822846FFF7BE
:1044B000F8FE306079E7172A00F07A82C0F0658252
:1044C000182A7FF471AF2021A94041F01301C9B22D
:1044D000002840F07E822846FFF7E3FE306064E764
:1044E000AB2A00F0238461D8A52A00F0288331D8B4
:1044F000A22A00F0DD8218D81D2A00F08C828C2AB6
:104500007FF452AF002840F08E82090141F06C0127
:1045100001F0FC012846FFF7C4FE4FF48073C0F39E
:10452000036043FA00F030603FE7A32A00F0DC822A
:10453000A42A7FF439AF0F0147F06C07FFB2394668
:104540002846002C40F0EC82FFF7ABFEC0F30030B1
:1045500030602AE7A82A00F09E8312D8A62A00F02D
:104560004483A72A7FF420AF0F0147F06C07FFB206
:1045700039462846002C40F08383FFF792FE3460D2
:1045800013E7A92A00F0A483AA2A7FF40DAF0F0134
:1045900047F06D07FFB239462846002C40F0B6833D
:1045A000FFF77FFEC0F303203060FEE6B52A00F07F
:1045B0004D842CD8AE2A00F0068414D8AC2A00F022
:1045C000D583AD2A7FF4F0AE0F0147F06D07FFB23F
:1045D00039462846002C40F0E683FFF762FEC0F320
:1045E00000603060E1E6B32A00F01284B42A7FF460
:1045F000DBAE002840F0CF84090141F06F01C9B261
:104600002846FFF74EFEC0F304403060CDE6CE2AC8
:1046100000F0678414D8B62A00F04084B82A7FF4EA
:10462000C3AE0F0147F06C07FFB239462846002C95
:1046300040F04784FFF735FEC0F340303060B4E609
:10464000D12AFFF4B1AED22A40F29384D32A7FF468
:10465000ABAE002840F06084002900F050840129AE
:104660007FF4A3AE01462846FFF71BFE00F0600072
:10467000A0F1200358425841306096E62021A9401D
:1046800041F00D01C9B220B92846FFF70AFE30609B
:104690008BE61A682846FFF78BFD002485E620216B
:1046A000A94041F00101C9B220B92846FFF7F9FD40
:1046B00030607AE61A682846FFF77AFD002474E62F
:1046C0002021A94041F00701C9B238B92846FFF7B7
:1046D000E8FD306069E600BF3450FF1FB34B2B4448
:1046E000012283F894223268002AB8BF5242284639
:1046F000FFF75EFD002458E6002840F03D842021AD
:10470000A94041F00201C9B22846FFF7CAFD10F4E2
:10471000000318BF4FF07F431843306045E632680E
:10472000002AB8BF52425A60C9B22846FFF7B9FD05
:10473000044608B1002438E63268002AB8BF524265
:10474000F9B22846FFF734FD2FE62021A94041F0B9
:104750000601C9B220B92846FFF7A3FD306024E660
:104760001A682846FFF724FD00241EE620278F4004
:1047700047F01007FFB2394628462CB9FFF791FDE4
:10478000C0F30420306010E6FFF78BFD33681B0296
:1047900003F4F85320F4F8521A4339462846FFF739
:1047A00007FD002401E6FFF77CFD336820F01F02BF
:1047B00003F01F031A4339462846FFF7F9FC00248B
:1047C000F3E5002840F0DB832021A94041F01501EA
:1047D000C9B22846FFF765FDC0F340203060E4E52C
:1047E000002840F0CF832021A94041F01501C9B233
:1047F0002846FFF756FD10F0020F0CBF01230023DF
:104800003360D2E520278F4047F01407FFB23946C6
:1048100028462CB9FFF745FDC0F340003060C4E5E1
:10482000FFF73FFD3368002B0CBF0023022320F06D
:1048300002021A4339462846FFF7BAFC3946284691
:10484000FFF72FFD3368022B20F0080214BF00236E
:1048500008231A4339462846FFF7AAFC0024A4E59A
:1048600020278F4047F01407FFB2394628462CB95D
:10487000FFF717FD00F00100306096E5FFF711FD2E
:10488000326820F00100002A0CBF024640F001020D
:1048900039462846FFF78CFC39462846FFF701FDCC
:1048A0003368022B20F0040214BF002304231A43B0
:1048B00039462846FFF77CFC002476E51A6828462E
:1048C000FFF776FC002470E52021A94041F00401A7
:1048D000C9B220B92846FFF7E4FC306065E51A68E4
:1048E0002846FFF765FC00245FE52021A94041F040
:1048F0000501C9B220B92846FFF7D3FC306054E562
:104900001A682846FFF754FC00244EE51A6828462A
:10491000FFF74EFC002448E52021A94041F00A01A0
:10492000C9B220B92846FFF7BCFC30603DE51A68E3
:104930002846FFF73DFC002437E52021A94041F03F
:104940000301C9B220B92846FFF7ABFC30602CE563
:104950001A682846FFF72CFC002426E51A6828462A
:10496000FFF726FC002420E52021A94041F00C019E
:10497000C9B220B92846FFF794FC306015E51A68E3
:104980002846FFF715FC00240FE52021A94041F03F
:104990001101C9B220B92846FFF783FC306004E555
:1049A0001A682846FFF704FC0024FEE43C50FF1F71
:1049B0002021A94041F01201C9B220B92846FFF7D1
:1049C00070FC3060F1E41A682846FFF7F1FB002420
:1049D000EBE41A682846FFF7EBFB0024E5E40F013F
:1049E00047F06C07FFB2394628462CB9FFF759FC4F
:1049F000C0F380403060D8E4FFF753FC33689B0479
:104A000003F4802320F480221A4339462846FFF716
:104A1000CFFB0024C9E4002840F0BA82CA4B53F807
:104A200021303360C1E41B68102B3BD00DDC022B1E
:104A300034D004DC012B16D04FF0FF3314E0042BEC
:104A40002ED0082BF8D105230EE0402B2CD003DC10
:104A5000202BF1D1032307E0802B27D0B3F5807FF3
:104A6000EAD1002300E008233360336801333FF4C8
:104A700061AE2C0144F06C04E4B221462846FFF7F5
:104A800010FC33681B0603F0706320F0706221464F
:104A90001A432846FFF78CFB002486E40723E3E74C
:104AA0000623E1E70423DFE70223DDE70123DBE759
:104AB0000F0147F06C07FFB2394628462CB9FFF7C3
:104AC000F0FBC0F3C13030606FE4FFF7EAFB3368FE
:104AD000DB0303F4C03320F4C0321A4339462846BE
:104AE000FFF766FB002460E40F0147F06C07FFB29C
:104AF000394628462CB9FFF7D4FBC0F3803030602C
:104B000053E4FFF7CEFB33689B0303F4804320F4A8
:104B100080421A4339462846FFF74AFB002444E402
:104B2000FFF7BFFB33681B0303F4805320F480526C
:104B30001A4339462846FFF73BFB002435E40F01B2
:104B400047F06C07FFB239462846FFF7AAFB00F48E
:104B50008048B4B9B8F1000F07D039462846FFF7AE
:104B6000A0FBC0F3C31030601FE40311010503F084
:104B7000700301D43360DDE543F00803336044463D
:104B800013E439462846B8F1000F0FD0FFF789FB30
:104B90003368DB0103F4F06320F4F0621A43394612
:104BA0002846FFF705FB0024FFF7FFBBFFF779FB63
:104BB0003268120220F4006002F4006202433946B7
:104BC0002846FFF7F5FA39462846FFF76AFB3368AF
:104BD0001B0103F0700320F070021A433946284687
:104BE000FFF7E6FA4446FFF7E0BB0F0147F06C071A
:104BF000FFB239462846FFF754FB3946804628461F
:104C0000C4B918F4804407D0FFF74BFBC0F302107F
:104C100030600024FFF7C9BBFFF743FB18F4006FB7
:104C2000C0F3C31001D1306084E540F0080030606B
:104C3000FFF7BBBBFFF735FB10F48044394628462D
:104C40000FD0FFF72EFB33681B0103F0700320F039
:104C500070021A4339462846FFF7AAFA0024FFF7E4
:104C6000A4BBFFF71EFB3368DB0103F4F06320F401
:104C7000F0621A4339462846FFF79AFAFFF795BBC8
:104C8000FFF70FFB394620F00F022846FFF790FA96
:104C90000024FFF78ABB0F0147F06D07FFB23946CA
:104CA000284634B9FFF7FDFAC0F3C0303060FFF793
:104CB0007CBBFFF7F6FA3368DB039BB220F40042BB
:104CC0001A4339462846FFF773FA0024FFF76DBBF5
:104CD0000F0147F06D07FFB23946284634B9FFF798
:104CE000E0FAC0F341303060FFF75FBBFFF7D9FA5D
:104CF00033685B0303F4C04320F4C0421A433946CF
:104D00002846FFF755FA0024FFF74FBBFFF7C9FA13
:104D100033681B0203F4706320F470621A4339464F
:104D20002846FFF745FA0024FFF73FBB0F0147F085
:104D30006D07FFB23946284644B9FFF7B2FAC0F30F
:104D400041103060FFF731BB3C50FF1FFFF7A9FA5D
:104D500033685B0103F0600320F060021A433946B8
:104D60002846FFF725FA0024FFF71FBB0F0147F085
:104D70006D07FFB23946284634B9FFF792FA00F0C2
:104D80000F003060FFF711BBFFF78BFA336820F09C
:104D90000F0203F00F031A4339462846FFF708FABB
:104DA0000024FFF702BBFFF77CFA33681B0603F011
:104DB000807320F080721A4339462846FFF7F8F9CD
:104DC0000024FFF7F2BA0F0147F06D07FFB2394632
:104DD00028466CB9FFF765FA001400F07F0310F065
:104DE000400018BF6FF07F0018433060FFF7DDBA56
:104DF000FFF757FA33681B0403F4FE0320F4FE02A6
:104E00001A4339462846FFF7D3F90024FFF7CDBAF5
:104E10000F0147F06C07FFB23946284634B9FFF757
:104E200040FAC0F340403060FFF7BFBAFFF739FAED
:104E300033685B0403F4003320F400321A4339462C
:104E40002846FFF7B5F90024FFF7AFBA20278F40B7
:104E50007FB247F01101C9B228B92846FFF721FAFD
:104E60003060FFF7A2BA47F014041A68E4B228468B
:104E7000FFF79EF921462846FFF713FA3368002B07
:104E800020F480620CBF00234FF4806321461A4354
:104E90002846FFF78DF90024FFF787BA2021A940A3
:104EA00041F01101C9B228B92846FFF7FAF930607C
:104EB000FFF77BBA1A682846FFF77AF90024FFF754
:104EC00074BAFFF7EEF933685B0303F4005320F480
:104ED00000521A4339462846FFF76AF90024FFF7C3
:104EE00064BA00285AD1090141F06F01C9B22846BD
:104EF000FFF7D7F9C0F309003060FFF756BA08464C
:104F0000FFF7CFF900F01800A0F110025042504115
:104F100030602C46FFF749BA21B1012915D0002491
:104F2000FFF743BA0846FFF7BCF9336820F01802D0
:104F300043B142F0100200210846FFF739F900247E
:104F4000FFF733BA42F00802F5E700212846FFF7E1
:104F5000A8F9336820F0600243B142F0200200213A
:104F60000120FFF725F90024FFF71FBA42F04002A5
:104F7000F5E70024FFF719BA0424FFF716BA042452
:104F8000FFF713BA0424FFF710BA0424FFF70DBA91
:104F90000424FFF70ABA0424FFF707BA0424FFF732
:104FA00004BA07B50129019207D8024601AB0120D6
:104FB000FFF7DEF903B05DF804FB0820FAE70129EA
:104FC000134603D802460020FFF7D2B908207047E5
:104FD00008B522210020FFF764F950B942210120D1
:104FE000FFF75FF928B9044B1868BDE808400CF0DA
:104FF0004FBF002008BD00BF3450FF1F70B52D4EBD
:105000002D482E4D0CF0C6FEF468636803F58272DD
:1050100003F1640003F59273AB6023686A60DB6898
:1050200028609847236868681B6998472368A868C0
:105030001B699847224B32691A606368214903F55E
:1050400031735360204B5A690A602049C2F8041238
:105050001F49C2F8081201211170002151701D4A28
:105060001A621D4ADA611D4A9A611D4A5A621D4A36
:105070009A631D4A5A631D4A9A621D4ADA621D4AA2
:105080009A641D4A5A641D4A5A651D4A1A651D4A8A
:10509000DA641D4A1A661D4ADA6502204FF48C72E2
:1050A0003221C3E902211874194A9A65BDE870409B
:1050B000FFF70CB8847E02003C50FF1F8C17FF1FC7
:1050C0003850FF1F3450FF1F6434FF1FD14F0100C1
:1050D0008140010041420100A14201009D420100C6
:1050E00099420100BF4F0100A34F0100D3410100CD
:1050F0004F430100CD4101004143010055400100F3
:105100008D40010031400100CD40010049400100C7
:105110000D41010001289FBF044B03EB8000C369D0
:105120000B6094BF00200820704700BFD852FF1FBB
:10513000014B00225A6070476434FF1F024B024645
:10514000196802480CF0AEBFD452FF1FD852FF1F9F
:105150000A46014601480CF0D7BE00BFD852FF1FD7
:1051600010B500201446FFF7F3FF206010BD38B5DE
:1051700014460A46014603481D460CF0C5FE204071
:10518000E84038BDD852FF1F13460A460146014881
:105190000CF0B6BED852FF1F0020F5E72DE9F0470E
:1051A0000C4D089C06460F4690460A460146284686
:1051B00099460CF0A9FE04FA09F2424002EA0802FC
:1051C00082EA000331463A462846BDE8F0470CF033
:1051D00097BE00BFD852FF1F014B18680CF024BFC8
:1051E000D452FF1F08B522210020FFF7B1FF50B9AC
:1051F00042210120FFF7ACFF28B9044B1868BDE835
:1052000008400CF008BF002008BD00BFD452FF1FAB
:10521000012810B5144611D003D302281AD0042057
:1052200009E0104B104ADB6824681B68D0681CB189
:105230005B699847002010BD9B69FAE7094B0A4A51
:10524000DB6850681B681B6A9847003018BF012054
:105250002060EFE7034B044ADB6890681B681B6A19
:10526000F2E700BF847E0200A417FF1F022804BFDC
:105270000B4B93F8D80030B90A4BDB681B685B69AD
:10528000094A10681847012809D1054B93F8D8300E
:10529000012B04D1034BDB681B689B69F0E7704767
:1052A0006434FF1F847E0200A417FF1F70B5002026
:1052B000FFF7DCFF104B114CDD6820682B689B6802
:1052C00098472B6860689B6898472B68A0689B6824
:1052D00098472B68A0699B6898472B6820699B6852
:1052E00098472B6860699B6898472B68E0689B68C3
:1052F000BDE87040184700BF847E0200A417FF1F5E
:1053000001282DE9F041044688461DD80F4F07EBD0
:1053100080072025FA6985406EB232B146F0070158
:10532000C9B2FFF731FF0023FB6146F00D01424691
:10533000C9B22046FFF728FF20460022E9B2FFF756
:1053400023FF0020BDE8F0810820FBE7A417FF1F22
:1053500038B50D462021814041F00101C9B2044613
:10536000FFF7F6FE2968014429602046BDE8384071
:10537000C6E701282DE9F0410446884621D8124F9E
:1053800007EB800720258540FB6945F00706F6B24C
:105390001BB93146FFF7DCFEF86188EAE872A2EB40
:1053A000E87231462046FFF7EFFEB8F1000F2046C5
:1053B000B4BF02220122E9B2FFF7E6FE0020BDE8F9
:1053C000F0810820FBE700BFA417FF1F0021D0E7F2
:1053D0004942CEE7CDE71C2A2DE9F34104460D46AC
:1053E0001E4600F0FB8200F2AD800C2A00F03B82EA
:1053F00051D8052A00F0E3811ED8022A00F0A281CC
:1054000007D8002A00F07681012A00F08781042461
:105410007AE1032A00F0AA81042AF8D1C84B20219E
:10542000A9401B6841F00707BA001344002840F068
:10543000B0815B68336067E1082A00F0F28113D81D
:10544000062A00F0CD81072AE1D12021A94041F0B0
:105450001001C9B2002840F0DB8103461F22284614
:10546000FFF785FE30604FE10A2A00F0EA810B2A3F
:10547000CDD1002840F04D852021A94041F01501F3
:1054800003460122C9B22846FFF771FEB0FA80F048
:105490004009306038E1122A00F03F8227D80F2AF5
:1054A00000F0138211D80D2A00F0F3810E2AAED13C
:1054B0002021A94041F01401C9B2002840F0FF8129
:1054C0002846FFF745FE30601EE1102A00F00E82EC
:1054D000112A9CD12021A94041F00801C9B200281D
:1054E00040F015822846FFF733FE30600CE1152AA4
:1054F00000F03B8211D8132A00F02082142A86D1B2
:105500002021A94041F00B01C9B2002840F02782B8
:105510002846FFF71DFE3060F6E0172A00F04782AC
:10552000C0F03482182A7FF472AF2021A94041F0E4
:105530001301C9B2002840F04B822846FFF708FE4D
:105540003060E1E0AC2A00F0CA8362D8A52A00F0FE
:10555000DB8232D8A22A00F09F8219D81D2A00F0DF
:1055600054828C2A7FF453AF002840F057820901FF
:1055700041F06C0118234FF0706201F0FC012846E5
:10558000FFF7F5FD4FF4807343FA00F03060BBE0A5
:10559000A32A00F09882A42A7FF439AF090141F0D0
:1055A0006C01C9B2002840F0A5820C234FF4805250
:1055B0002846FFF7DCFD3060A6E0A82A00F0438310
:1055C00013D8A62A00F0F382A72A7FF420AF09019E
:1055D00041F06C01C9B2002840F02C8303460F2231
:1055E0002846FFF7C4FD30608EE0AA2A4FEA011179
:1055F00000F0568340F23E8341F06D01C9B20028AD
:1056000040F06483052360222846FFF7B0FD306038
:105610007AE0B62A00F0D7833DD8B32A00F0988309
:105620001AD8AD2A00F07383AE2A7FF4F0AE0901D8
:1056300041F06D01C9B2002840F0808310234FF47F
:10564000FE022846FFF793FD10F0400318BF6FF0ED
:105650007F031843306057E0B42A00F09083B52AE6
:105660007FF4D5AE20278F407FB247F014085FFA51
:1056700088F8002840F0928341462846FFF768FDED
:10568000410540F1918047F01101C9B22846FFF76A
:105690005FFD306038E0CE2A00F0C78314D8B82A06
:1056A00000F0A283B92A7FF4B2AE090141F06C0187
:1056B000C9B2002840F0AF8314234FF4700228468B
:1056C000FFF755FD30601FE0D22A00F0C283D32AD5
:1056D00000F0D083D12A7FF49AAE2021A94041F076
:1056E0001901C9B2002840F0AE832846FFF730FD0B
:1056F000306009E02021A94041F00D01C9B238B95C
:105700002846FFF725FD3060204602B0BDE8F08155
:105710001A682846FFF738FD0024F5E72021A94044
:1057200041F00101C9B220B92846FFF711FD3060F0
:10573000EAE71A682846FFF727FD0024E4E700BFE0
:10574000D452FF1F2021A94041F00701C9B220B95E
:105750002846FFF7FDFC3060D6E71A68002AB8BF7C
:1057600052422846FFF710FD0024CDE7002840F004
:10577000C8832021A94041F00201C9B22846FFF7A1
:10578000E7FC10F4000318BF4FF07F43184330606C
:10579000BAE73268002AB8BF52425A60C9B22846F6
:1057A000FFF7D6FC044608B10024ADE73268002AB2
:1057B000B8BF5242F9B22846FFF7E6FCA4E7202121
:1057C000A94041F00601C9B220B92846FFF7C0FC44
:1057D000306099E71A682846FFF7D6FC002493E763
:1057E0002021A94041F01001C9B238B908234FF473
:1057F000F8522846FFF7BBFC306085E71B68009332
:105800004FF4F85208232846FFF7C8FC00247BE732
:105810001B6800931F2200232846FFF7BFFC0024CB
:1058200072E7002840F06F832021A94041F0150164
:1058300009234FF40072C9B22846FFF798FC306084
:1058400062E7002840F062832021A94041F0150161
:1058500001230222C9B22846FFF789FCB0FA80F082
:105860004009306050E72021A94041F01401C9B23D
:1058700030B9012302222846FFF779FC306043E764
:105880001B680093022201232846FFF787FC0024AF
:105890003AE72021A94041F01401C9B230B90023F0
:1058A00001222846FFF763FC30602DE71B68009358
:1058B000012200232846FFF771FC002424E71A6820
:1058C0002846FFF761FC00241EE72021A94041F093
:1058D0000401C9B220B92846FFF73AFC306013E74B
:1058E0001A682846FFF750FC00240DE72021A94044
:1058F00041F00501C9B220B92846FFF729FC306004
:1059000002E71A682846FFF73FFC0024FCE61A6805
:105910002846FFF739FC0024F6E62021A94041F093
:105920000A01C9B220B92846FFF712FC3060EBE645
:105930001A682846FFF728FC0024E5E62021A94044
:1059400041F00301C9B220B92846FFF701FC3060DD
:10595000DAE61A682846FFF717FC0024D4E61A682E
:105960002846FFF711FC0024CEE62021A94041F093
:105970000C01C9B220B92846FFF7EAFB3060C3E644
:105980001A682846FFF700FC0024BDE62021A94044
:1059900041F01101C9B220B92846FFF7D9FB3060A8
:1059A000B2E61A682846FFF7EFFB0024ACE6202198
:1059B000A94041F01201C9B220B92846FFF7C8FB3F
:1059C0003060A1E61A682846FFF7DEFB00249BE65C
:1059D0001A682846FFF7D8FB002495E6090141F034
:1059E0006C01C9B238B912234FF480222846FFF760
:1059F000BEFB306088E61B6800934FF480221223C0
:105A00002846FFF7CBFB00247EE6002840F0848286
:105A1000B94800EB8100C369336075E61B68102B41
:105A200034D00DDC022B2DD004DC012B16D04FF02E
:105A3000FF3314E0042B27D0082BF8D105230EE008
:105A4000402B25D003DC202BF1D1032307E0802B52
:105A500020D0B3F5807FEAD1002300E00823336033
:105A60003368581C3FF4A0AE290141F06C0100934B
:105A70004FF07062182301F0FC012846FFF78EFBFF
:105A8000002441E60723EAE70623E8E70423E6E7E4
:105A90000223E4E70123E2E7090141F06C01C9B206
:105AA00038B90F234FF4C0322846FFF760FB30604F
:105AB0002AE61B6800934FF4C0320F232846FFF7F5
:105AC0006DFB002420E6090141F06C01C9B238B930
:105AD0000E234FF480422846FFF749FB306013E65F
:105AE0001B6800934FF480420E232846FFF756FBB5
:105AF000002409E61B6800934FF480520C232846CB
:105B0000FFF74CFB0024FFE50F0147F06C07FFB2E5
:105B100040BB0E234FF4804239462846FFF727FB4F
:105B2000804640B107234FF4F06239462846FFF71C
:105B30001EFB3060E8E50423702239462846FFF753
:105B400016FB0B2330604FF4006239462846FFF7FE
:105B50000EFB00283FF428AE336843F0080333609F
:105B60004446D1E539462846FFF7F2FA10F480445E
:105B7000336809D000934FF4F06207233946284672
:105B8000FFF70CFB0024BFE5C3F3C00300933946C5
:105B900028460B234FF40062FFF700FB33680093A5
:105BA0007022042339462846FFF7F8FAACE50F01C6
:105BB00047F06C07FFB23946284624BBFFF7C8FA06
:105BC00010F4804408D00423702239462846FFF799
:105BD000CEFA0024306097E507234FF4F06239468F
:105BE0002846FFF7C4FA0B2330604FF400623946B1
:105BF0002846FFF7BCFA00283FF4D6AD336843F0DF
:105C00000803336080E5FFF7A3FA3368009310F4CC
:105C1000804407D00423702239462846FFF7BEFA95
:105C2000002471E507234FF4F06239462846FFF758
:105C3000B5FA69E51B6800930F2200232846FFF799
:105C4000ADFA002460E5090141F06D01C9B238B92F
:105C50000F234FF400422846FFF789FA306053E5DE
:105C60001B6800934FF400420F232846FFF796FA73
:105C7000002449E541F06D01C9B238B90D234FF454
:105C8000C0422846FFF773FA30603DE51B68009379
:105C90004FF4C0420D232846FFF780FA002433E575
:105CA00041F06D01C9B238B908234FF4706228463B
:105CB000FFF75DFA306027E51B6800934FF47062D0
:105CC00008232846FFF76AFA00241DE51B680093A5
:105CD000602205232846FFF761FA002414E5090134
:105CE00041F06D01C9B248B903460F222846FFF7BB
:105CF0003EFA306008E500BFD852FF1F1B680093D2
:105D00000F2200232846FFF749FA0024FCE409018A
:105D100041F06D01C9B238B918234FF0807228469E
:105D2000FFF725FA3060EFE41B6800934FF08072B4
:105D300018232846FFF732FA0024E5E41B68009395
:105D40004FF4FE0210232846FFF728FA0024DBE474
:105D5000090141F06C01C9B238B911234FF4003286
:105D60002846FFF704FA3060CEE41B6800934FF436
:105D7000003211232846FFF711FA0024C4E400285A
:105D800040F0CD80090141F06F0110234FF4F8126B
:105D9000C9B22846FFF7EBF93060B5E447F01101CE
:105DA0001A68C9B22846FFF7EFF93368003318BF05
:105DB000012300934FF480620A2341462846FFF7EF
:105DC000EDF90024A0E42021A94041F01101C9B25D
:105DD00020B92846FFF7BCF9306095E41A682846D8
:105DE000FFF7D2F900248FE4090141F06C01C9B238
:105DF00038B90D234FF400522846FFF7B8F9306048
:105E000082E41B6800934FF400520D232846FFF7ED
:105E1000C5F9002478E41B6800934FF47002142342
:105E20002846FFF7BBF900246EE400287AD1090167
:105E300041F06F01034640F2FF32C9B22846FFF736
:105E400096F9306060E41A682846FFF79DF900244F
:105E50005AE42021A94041F01A01C9B220B92846CC
:105E6000FFF776F930604FE41A682846FFF78CF99F
:105E7000002449E4D8B971B101297FF445AC014649
:105E80002846FFF765F900F06000A0F120035842B2
:105E90005841306038E40846FFF75AF900F018001E
:105EA000A0F110025042504130602C462CE419B150
:105EB000012913D0002427E40846FFF749F9336885
:105EC00020F018023BB142F0100200210846FFF713
:105ED0005BF9002418E442F00802F6E700212846A6
:105EE000FFF736F9336820F060023BB142F0200240
:105EF00000210120FFF748F9002405E442F04002A8
:105F0000F6E7042400E40424FFF7FEBB0424FFF7B3
:105F1000FBBB0424FFF7F8BB0424FFF7F5BB042404
:105F2000FFF7F2BB0424FFF7EFBB07B5012901928D
:105F300007D8024601AB0120FFF74DFA03B05DF828
:105F400004FB0820FAE70129134603D80246002083
:105F5000FFF741BA08207047012810B40C4606D854
:105F6000044B1B6820469B6810BC11461847002054
:105F700010BC70470055FF1FF0B5564E564F574B9B
:105F8000574C8BB00021304601220CF008F8FD6818
:105F90006B6803F58272626003F59272A26003F58A
:105FA0007172E26003F5797203F16400226103F219
:105FB000044203F22443A3612B686261DB68206022
:105FC00098472B68E068DB6898472B68E0689B6916
:105FD00098472B6860681B6998472B68A0681B6905
:105FE00098472B68A0691B6998472B6820691B6933
:105FF00098472B6860691B693A4C98473A4B3A6955
:106000001A606B68394803F5317353606369384A25
:10601000136004333360374B009303F19F2303F580
:106020006A0356330193344A344BCDE90223344B8F
:106030006FF08061CDE90413A3F1D943A3F5911367
:10604000A3F2272306932F4B6A46CDE907030021CD
:106050004FF477433046ADF824300CF088F86A46A8
:10606000012130460CF083F86369274AC3F8042203
:10607000264AC3F808220120002218705A70244BC7
:106080002362244BE361244BA361244B6362244BC2
:10609000A363244B6363244BA362244BE362244B2E
:1060A000A364244B6364244B6365244B2365244B16
:1060B000E364244B2366244BE365022323743225D7
:1060C000DE23C4E90235214BA365FFF7CFF80BB0FF
:1060D000F0BD00BFD852FF1F847E02000024F400F0
:1060E000A417FF1F6434FF1F0055FF1F224240000A
:1060F000D452FF1F54B5AAAA2929492422421010BC
:106100007D77BBB580FFFF56E5510100D9510100F5
:1061100073530100D5530100D1530100CD53010049
:10612000475F01002B5F0100015301005153010043
:1061300099510100615101003D51010011520100CE
:10614000155101006D52010031510100AD520100A5
:1061500001289FBF034B53F820300B60002088BFFD
:10616000082070470855FF1F014B00225A607047F6
:106170006434FF1F70B5084E084D336804462A4644
:10618000014600200CF0B0F933682A462146012070
:10619000BDE870400CF0A8B90455FF1F0855FF1F5B
:1061A00010B5002014460CF010F9206010BD00203E
:1061B0000CF0FDB80A46014601480CF018BA00BFC1
:1061C0000855FF1F0968F5E70A46014601480CF02B
:1061D000DFB900BF0855FF1F0021F5E74942F3E78B
:1061E000F2E7024B18680CF0CAB900BF0455FF1F54
:1061F00008B5222108480CF0E8F850B942210648B9
:106200000CF0E3F828B9054B1868BDE808400CF01D
:10621000ADB9002008BD00BF0855FF1F0455FF1F82
:10622000012810B5144611D003D302281AD0042037
:1062300009E0104B104ADB6824681B68D0681CB169
:106240005B699847002010BD9B69FAE7094B0A4A31
:10625000DB6850681B681B6A9847003018BF012034
:106260002060EFE7034B044ADB6890681B681B6AF9
:10627000F2E700BF847E0200D417FF1F022804BF8C
:106280000B4B93F8D80030B90A4BDB681B685B698D
:10629000094A10681847012809D1054B93F8D830EE
:1062A000012B04D1034BDB681B689B69F0E7704747
:1062B0006434FF1F847E0200D417FF1F70B50020D6
:1062C000FFF7DCFF104B114CDD6820682B689B68E2
:1062D00098472B6860689B6898472B68A0689B6804
:1062E00098472B68A0699B6898472B6820699B6832
:1062F00098472B6860699B6898472B68E0689B68A3
:10630000BDE87040184700BF847E0200D417FF1F0D
:106310001C2AF7B506460C461F4600F0298300F2FA
:10632000AB800C2A00F035824FD8052A00F0D481CA
:106330001ED8022A00F0908107D8002A00F064815C
:10634000012A00F07481042668E1032A00F09B8191
:10635000042AF8D1BE4B2021A1401B6841F007055B
:10636000AA001344002840F0A1815B683B6055E11E
:10637000082A00F0F08114D8062A00F0BE81072A0E
:10638000E1D1202101FA04F444F01004E4B22146E2
:10639000B048002E40F0CF810CF017F8C0B2386042
:1063A0003CE10A2A00F0E6810B2ACCD1002840F01B
:1063B000ED852021A14041F01501C9B2A5480CF09E
:1063C00004F800F00100386028E1122A00F06D8224
:1063D00027D80F2A00F0418211D80D2A00F0088238
:1063E0000E2AB0D12021A14041F01401C9B20028E9
:1063F00040F02D8297480BF0E8FF38600EE1102A3C
:1064000000F03C82112A9ED12021A14041F00801D8
:10641000C9B2002840F043828E480BF0D6FF3860A6
:10642000FCE0152A00F0698211D8132A00F04E8290
:10643000142A88D12021A14041F00B01C9B20028C3
:1064400040F0558283480BF0C0FF3860E6E0172A21
:1064500000F07782C0F06482182A7FF474AF2021A4
:10646000A14041F01301C9B2002840F07B82794875
:106470000BF0ABFF3860D1E0AB2A00F00D8463D89D
:10648000A52A00F0258331D8A22A00F0DA8218D894
:106490001D2A00F089828C2A7FF455AF002840F035
:1064A0008B82090141F06C0101F0FC0169480BF09D
:1064B0008CFF4FF4807300F00F0043FA00F0386057
:1064C000ACE0A32A00F0D982A42A7FF43CAF0C01EF
:1064D00044F06C04E4B221465E48002E40F0E982AC
:1064E0000BF073FFC0F30030386097E0A82A00F08B
:1064F0008D8314D8A62A00F03483A72A7FF423AF13
:106500000C0144F06C04E4B221465248002E40F0E5
:106510006F830BF05AFF00F00F0038607EE0A92A6D
:1065200000F08F83AA2A7FF40EAF0C0144F06D04B3
:10653000E4B221464748002E40F09F830BF045FF10
:10654000C0F30320386069E0B52A00F02A842CD813
:10655000AE2A00F0E78314D8AC2A00F0B983AD2A44
:106560007FF4F1AE0C0144F06D04E4B221463948E9
:10657000002E40F0C8830BF028FFC0F300603860A5
:106580004CE0B32A00F0F183B42A7FF4DCAE00289B
:1065900040F00285090141F06F01C9B22D480BF0AE
:1065A00014FFC0F30440386038E0CE2A00F04F8476
:1065B00014D8B62A00F02884B82A7FF4C4AE0C019F
:1065C00044F06C04E4B221462248002E40F02F84AF
:1065D0000BF0FBFEC0F3403038601FE0D22A00F021
:1065E0004C84D32A00F05C84D12A7FF4ACAE202105
:1065F000A14041F01901C9B2002840F03784154884
:106600000BF0E3FE386009E02021A14041F00D01CC
:10661000C9B230B90F480BF0D8FE3860304603B02D
:10662000F0BD1A680B480BF0C2FE0026F6E72021E9
:10663000A14041F00101C9B220B906480BF0C5FEE6
:106640003860EBE71A6803480BF0B1FE0026E5E777
:106650000455FF1F0855FF1F2021A14041F00701ED
:10666000C9B2AB481EB90BF0B0FE3860D6E704449F
:10667000012384F894323A68002AB8BF52420BF0E2
:1066800096FE0026CAE7002840F077842021A1402A
:1066900041F00201C9B29E480BF097FE10F40003CE
:1066A00018BF4FF07F4318433860B7E73A689848FF
:1066B000002AB8BF52425A60C9B20BF086FE0646A5
:1066C00008B10026AAE73A689148002AB8BF5242AA
:1066D000E9B20BF06CFEA1E72021A14041F00601D8
:1066E000C9B220B98A480BF070FE386096E71A6884
:1066F00087480BF05CFE002690E7202101FA04F4A5
:1067000044F01004E4B2214681482EB90BF05DFE3E
:10671000C0F30720386081E70BF057FEC3B2019346
:106720003B7800930022C0F30743214678480BF0E2
:1067300007FE002672E70BF048FE3B780193C0F39A
:10674000072300930022C0F30743214670480BF053
:10675000F7FD002662E7002840F012842021A140C6
:1067600041F01501C9B26A480BF02FFEC0F340207A
:10677000386053E7002840F006842021A14041F012
:106780001501C9B262480BF020FEC0F3400038602A
:1067900044E7202101FA04F444F01404E4B2214651
:1067A0005B482EB90BF011FEC0F34000386035E7AE
:1067B0000BF00BFE3B68002BD4BF0023022320F01C
:1067C00002021A43214652480BF0F1FD214650487F
:1067D0000BF0FBFD3B68022B20F0080214BF0023E6
:1067E00008231A4321464A480BF0E1FD002615E72D
:1067F000202101FA04F444F01404E4B22146444890
:106800002EB90BF0E2FD00F00100386006E70BF056
:10681000DCFD3A6820F00100002AD4BF024640F0B7
:10682000010221463A480BF0C2FD214638480BF0E0
:10683000CCFD3B68022B20F0040214BF002304238C
:106840001A43214632480BF0B2FD0026E6E61A68EC
:106850002F480BF0ACFD0026E0E62021A14041F0DE
:106860000401C9B220B92A480BF0AFFD3860D5E663
:106870001A6827480BF09BFD0026CFE62021A14097
:1068800041F00501C9B220B921480BF09EFD3860E6
:10689000C4E61A681E480BF08AFD0026BEE61A6898
:1068A0001B480BF084FD0026B8E62021A14041F0F2
:1068B0000A01C9B220B916480BF087FD3860ADE671
:1068C0001A6813480BF073FD0026A7E62021A140AB
:1068D00041F00301C9B220B90D480BF076FD3860D4
:1068E0009CE61A680A480BF062FD002696E61A68D4
:1068F00007480BF05CFD002690E62021A14041F006
:106900000C01C9B230B902480BF05FFD386085E672
:106910000855FF1F1A68B5480BF049FD00267DE6B3
:106920002021A14041F01101C9B220B9AF480BF0BC
:106930004CFD386072E61A68AC480BF038FD002652
:106940006CE62021A14041F01201C9B220B9A7484C
:106950000BF03BFD386061E61A68A4480BF027FD98
:1069600000265BE61A68A1480BF021FD002655E6DB
:106970000C0144F06C04E4B221469C482EB90BF0A3
:1069800024FDC0F38040386048E60BF01EFD3B68F4
:106990009B0403F4802320F480221A432146934869
:1069A0000BF005FD002639E6002840F0F2828F4BFF
:1069B00053F821303B6031E61B68102B3BD00DDCD7
:1069C000022B34D004DC012B16D04FF0FF3314E03F
:1069D000042B2ED0082BF8D105230EE0402B2CD011
:1069E00003DC202BF1D1032307E0802B27D0B3F564
:1069F000807FEAD1002300E008233B603B6801333D
:106A00003FF45FAE240144F06C04E4B221467748C1
:106A10000BF0DBFC3B681B0603F0706320F0706238
:106A20001A43214671480BF0C2FC0026F6E5072305
:106A3000E3E70623E1E70423DFE70223DDE70123A1
:106A4000DBE70C0144F06C04E4B2214667482EB940
:106A50000BF0BBFCC0F3C1303860DFE50BF0B5FCD8
:106A60003B68DB0303F4C03320F4C0321A432146F1
:106A70005E480BF09CFC0026D0E50C0144F06C0451
:106A8000E4B2214659482EB90BF09FFCC0F34030C8
:106A90003860C3E50BF099FC3B685B0303F40053DB
:106AA00020F400521A43214650480BF080FC002687
:106AB000B4E50BF08AFC3B681B0303F4805320F41D
:106AC00080521A43214649480BF071FC0026A5E587
:106AD0000D0145F06C05EDB2294644480BF075FCFC
:106AE0002946C0F3803441486EB92CB10BF06DFCDF
:106AF000C0F3C310386091E50BF067FCC0F30210DF
:106B0000386026468AE574B10BF05FFC3B68DB0118
:106B100003F4F06320F4F0621A43294633480BF083
:106B200046FC00267AE50BF050FC3A68120220F48D
:106B3000006002F40062024329462C480BF037FC47
:106B400029462A480BF041FC3B681B0103F0700307
:106B500020F070021A43294624480BF028FC2646F0
:106B60005CE50D0145F06C05EDB229461F480BF0C0
:106B70002CFC2946C0F380341C48BEB92CB10BF064
:106B800024FCC0F30210386048E50BF01EFCC0F393
:106B9000C3103860294615480BF017FC3B68000A03
:106BA00000F0080003433B60264637E574B10BF064
:106BB0000CFC3B681B0103F0700320F070021A43C9
:106BC00029460A480BF0F3FB002627E50BF0FDFBF6
:106BD0003B68DB0103F4F06320F4F0621A432946BA
:106BE00002480BF0E4FB264618E500BF0855FF1FDE
:106BF0000BF0EBFB3B6820F00F0203F00F031A438E
:106C00002146BA480BF0D3FB002607E50C0144F0FF
:106C10006D04E4B22146B5482EB90BF0D6FBC0F3A3
:106C2000C0303860FAE40BF0D0FB3B68DB039BB26A
:106C300020F400421A432146AC480BF0B8FB002672
:106C4000ECE40C0144F06D04E4B22146A7482EB9EF
:106C50000BF0BBFBC0F341303860DFE40BF0B5FB59
:106C60003B685B0303F4C04320F4C0421A4321464F
:106C70009E480BF09CFB0026D0E40BF0A6FB3B6883
:106C80001B0203F4706320F470621A432146974894
:106C90000BF08DFB0026C1E40C0144F06D04E4B25E
:106CA000214692482EB90BF090FBC0F3411038609A
:106CB000B4E40BF08AFB3B685B0103F0600320F057
:106CC00060021A43214689480BF071FB0026A5E4B7
:106CD0000C0144F06D04E4B2214684482EB90BF057
:106CE00074FB00F00F00386098E40BF06EFB3B681B
:106CF00020F00F0203F00F031A4321467B480BF0EC
:106D000056FB00268AE40BF060FB3B681B0603F091
:106D1000807320F080721A43214674480BF047FBC1
:106D200000267BE40C0144F06D04E4B221466F4878
:106D300066B90BF04AFB001400F07F0310F040002E
:106D400018BF6FF07F001843386067E40BF03DFB1D
:106D50003B681B0403F4FE0320F4FE021A432146A1
:106D600062480BF024FB002658E40C0144F06C044C
:106D7000E4B221465D482EB90BF027FBC0F340403A
:106D800038604BE40BF021FB3B685B0403F40033F9
:106D900020F400321A43214654480BF008FB002629
:106DA0003CE42021A1404DB245F01404E4B288B97E
:106DB00021464E480BF009FB10F4806007D045F0E7
:106DC0001101C9B249480BF000FB386026E4386075
:106DD000064623E445F011011A684448C9B20BF095
:106DE000E6FA214641480BF0F0FA3B68002B20F40C
:106DF00080620CBF00234FF480631A4321463B4856
:106E00000BF0D5FA002609E42021A14041F0110140
:106E1000C9B228B935480BF0D8FA3860FFF7FEBB85
:106E20001A6832480BF0C3FA0026FFF7F7BB0BF0E5
:106E3000CCFA3B685B0303F4005320F400521A437E
:106E400021462A480BF0B3FA0026FFF7E7BB0028DB
:106E500040F0A580090141F06F01C9B223480BF051
:106E6000B4FAC0F309003860FFF7D8BB1A681F48AE
:106E70000BF09DFA0026FFF7D1BB2021A14041F085
:106E80001A01C9B228B919480BF09FFA3860FFF708
:106E9000C5BB1A6815480BF08AFA0026FFF7BEBB7F
:106EA000E8B979B101297FF4B9AB01460F480BF07D
:106EB0008CFA00F06000A0F120035842584138607D
:106EC000FFF7ACBB09480BF080FA00F01800A0F106
:106ED00010025042504138602646FFF79FBB39B13F
:106EE000012927D00026FFF799BB00BF0855FF1FD7
:106EF0002C480BF06AFA3B68002B14BF00230823D0
:106F000020F008021A43214626480BF050FA214689
:106F100024480BF05AFA3B68002B20F010020CBFFB
:106F2000002310231A4321461E480BF040FA264640
:106F3000FFF774BB00211B480BF047FA3B68002B9E
:106F40000CBF0023202320F020021A430021154803
:106F50000BF02DFA002113480BF037FA3B68002B99
:106F600020F0400214BF002340231A4300210D48A3
:106F70000BF01DFA0026FFF751BB0426FFF74EBBAE
:106F80000426FFF74BBB0426FFF748BB0426FFF798
:106F900045BB0426FFF742BB0426FFF73FBB042690
:106FA000FFF73CBB0855FF1F07B50129019207D821
:106FB000024601AB0120FFF7ABF903B05DF804FB1B
:106FC0000820FAE70129134603D802460020FFF7FC
:106FD0009FB908207047034B1B6808469B68114601
:106FE000184700BFA457FF1FF8B53F4C3F4F20463E
:106FF0000BF03CFA0026FD6884F896626B683C4C06
:1070000003F58272626003F59272A26003F57172F9
:10701000E26003F5797203F16400226103F2044235
:1070200003F22443A3612B686261DB682060984708
:107030002B68E068DB6898472B68E0689B69984795
:107040002B6860681B6998472B68A0681B69984784
:107050002B68A0691B6998472B6820691B699847B2
:107060002B6860691B699847224B3A691A606B6804
:10707000214903F531735360204B5A690A60204956
:10708000C2F804121F49C2F808120121117056708B
:107090001D4A1A621D4ADA611D4A9A611D4A5A62E6
:1070A0001D4A9A631D4A5A631D4A9A621D4ADA6252
:1070B0001D4A9A641D4A5A641D4A5A651D4A1A653A
:1070C0001D4ADA641D4A1A661D4ADA6502204FF429
:1070D0008C723221C3E9022118741A4A9A65BDE8FC
:1070E000F840FFF7CBB800BF0855FF1F847E0200B1
:1070F000D417FF1FA457FF1F0455FF1F6434FF1F41
:10710000F1610100E3610100C9610100E161010079
:10711000DD610100D9610100C56F0100A96F0100A7
:10712000B5610100C5610100AF610100A16101000D
:107130007561010021620100516101007D62010061
:1071400069610100BD62010018B9034B5B680B6007
:1071500070470820704700BFA857FF1F014B00224F
:107160005A6070476434FF1F0428F8B5144677D07E
:1071700008D8012845D01ED302285FD0032830D07C
:1071800004242FE0062800F09480C0F087800728B0
:1071900000F09680FC28F3D1514B524DDE68146804
:1071A00033682869002C00F09680DB6898473368C4
:1071B00028699B6914E0126832F0030340F08D8067
:1071C000474B484DDE6868683368D2070CD51B69A9
:1071D000984724683268286814F002040AD01369BA
:1071E000984700242046F8BDDB68984733686868F4
:1071F0009B69EDE7D3689847336828689B6998478F
:10720000F0E7126844F620639A4266DC354B586A10
:10721000334BDB6842F210711B688A42CCBF5B695A
:107220009B699847226842F2117392FBF3F003FBCB
:1072300010202D4B80B29B689847D2E7284B1468EA
:10724000DD68D5E9003000F5F2703CB1DB689847A5
:10725000D5E900309B6900F5F270C1E79B68CEE785
:107260001F4B204EDF6815683B68306945B1012D22
:107270000FD01B6998473B6830691B6A984706E046
:10728000DB6898473B689B693069984728462060CF
:10729000A7E7DB6898473B685B69F5E7104B114A45
:1072A000DB68D0691B681B6A9847003018BF012053
:1072B000EDE70B4B0B4ADB68106A1B681B6AF3E7B0
:1072C000084B12689869064BDB681B68012A0CBFE3
:1072D0005B699B6984E71B6991E7102482E700BF23
:1072E000847E0200FC17FF1F7409FF1F1C4B70B542
:1072F000DD681C4C2B68A0689B6998472B68A06AC6
:107300009B6898472B68606A9B6898472B68E06881
:107310009B6898472B6820699B6898472B68606931
:107320009B6898472B6820689B6898472B68606823
:107330009B6898472B68E0699B6898472B68206A90
:107340009B6898472B68A0699B6898472B68A06842
:107350009B689847044BBDE870405B68184700BFC6
:10736000847E0200FC17FF1F7409FF1F01480BF009
:10737000B6B900BFA857FF1F014601480BF030BA4D
:10738000A857FF1F10B5034814460BF0B6F920604C
:1073900010BD00BFA857FF1F08B5034B03481A686C
:1073A0000BF0AEFA002008BD3C5AFF1FA857FF1F84
:1073B00008B5034B03481A680BF08EFA002008BD8D
:1073C0003C5AFF1FA857FF1F08B502480BF081FA6F
:1073D000002008BDA857FF1F08B502480BF076FA39
:1073E000002008BDA857FF1F08B502480BF06CFA33
:1073F000002008BDA857FF1F08B502480BF050FA3F
:10740000002008BDA857FF1F01480BF0D0B900BFEE
:10741000A857FF1F38B522210B480BF06EF910B9A1
:1074200009480BF0AFF9094B094CDD68606A2B681D
:107430009B6998472B6820681B6998472B68606890
:107440001B699847012038BDA857FF1F847E0200A2
:10745000FC17FF1F022804BF0B4B93F8D80030B96C
:107460000A4BDB681B685B69094A9068184701286A
:1074700009D1054B93F8D830012B04D1034BDB68BD
:107480001B689B69F0E770476434FF1F847E02002D
:10749000FC17FF1F012903D1024A70210BF01FB90D
:1074A000704700BFC80405008C2970B50446154616
:1074B00000F01A8300F298800E2900F02F8241D844
:1074C000062900F0B38119D8022900F06C8107D891
:1074D000002900F04B81012900F0578104244BE181
:1074E000042900F07D8140F26C81002840F09781F2
:1074F0002621BE480BF001F928603DE10A2900F081
:10750000C4810FD8072900F0A9810829E6D10028F5
:1075100040F00C863521B5480BF0EFF8C0F3402061
:10752000286029E10C2900F0CA8140F2BC81342195
:10753000AE48002C40F0DF810BF0DFF800F00100D6
:10754000286019E1152900F03D821FD8112900F0AB
:1075500008820DD80F2900F0EF811029BED1002834
:1075600040F0F8812521A1480BF0C7F8286003E11D
:10757000132900F0128240F20282002840F01B82A0
:107580002B219A480BF0B9F82860F5E01C2900F08F
:107590005F821AD8182900F035821B2900F040823A
:1075A00017299BD1924E002840F01A8215218F484E
:1075B0000BF0A3F830B14FF08073B3FBF0F08642CC
:1075C00028BF06462E600024D6E0212900F058820C
:1075D000222900F06F821D2980D1002840F0AF855C
:1075E000824B5B681360C7E0B32900F0308457D842
:1075F000A82900F0958324D8A42900F0EB8210D8A4
:10760000A22900F0C082A3297FF468AF6C217748DB
:10761000002C40F0D0820BF070F8C0F3803028606E
:10762000AAE0A62900F02C8340F2EC826C216F487E
:10763000002C40F067830BF060F800F00F0028602A
:107640009AE0AB2900F0AD8310D8A92900F07F8320
:10765000AA297FF443AF6D216448002C40F0928347
:107660000BF04BF8C0F30320286085E0AD2900F053
:10767000C783C0F0AE83AE297FF430AF6D215B4885
:10768000002C40F0D5830BF038F8001400F07F0395
:1076900010F0400018BF6FF07F00184328606BE0C7
:1076A000BB2900F0898436D8B62900F017841FD88A
:1076B000B42900F0E483B5297FF410AF34214B489E
:1076C000002C40F0E9830BF018F8430540F1E28309
:1076D000142146480BF011F8454B30B14FF0807241
:1076E000B2FBF0F0834228BF03462B60002443E046
:1076F000B92900F0248400F23A84B8297FF4EEAE70
:107700006C213A48002C40F00B840AF0F6FFC0F3DD
:107710004030286030E0CC2900F0C88412D8BF295E
:1077200000F08084C02900F09D84BC297FF4D6AE8F
:1077300070212E48002C40F068840AF0DEFFC0B2B1
:10774000286019E0D12900F0CB84D22900F0D88438
:10775000CE297FF4C3AE002840F0F7846F21234880
:107760000AF0CBFFC0F30900286005E030B92D21F5
:107770001E480AF0C2FF2860204670BD12681B48F0
:107780002D210AF0ACFF0024F6E728B92121174883
:107790000AF0B3FF2860EFE71268144821210AF0CD
:1077A0009EFF0024E8E728B9272110480AF0A5FF2A
:1077B0002860E1E712680D4827210AF090FF0024B5
:1077C000DAE7002840F0AC84222108480AF095FF4F
:1077D00010F4000318BF4FF07F4318432860CBE735
:1077E000044E48B933681360C6E700BFA857FF1FAF
:1077F000FFFF0F003C5AFF1F1368A648002BB8BFBD
:107800005B42202133600AF078FF0446002840F0F4
:107810008A8432689F4827210AF061FFACE712682A
:107820009C4826210AF05BFF0024A5E71021994817
:107830002CB90AF062FFC0F3042028609CE70AF02C
:107840005CFF2B681B0203F4F85320F4F8521A4330
:10785000102190480AF043FF00248DE710218D4845
:107860002CB90AF04AFF00F01F00286084E70AF0F4
:1078700044FF2B6820F01F0203F01F031A4310215E
:1078800084480AF02CFF002476E7002840F0518459
:10789000352180480AF031FF10F0020F0CBF0123A0
:1078A00000232B6068E7002840F0468435217948A2
:1078B0000AF023FFC04300F0010028605CE7342198
:1078C00074482CB90AF019FFC0F34000286053E750
:1078D0000AF013FF2C6834B940F0020234216D48DD
:1078E0000AF0FDFE48E720F00202342169480AF060
:1078F000F6FE002440E70AF000FF2C6834B940F09F
:107900000102342163480AF0EAFE35E720F0010263
:10791000342160480AF0E3FE00242DE728B9342121
:107920005C480AF0EAFE286026E7126859483421CC
:107930000AF0D5FE00241FE728B9242155480AF093
:10794000DCFE286018E71268524824210AF0C7FEBE
:10795000002411E712684F4825210AF0C0FE0024D8
:107960000AE728B928214B480AF0C7FE286003E738
:107970001268484828210AF0B2FE0024FCE628B923
:107980002A2144480AF0B9FE2860F5E61268414809
:107990002A210AF0A4FE0024EEE628B923213D485E
:1079A0000AF0ABFE2860E7E612683A4823210AF0A5
:1079B00096FE0024E0E6126836482B210AF08FFE7E
:1079C0000024D9E628B92C2132480AF096FE286016
:1079D000D2E612682F482C210AF081FE0024CBE663
:1079E00013686BB14FF0807292FBF3F2B242A8BF02
:1079F00032462A60152127480AF071FE0024BBE6B2
:107A00003246F6E728B9332122480AF076FE28608C
:107A1000B2E612681F4833210AF061FE0024ABE68B
:107A20006C211C482CB90AF068FEC0F3C0402860E5
:107A3000A2E60AF062FE2B68DB0403F4002320F4C4
:107A400000221A436C2113480AF049FE002493E6F1
:107A50006C2110482CB90AF050FEC0F38040286019
:107A60008AE60AF04AFE2B689B0403F4802320F484
:107A700080221A436C2107480AF031FE00247BE67D
:107A80000021044844B90AF038FE00F001002860E3
:107A900072E600BFA857FF1F0AF02FFE2B6820F0E8
:107AA000010203F001031A430021B5480AF017FE52
:107AB000002461E638B90146B1480AF01EFEC0F361
:107AC0004000286058E60021AD480AF016FE2B68F9
:107AD0005B0003F0020320F002021A430021A848D1
:107AE0000AF0FDFD002447E658B96C21A4480AF0CD
:107AF00004FE4FF48073C0F3036043FA00F0286083
:107B00003AE61368102B27D00DDC022B20D004DCC2
:107B1000012B16D04FF0FF3314E0042B1AD0082BA2
:107B2000F8D105230EE0402B18D003DC202BF1D137
:107B3000032307E0802B13D0B3F5807FEAD1002325
:107B400000E008232B602B6801330BD1102413E6CF
:107B50000723F7E70623F5E70423F3E70223F1E71A
:107B60000123EFE76C2186480AF0C7FD2B681B064E
:107B700003F0706320F070621A436C2180480AF0B1
:107B8000AEFD0024F8E56C217D482CB90AF0B5FD66
:107B9000C0F3C1302860EFE50AF0AFFD2B68DB03CE
:107BA00003F4C03320F4C0321A436C2174480AF045
:107BB00096FD0024E0E50AF0A0FD2B689B0303F48A
:107BC000804320F480421A436C216D480AF087FDFF
:107BD0000024D1E56C216A482CB90AF08EFDC0F36F
:107BE00000302860C8E50AF088FD2B681B0303F409
:107BF000805320F480521A436C2161480AF06FFDD3
:107C00000024B9E56C215E480AF077FD00F480435A
:107C100094B93BB16C215A480AF06FFDC0F3C31010
:107C20002860A9E5C0F3021300F4006003430CBF11
:107C3000002308232B609FE583B16C2150480AF094
:107C40005CFD2B68DB0103F4F06320F4F0621A435F
:107C50006C214B480AF043FD00248DE52A6811078A
:107C60004CBF40F4006020F40060120120F070006E
:107C7000D2B202436C2142480AF031FD00247BE578
:107C80006C213F480AF039FDACB910F4804307D0AD
:107C90006C213B480AF031FDC0F3021028606BE50F
:107CA000C0F3C31200F4006002430CBF002208229C
:107CB0002A601C4660E56C2131480AF01EFD10F474
:107CC00080444FF06C012E480ED00AF016FD2B6850
:107CD0001B0103F0700320F070021A436C21284846
:107CE0000AF0FDFC002447E50AF007FD2B68DB01E4
:107CF00003F4F06320F4F0621A436C2120480AF088
:107D0000EEFC39E50AF0F9FC2B6820F00F0203F0D5
:107D10000F031A436C211A480AF0E1FC00242BE5FA
:107D20006D2117482CB90AF0E8FCC0F3C030286078
:107D300022E50AF0E2FC2B68DB039BB220F4004250
:107D40001A436D210E480AF0CAFC002414E56D2187
:107D50000B482CB90AF0D1FCC0F3413028600BE588
:107D60000AF0CBFC2B685B0303F4C04320F4C04251
:107D70001A436D2102480AF0B2FC0024FCE400BF63
:107D8000A857FF1F0AF0B9FC2B681B0203F47063AD
:107D900020F470621A436D21B7480AF0A0FC002459
:107DA000EAE46D21B4482CB90AF0A7FCC0F34110F5
:107DB0002860E1E40AF0A1FC2B685B0103F060039A
:107DC00020F060021A436D21AB480AF088FC0024C1
:107DD000D2E46D21A8482CB90AF08FFC00F00F0006
:107DE0002860C9E40AF089FC2B6820F00F0203F038
:107DF0000F031A436D21A0480AF071FC0024BBE474
:107E00006D219D482CB90AF078FCC0F30060286011
:107E1000B2E40AF072FC2B681B0603F0807320F0BA
:107E200080721A436D2194480AF059FC0024A3E49F
:107E30000AF063FC2B681B0403F4FE0320F4FE022B
:107E40001A436D218C480AF04AFC002494E46C210A
:107E500089482CB90AF051FCC0F3404028608BE4FB
:107E60000AF04BFC2B685B0403F4003320F400326F
:107E70001A436C2180480AF032FC00247CE400287C
:107E800040F060816F217C480AF037FCC0F3044069
:107E9000286071E42C606FE40AF02FFC2B68002B43
:107EA0000CBF00234FF4806320F480621A43342116
:107EB00071480AF014FC2968704B69B14FF0807268
:107EC00092FBF1F29A42A8BF1A462A6014216A482E
:107ED0000AF005FC00244FE41A46F6E7674E70B935
:107EE000142165480AF009FC30B14FF08072B2FBF2
:107EF000F0F2964228BF16462E6000243CE4136838
:107F000063B14FF0807292FBF3F2B242A8BF3246E7
:107F1000142159480AF0E3FB00242DE43246F7E728
:107F20000AF0EBFB2B685B0303F4005320F40052D0
:107F30001A436C2150480AF0D2FB00241CE46C2147
:107F40004D482CB90AF0D9FBC0F30350286013E464
:107F50000AF0D3FB2B681B0503F4700320F47002B6
:107F60001A436C2144480AF0BAFB002404E4434E4F
:107F700078B9132140480AF0C0FB30B14FF080734C
:107F8000B3FBF0F0864228BF06462E600024FFF7C0
:107F9000F3BB136873B14FF0807292FBF3F2B242FD
:107FA000A8BF32462A60132133480AF098FB002408
:107FB000FFF7E2BB3246F5E770212F4834B90AF0EB
:107FC0009CFBC0F307202860FFF7D6BB0AF095FBA7
:107FD0002A68120220F47F4092B2024370212648A0
:107FE0000AF07DFB002124480AF087FB2B68002B58
:107FF00020F004020CBF002304231A4300211E4872
:108000000AF06DFB0024FFF7B7BB0AF076FB2A7875
:1080100020F0FF000243702117480AF060FB0024A3
:10802000FFF7AABB40B9702113480AF066FBC0F302
:1080300001402860FFF7A0BB1368032B3FF686AD15
:1080400070210D480AF059FB2B681B0403F44033E0
:1080500020F440321A43702107480AF040FB002404
:10806000FFF78ABB60B9702103480AF046FBC0F3F2
:1080700080402860FFF780BBA857FF1FFFFF0F005D
:108080001368012B3FF662AD702131480AF035FBD1
:108090002B689B0403F4802320F480221A43702170
:1080A0002B480AF01CFB0024FFF766BB7021284810
:1080B00034B90AF022FBC0F301502860FFF75CBB23
:1080C0000AF01BFB2B681B0503F4401320F440123D
:1080D0001A4370211E480AF002FB0024FFF74CBB34
:1080E00030B939211A480AF008FB2860FFF744BB71
:1080F0001268174839210AF0F2FA0024FFF73CBB56
:1081000030B93A2112480AF0F8FA2860FFF734BB78
:1081100012680F483A210AF0E2FA0024FFF72CBB5C
:108120000424FFF729BB0024FFF726BB0424FFF734
:1081300023BB0424FFF720BB0424FFF71DBB04244A
:10814000FFF71ABB0424FFF717BB0424FFF714BB87
:10815000A857FF1F07B5019239B9014601AA0120AE
:10816000FFF7A2F903B05DF804FB0820FAE70B461D
:1081700019B901461846FFF797B908207047034B15
:108180001B680846DB681146184700BF385AFF1FB6
:108190002DE9F041584E594CF568594F6B6803F181
:1081A0006402A26003F1A402E26003F1C40222614E
:1081B00003F59272226003F5A272626003F5D27237
:1081C000626203F5E272A26203F5617203F1840058
:1081D000A26103F5697203F57173E3612B68226292
:1081E0001B69606198472B6820691B6998472B6859
:1081F000E0681B6998472B68E0691B6998472B6802
:10820000206A1B6998472B68A069DB6898472B6830
:1082100020681B6998472B6860681B6998472B6822
:10822000A068DB6898472B68606ADB6898472B6812
:10823000A06ADB6898472B68A0699B699847314B17
:1082400032691A606B683049304803F53173536006
:108250002F4B5A69C2F804122E49C2F808120026A0
:1082600001211170567018622B48D8612B48986113
:108270002B4858622B4898632B4858632B489862C8
:108280002B48D8622B4898642B4858642B48586573
:108290002B4818652B48D8642B4818662B48D8659E
:1082A000197432204FF4F071C3E90210284999651E
:1082B0003846284B31460AF048FA274938460AF032
:1082C0008BFA3B68D3F8A020244B02201A60FFF7FA
:1082D000C1F82B68A06ADB689847A06A204C042389
:1082E00043752B681B68984723689847A3683046F6
:1082F000BDE8F041184700BF847E0200FC17FF1F55
:10830000A857FF1F385AFF1F15740100F9730100A9
:108310006434FF1F09740100E9730100D97301007F
:10832000C97301006F81010055810100B173010023
:10833000997301006D730100857301007973010069
:108340006971010049710100557401005D710100FE
:10835000ED7201007C7A0200957401003C5AFF1F07
:108360007409FF1F18B9034B1B680B607047082086
:10837000704700BF485AFF1F014B00225A607047E8
:108380006434FF1F0428F8B50C46154667D005D89D
:1083900002283DD04ED8B0B104242AE0062800F0CF
:1083A00087807AD3FC28F7D1474B484EDF681468A2
:1083B0003B683069002C00F08280DB6898473B689E
:1083C00030699B6913E0126832F0030379D13E4BA8
:1083D0003E4EDF6870683B68D2070CD51B69984732
:1083E0002C683B68306814F002040AD01B69984777
:1083F00000242046F8BDDB6898473B6870689B699D
:10840000EDE7DB6898473B6830689B699847F0E781
:108410002D4B1468DE68D6E9003000F5F2703CB1EF
:10842000DB689847D6E900309B6900F5F270DEE71B
:108430009B68EBE7254B9869234BDB681B6839B1D8
:10844000146814F0010401D05B69D0E79B69DDE793
:108450001B6A9847003018BF01202860C9E71A4BF3
:108460001A4EDF6814683B68306944B1012C0FD0A4
:108470001B6998473B6830691B6A984706E0DB68D0
:1084800098473B689B693069984720462860AFE76A
:10849000DB6898473B685B69F5E70B4B0B4ADB6889
:1084A000106A1B681B6A9847003018BF0120EDE76F
:1084B000054B064ADB68506A1B681B6AF3E71B69B9
:1084C000A4E7102495E700BF847E02003418FF1F44
:1084D0001C4B70B5DD681C4C2B68A0689B699847E5
:1084E0002B68A0699B6998472B68E0699B6998474E
:1084F0002B68E0689B6898472B6820699B689847C1
:108500002B6860699B6898472B6820689B68984730
:108510002B6860689B6898472B68206A9B6898471F
:108520002B68606A9B6898472B68A0689B6898478F
:108530002B68A0699B6898472B68E0699B68BDE839
:1085400070401847847E02003418FF1F034B044A12
:108550001B68014600200AF01ABA00BF445AFF1FE8
:10856000485AFF1F014B18680AF04BBA445AFF1FC4
:10857000022804BF0B4B93F8D80030B90A4BDB68D4
:108580001B685B69094A90681847012809D1054BA7
:1085900093F8D830012B04D1034BDB681B689B692F
:1085A000F0E770476434FF1F847E02003418FF1F19
:1085B0002DE9F0471C4D9DF820709DF824609946E8
:1085C00055F82030044688469B68002148F080001A
:1085D0009246984755F8243000219B6850469847AA
:1085E00055F8243000219B684846984755F82430B8
:1085F00000219B683846984755F8243030469B68E0
:1086000001219847094B53F8243049EA0A2908F018
:108610007F0847EA092703EB880846EA0726C8F8D7
:108620000460BDE8F08700BF405AFF1F445AFF1F97
:1086300007B5D3B20193C2F307230093C2F30743F4
:10864000120EFFF7B5FF03B05DF804FB0020FFF743
:10865000EFBF73B50D460646E8B9104C94F82830C4
:1086600043B10F4B1B682721D3F8A020FFF7E0FF91
:1086700084F8286000242A462D210020FFF7D8FF27
:108680002046CDE90044234622462021FFF790FFF3
:10869000204602B070BD0820FBE700BF3418FF1F62
:1086A000445AFF1F37B50D460446C8B90D4B012289
:1086B00083F8282081EAE172A2EBE1722721FFF71B
:1086C000B7FF002DACBF01230223CDE900432046B4
:1086D000234622462021FFF76BFF204603B030BD22
:1086E0000820FBE73418FF1F0021DBE74942D9E7E8
:1086F000D8E770B52B4A4FF4247301F07F0403FBD5
:1087000000232344054693F80C32DB0706D4264B9E
:1087100053F8203003EB8404606870BD234E56F894
:10872000203000219B682046984756F825300021CC
:108730009B680846984756F8253000219B680846F4
:10874000984756F8253000219B680846984756F808
:10875000253001219B680020984756F825300021DC
:108760009B682046984756F8253000219B680846AC
:10877000984756F82530002104029B680846984720
:1087800056F82530002104439B680846984756F860
:108790002530240204439B680121002098472402CD
:1087A0002043BAE7485AFF1F445AFF1F405AFF1F91
:1087B00010B500201446FFF79CFF206010BD38B5AF
:1087C0000C4621210546FFF794FF216801442160F2
:1087D0002846BDE838403CE7222970B504461546D6
:1087E00000F0E98200F287800E2900F00B823ED86B
:1087F000062900F0998118D8022900F04F8107D886
:10880000002900F02F81012900F03B8104242FE191
:10881000042900F0658140F25581002840F07D81F7
:108820002621FFF766FF286022E10A2900F0AB81CC
:108830000ED8072900F090810829E7D1002840F0E0
:10884000E8853521FFF755FFC0F3402028600FE190
:108850000C2900F0B08140F2A3813421002840F0BF
:10886000C281FFF746FF00F00100286000E11529F2
:1088700000F019821DD8112900F0E6810CD80F29CB
:1088800000F0CD811029C1D1002840F0D6812521EA
:10889000FFF72FFF2860EBE0132900F0EF8140F293
:1088A000E081002840F0F8812B21FFF722FF2860AB
:1088B000DEE01B2900F038820CD8172900F007826F
:1088C0001829A3D1002840F028823321FFF711FF97
:1088D0002860CDE01D2900F05782C0F03D8221299B
:1088E00094D1002840F057820146FFF702FF00F0C4
:1088F00001002860BCE0AE2900F01D8450D8A729F3
:1089000000F0848329D8A32900F0CD820FD88C29C8
:1089100000F06A82A2297FF479AF6C21002840F030
:10892000B282FFF7E6FEC0F3C1302860A0E0A529BF
:1089300000F0E98240F2CF826C210020FFF7D9FEDF
:1089400000F48046002C40F03B83002E00F02D8385
:10895000000900F0700028608AE0AA2900F09483E2
:108960000FD8A82900F06983A9297FF44FAF6D21A2
:10897000002840F07983FFF7BCFEC0F34130286047
:1089800076E0AC2900F0B08340F296836D21002898
:1089900040F0C183FFF7ADFEC0F30060286067E0E0
:1089A000BB2900F0858434D8B62900F013841ED882
:1089B000B42900F0DF83B5297FF428AF34210028E3
:1089C00040F0E583FFF795FE430540F1DE83142177
:1089D0002046FFF78EFEB74B30B14FF08072B2FBEE
:1089E000F0F0834228BF03462B60002440E0B92901
:1089F00000F0228400F23884B8297FF407AF6C219C
:108A0000002840F00984FFF774FEC0F3403028606E
:108A10002EE0CC2900F0C18411D8BF2900F07E845B
:108A2000C02900F09B84BC297FF4F0AE702100289F
:108A300040F06684FFF75DFEC0B2286018E0D129DF
:108A400000F0C584D22900F0D284CE297FF4DEAEB6
:108A5000002840F0ED846F21FFF74BFEC0F30900C2
:108A6000286005E030B92D210020FFF742FE286084
:108A7000204670BD12682D210020FFF7D9FD00248B
:108A8000F6E720B92121FFF734FE2860F0E71268ED
:108A900021210020FFF7CCFD0024E9E720B92721A0
:108AA000FFF727FE2860E3E71268002AB8BF5242AA
:108AB00027210020FFF7BCFD7F4B012283F82820EF
:108AC0000024D5E7002840F0A1842221FFF711FE01
:108AD00010F4000318BF4FF07F4318432860C7E726
:108AE000764B1A6818B9D2F8A0302B60C0E72B6813
:108AF000002BB8BF5B42C2F8A03020210020FFF756
:108B0000F8FD044608B10024B2E72A68002AB8BF7D
:108B100052422721FFF78CFDAAE712682621002088
:108B2000FFF786FD0024A3E7102128B9FFF7E1FD38
:108B3000C0F3042028609BE70020FFF7DAFD2B68D4
:108B40001B0203F4F85320F4F8521A4310210020BA
:108B5000FFF76EFD00248BE7102100202CB9FFF7F2
:108B6000C8FD00F01F00286082E7FFF7C2FD2B68F8
:108B700020F01F0203F01F031A4310210020FFF70B
:108B800057FD002474E7002840F046843521FFF7A4
:108B9000B0FD10F0020F0CBF012300232B6067E72C
:108BA000002840F03C843521FFF7A3FDC04300F0CE
:108BB000010028605CE7342100202CB9FFF799FD03
:108BC000C0F34000286053E7FFF793FD2B685B007C
:108BD00003F0020320F002021A4334210020FFF7C1
:108BE00027FD002444E70020FFF783FD2B6820F0D9
:108BF000010203F001031A4334210020FFF718FD9E
:108C0000002435E720B93421FFF773FD28602FE7F2
:108C1000126834210020FFF70BFD002428E728B953
:108C200024210020FFF765FD286021E71268242138
:108C30000020FFF7FDFC00241AE712682521002020
:108C4000FFF7F6FC002413E720B92821FFF751FDB8
:108C500028600DE7126828210020FFF7E9FC0024B6
:108C600006E720B92A21FFF744FD286000E71268D3
:108C70002A210020FFF7DCFC0024F9E628B9232193
:108C80000020FFF736FD2860F2E61268232100205D
:108C9000FFF7CEFC0024EBE612682B210020FFF743
:108CA000C7FC0024E4E658B92C21FFF722FD286018
:108CB000DEE600BFFFFF0F003418FF1F445AFF1FFE
:108CC00012682C210020FFF7B3FC0024D0E688B9FD
:108CD00015210020FFF70DFD50B14FF08073B3FB5D
:108CE000F0F0C04B984228BF184628600024BFE629
:108CF000BC48FAE7136873B14FF0807292FBF3F24D
:108D0000B84B9A42A8BF1A462A6015210020FFF7E7
:108D10008FFC0024ACE6B34AF6E71268332100204A
:108D2000FFF786FC0024A3E66C2128B9FFF7E1FCDD
:108D3000C0F3C04028609BE60020FFF7DAFC2B68F8
:108D4000DB0403F4002320F400221A436C210020EA
:108D5000FFF76EFC00248BE66C2128B9FFF7C9FCF5
:108D6000C0F38040286083E60020FFF7C2FC2B6838
:108D70009B0403F4802320F480221A436C210020FA
:108D8000FFF756FC002473E6002840F04B83964B17
:108D90001B6813606CE600210846FFF7AAFC2B68ED
:108DA00020F0010203F0010300211A430846FFF7F7
:108DB0003FFC00245CE630B90146FFF79AFCC0F3A3
:108DC0004000286054E600210846FFF792FC2B681B
:108DD0005B0003F0020320F0020200211A43084660
:108DE000FFF726FC002443E658B96C210020FFF76A
:108DF00080FC4FF48073C0F3036043FA00F02860F6
:108E000036E61368102B27D00DDC022B20D004DCB3
:108E1000012B16D04FF0FF3314E0042B1AD0082B8F
:108E2000F8D105230EE0402B18D003DC202BF1D124
:108E3000032307E0802B13D0B3F5807FEAD1002312
:108E400000E008232B602B6801330BD110240FE6C0
:108E50000723F7E70623F5E70423F3E70223F1E707
:108E60000123EFE76C210020FFF743FC2B681B0672
:108E700003F0706320F070621A436C210020FFF74A
:108E8000D7FB0024F4E50020FFF733FC2B68DB035D
:108E900003F4C03320F4C0321A436C210020FFF7E2
:108EA000C7FB0024E4E56C2128B9FFF722FCC0F3DE
:108EB00080302860DCE50020FFF71BFC2B689B035B
:108EC00003F4804320F480421A436C210020FFF712
:108ED000AFFB0024CCE56C2128B9FFF70AFCC0F3F6
:108EE00000302860C4E50020FFF703FC2B681B035B
:108EF00003F4805320F480521A436C210020FFF7C2
:108F000097FB0024B4E56C210020FFF7F2FB064636
:108F1000CCB910F4804405D0C60906F4F0662E6082
:108F20000024A5E56C212046FFF7E3FB16F00B0FAC
:108F30004FEA201000F0700001D12860E3E540F016
:108F40000800286094E56C210020FFF7D2FB10F4A4
:108F500080444FF06C010FD00020FFF7CAFB2B6854
:108F6000DB0103F4F06320F4F0621A436C2100206B
:108F7000FFF75EFB00247BE52046FFF7BAFB6C2180
:108F800020F400622046FFF753FB6C212046FFF7D8
:108F9000B0FB2B681B0103F0700320F070021A4332
:108FA0006C212046FFF744FB62E5C309020503F488
:108FB000F06301D42B60A6E543F008032B6057E56E
:108FC0006C219EB10020FFF794FB2B681B0103F07E
:108FD000700320F070021A436C210020FFF728FB79
:108FE000002445E5FFFF0F00485AFF1F3046FFF7FA
:108FF00080FB2B68DB0103F4F06320F4F0621A437A
:109000006C213046FFF714FB344631E56C2128B95A
:10901000FFF76FFB00F00F00286029E50020FFF745
:1090200068FB2B6820F00F0203F00F031A436C213A
:109030000020FFF7FDFA00241AE56D2100202CB96D
:10904000FFF757FBC0F3C030286011E5FFF751FB75
:109050002B68DB039BB220F400421A436D210020F1
:10906000FFF7E6FA002403E50020FFF742FB2B6838
:109070005B0303F4C04320F4C0421A436D21002077
:10908000FFF7D6FA0024F3E46D2128B9FFF731FB8E
:10909000C0F303202860EBE40020FFF72AFB2B68D5
:1090A0001B0203F4706320F470621A436D210020E8
:1090B000FFF7BEFA0024DBE46D2128B9FFF719FBA6
:1090C000C0F341102860D3E40020FFF712FB2B68A7
:1090D0005B0103F0600320F060021A436D21002061
:1090E000FFF7A6FA0024C3E46D2100202CB9FFF796
:1090F00000FB00F00F002860BAE4FFF7FAFA2B68D3
:1091000020F00F0203F00F031A436D210020FFF738
:109110008FFA0024ACE40020FFF7EBFA2B681B0663
:1091200003F0807320F080721A436D210020FFF756
:109130007FFA00249CE46D2160B9FFF7DAFA00148D
:1091400000F07F0310F0400018BF6FF07F0018435D
:1091500028608DE40020FFF7CCFA2B681B0403F491
:10916000FE0320F4FE021A436D210020FFF760FA8F
:1091700000247DE4002840F058816F210020FFF793
:10918000B8FAC0F30440286072E42C6070E4002058
:10919000FFF7AFFA2B68002B0CBF00234FF480635E
:1091A00020F480621A4334210020FFF741FA296835
:1091B000A14B69B14FF0807292FBF1F29A42A8BFC5
:1091C0001A462A6014210020FFF732FA00244FE4E7
:1091D0001A46F6E7984E68B91421FFF78AFA30B1BB
:1091E0004FF08073B3FBF0F0864228BF06462E6036
:1091F00000243DE413686BB14FF0807292FBF3F2F0
:10920000B242A8BF32462A6014210020FFF710FAAC
:1092100000242DE43246F6E70020FFF76AFA2B68B7
:109220005B0303F4005320F400521A436C21002026
:10923000FFF7FEF900241BE46C2100202CB9FFF796
:1092400058FAC0F30350286012E4FFF752FA2B6873
:109250001B0520F4700203F470031A436C210020F4
:10926000FFF7E6F9002403E4734E70B91321FFF70A
:1092700040FA30B14FF08073B3FBF0F0864228BF64
:1092800006462E600024FFF7F3BB136873B14FF05E
:10929000807292FBF3F2B242A8BF32462A601321D9
:1092A0000020FFF7C5F90024FFF7E2BB3246F5E7DF
:1092B000702130B9FFF71DFAC0F307202860FFF7CF
:1092C000D7BB0020FFF715FA2A68120220F47F406E
:1092D00092B2024370210020FFF7AAF9002108464C
:1092E000FFF707FA2B689B0003F0040320F0040249
:1092F00000211A430846FFF79BF90024FFF7B8BB8B
:109300000020FFF7F6F92A7820F0FF0002437021D1
:109310000020FFF78DF90024FFF7AABB40B97021A8
:109320000020FFF7E6F9C0F301402860FFF7A0BB7B
:109330001368032B3FF68AAD70210020FFF7D9F99F
:109340002B681B0403F4403320F440321A4370218D
:109350000020FFF76DF90024FFF78ABB38B97021B0
:10936000FFF7C7F9C0F380402860FFF781BB13689F
:10937000012B3FF66BAD70210020FFF7BAF92B6887
:109380009B0403F4802320F480221A4370210020E0
:10939000FFF74EF90024FFF76BBB702130B9FFF7E0
:1093A000A8F9C0F301502860FFF762BB0020FFF767
:1093B000A0F92B681B0503F4401320F440121A4354
:1093C00070210020FFF734F90024FFF751BB30B9BA
:1093D00039210020FFF78DF92860FFF749BB12689B
:1093E00039210020FFF724F90024FFF741BB28B9F9
:1093F0003A21FFF77EF92860FFF73ABB12683A215D
:109400000020FFF715F90024FFF732BB0424FFF713
:109410002FBB0424FFF72CBB0424FFF729BB042433
:10942000FFF726BB0424FFF723BB0424FFF720BB70
:109430000424FFF71DBB00BFFFFF0F0007B501921B
:1094400039B9014601AA0120FFF7C6F903B05DF85A
:1094500004FB0820FAE70B4619B901461846FFF746
:10946000BBB90820704738B522210020FFF741F929
:1094700018B9084B186809F0BBFA074B074CDD68B0
:1094800020682B681B6998472B6860681B699847A0
:10949000012038BD445AFF1F847E02003418FF1F8C
:1094A00070B5524E5248534C09F03AFAF5686B6861
:1094B00003F18402626103F1A402E26003F1C402D9
:1094C000226103F59272226003F5A272626003F5D5
:1094D000C272A26103F5E27203F16400E26103F576
:1094E000697203F5717323622B686262DB68A060A6
:1094F00098472B68A069DB6898472B68E069DB68B0
:1095000098472B68A0685B6998472B68A0699B699E
:1095100098472B68E0695B6998472B6860691B690D
:1095200098472B6820691B6998472B68E0681B697E
:1095300098472B68206A1B6998472B68606A1B69EB
:1095400098472B6820681B6998472B6860681B69DF
:109550009847D5E90030DB6800F5F2709847D5E907
:1095600000309B6900F5F2709847234B32691A600E
:109570006B68224903F531735360214B5A690A60C5
:109580002049C2F804122049C2F808120020012123
:10959000117050701D4A1A621D4ADA611D4A9A61A3
:1095A0001D4A5A621D4A9A631D4A5A631D4A9A62AD
:1095B0001D4ADA621D4A9A641D4A5A641D4A5A6558
:1095C0001D4A1A651D4ADA641D4A1A661D4ADA6583
:1095D00019744FF425723221C3E902211A4A9A659F
:1095E0000220BDE87040FEF7C3BF00BF847E0200CA
:1095F000485AFF1F3418FF1F405AFF1F445AFF1FCD
:109600006434FF1F6794010065850100A586010091
:10961000F1860100ED860100E98601005794010002
:109620003D94010053860100BF8701004D86010073
:10963000B18701004D85010085830100658301002C
:109640007185010079830100D184010018B9034BB1
:109650005B680B6070470820704700BF6C18FF1FE5
:10966000014B00225A6070476434FF1F0428F8B58C
:109670000C46154670D005D8022845D056D8C8B13A
:10968000042430E0062800F09480C0F08680FC2896
:10969000F6D14E4B4E4EDF6814683B68D6F8A002F8
:1096A000002C00F08E80DB6898473B68D6F8A0025B
:1096B0009B6916E0126832F0030340F08480434B4C
:1096C000434EDF68D6F894023B68D2070DD51B697C
:1096D00098472C683B68D6F8900214F002040BD02F
:1096E0001B69984700242046F8BDDB6898473B6813
:1096F000D6F894029B69EBE7DB6898473B68D6F89D
:1097000090029B699847EEE7304B1468DE68D6E913
:10971000003000F5F2703CB1DB689847D6E90030C4
:109720009B6900F5F270DCE79B68EBE7284BD3F808
:10973000A802264BDB681B6839B1146814F00104D9
:1097400001D05B69CDE79B69DCE71B6A9847003075
:1097500018BF01202860C6E71C4B1D4EDF68146847
:109760003B68D6F8A0024CB1012C11D01B69984778
:109770003B68D6F8A0021B6A984707E0DB68984769
:109780003B689B69D6F8A002984720462860A9E765
:10979000DB6898473B685B69F4E70C4B0C4ADB6875
:1097A000D2F8B0021B681B6A9847003018BF01202E
:1097B000ECE7064B064ADB68D2F8B4021B681B6A6A
:1097C000F2E71B699EE710248DE700BF847E02004C
:1097D0006C18FF1F234B70B5DD68234C2B68D4F841
:1097E00098029B6998472B68D4F8A8029B69984710
:1097F0002B68D4F8AC029B6998472B68D4F89C027C
:109800009B6898472B68D4F8A0029B6898472B6800
:10981000D4F8A4029B6898472B68D4F890029B6800
:1098200098472B68D4F894029B6898472B68D4F823
:10983000B0029B6898472B68D4F8B4029B6898479D
:109840002B68D4F898029B6898472B68D4F8A80234
:109850009B6898472B68D4F8AC029B68BDE87040C1
:10986000184700BF847E02006C18FF1F01460148A4
:1098700009F054B96C18FF1F10B50348144609F0DD
:109880000AF9206010BD00BF6C18FF1F014809F0E5
:10989000F4B800BF6C18FF1F10B5064A0446092132
:1098A00009F0EBF82046044A0A21BDE8104009F00F
:1098B000E4B800BF0C0C01000002080008B5034822
:1098C000D0F8B82209F0E8F9002008BD6C18FF1F95
:1098D00008B50348D0F8B82209F0CAF9002008BD3D
:1098E0006C18FF1F08B5024809F0BFF9002008BD39
:1098F0006C18FF1F08B5024809F0B4F9002008BD34
:109900006C18FF1F08B5024809F0AAF9002008BD2D
:109910006C18FF1F08B5024809F08EF9002008BD39
:109920006C18FF1F014809F06EB900BF6C18FF1FCB
:1099300038B522210A480A4C09F0ADF810B9204682
:1099400009F04CF9074BD4F89002DD682B681B69CD
:1099500098472B68D4F894021B699847012038BDBA
:109960006C18FF1F847E0200022804BF0C4B93F882
:10997000D80038B90B4BDB681B685B690A4AD2F820
:1099800098021847012809D1054B93F8D830012BCC
:1099900004D1044BDB681B689B69EFE7704700BF8D
:1099A0006434FF1F847E02006C18FF1F222970B5EB
:1099B0000446154600F0FC8200F28E800E2900F06D
:1099C0001C8241D8062900F0A98119D8022900F08B
:1099D0005E8107D8002900F03D81012900F049810E
:1099E00004243DE1042900F0728140F261810028E5
:1099F00040F08D812621B94809F04DF828602FE10B
:109A00000A2900F0BA810FD8072900F09F810829A0
:109A1000E6D1002840F0F9853521B04809F03BF83F
:109A2000C0F3402028601BE10C2900F0C08140F207
:109A3000B2813421A948002C40F0D18109F02BF8E3
:109A400000F0010028600BE1152900F02A821FD8E0
:109A5000112900F0F5810DD80F2900F0DC811029C3
:109A6000BED1002840F0E58125219C4809F013F87B
:109A70002860F5E0132900F0FF8140F2EF81002813
:109A800040F008822B21954809F005F82860E7E0AE
:109A90001B2900F041820DD8172900F010821829E7
:109AA0009ED1002840F0318233218C4808F0F3FF2A
:109AB0002860D5E01D2900F05F82C0F04582212991
:109AC0008ED1002840F064820146844808F0E3FF0C
:109AD00000F001002860C3E0AE2900F0238453D8D1
:109AE000A72900F08A832AD8A32900F0D98210D8A8
:109AF0008C2900F07782A2297FF472AF6C2177481D
:109B0000002C40F0BE8208F0C6FFC0F3C1302860D0
:109B1000A6E0A52900F0F48240F2DA826C216F48B9
:109B200008F0B9FF00F48046002C40F04583002E79
:109B300000F03783000900F07000286090E0AA2947
:109B400000F09A8310D8A82900F06E83A9297FF429
:109B500047AF6D216148002C40F07D8308F09BFFEA
:109B6000C0F3413028607BE0AC2900F0B58340F2BF
:109B70009B836D215948002C40F0C58308F08BFF72
:109B8000C0F3006028606BE0BB2900F0888436D801
:109B9000B62900F015841FD8B42900F0E283B52956
:109BA0007FF41EAF34214D48002C40F0E78308F0CD
:109BB00072FF430540F1E0831421484808F06BFF31
:109BC000474B30B14FF08072B2FBF0F0834228BFB8
:109BD00003462B60002443E0B92900F0238400F2FF
:109BE0003984B8297FF4FCAE6C213C48002C40F04D
:109BF0000A8408F050FFC0F34030286030E0CC29E0
:109C000000F0C68412D8BF2900F07E84C02900F07D
:109C10009B84BC297FF4E4AE70213048002C40F0D6
:109C2000668408F038FFC0B2286019E0D12900F03E
:109C3000C984D22900F0D684CE297FF4D1AE002881
:109C400040F0F2846F21254808F025FFC0F3090099
:109C5000286005E030B92D21204808F01CFF28605D
:109C6000204670BD12681D482D2108F006FF002413
:109C7000F6E728B92121194808F00DFF2860EFE721
:109C800012681648212108F0F8FE0024E8E728B9F8
:109C90002721124808F0FFFE2860E1E712680F480C
:109CA000002AB8BF5242272108F0E7FE0024D7E778
:109CB000002840F0A7842221084808F0ECFE10F4A8
:109CC000000318BF4FF07F4318432860C8E7034ED6
:109CD00040B9D6F8B8321360C2E700BF6C18FF1F56
:109CE000FFFF0F001368A848002BB8BF5B4220217C
:109CF000C6F8B83208F0CFFE044608B10024AFE73A
:109D0000D6F8B822A048272108F0B7FEA8E71268C5
:109D10009D48262108F0B1FE0024A1E710219A48B1
:109D20002CB908F0B8FEC0F30420286098E708F0CA
:109D3000B2FE2B681B0203F4F85320F4F8521A43C6
:109D40001021914808F099FE002489E710218E48DF
:109D50002CB908F0A0FE00F01F00286080E708F092
:109D60009AFE2B6820F01F0203F01F031A431021F4
:109D7000854808F082FE002472E7002840F04884FD
:109D80003521814808F087FE10F0020F0CBF012337
:109D900000232B6064E7002840F03D8435217A4899
:109DA00008F079FEC04300F00100286058E7342134
:109DB00075482CB908F06FFEC0F3400028604FE7EB
:109DC00008F069FE2B685B0003F0020320F002023A
:109DD0001A4334216C4808F050FE002440E708F094
:109DE0005AFE2B6820F0010203F001031A433421CC
:109DF000654808F042FE002432E728B93421624861
:109E000008F049FE28602BE712685F48342108F00B
:109E100034FE002424E728B924215B4808F03BFEE7
:109E200028601DE712685848242108F026FE002407
:109E300016E712685448252108F01FFE00240FE79A
:109E400028B92821504808F026FE286008E7126843
:109E50004D48282108F011FE002401E728B92A21E5
